:020000040800F2
:1000000000040020E1010008090E00080D0E0008A0
:10001000610E00080D0E0008350E0008E30100080F
:10002000E3010008E3010008E3010008392F00089C
:10003000E3010008E3010008E3010008E301000810
:10004000E3010008E3010008E3010008E301000800
:10005000E3010008E301000899310008C5310008F8
:10006000F13100081D32000849320008E3010008A0
:10007000E3010008E3010008E3010008E3010008D0
:10008000E3010008E3010008E3010008E3010008C0
:10009000E3010008E3010008E301000875320008ED
:1000A000E3010008E3010008E3010008E3010008A0
:1000B000B52F0008E3010008E3010008E301000890
:1000C000E3010008E3010008E3010008E301000880
:1000D000E3010008E3010008E3010008E301000870
:1000E000DD320008E3010008E3010008E301000835
:1000F000E3010008E3010008E3010008E301000850
:10010000E3010008E3010008E3010008E30100083F
:10011000E3010008E3010008E3010008E30100082F
:10012000E3010008E3010008E3010008E30100081F
:10013000E3010008E3010008E3010008E30100080F
:10014000E3010008E3010008E30100088D26000830
:10015000E3010008E3010008E3010008E3010008EF
:10016000E3010008E3010008E3010008E3010008DF
:10017000E3010008E3010008E3010008E3010008CF
:10018000E3010008E3010008E3010008E3010008BF
:10019000E3010008E3010008E3010008E3010008AF
:1001A000E3010008E3010008E3010008E30100089F
:1001B000E3010008E3010008E3010008E30100088F
:1001C000E3010008E3010008E3010008E30100087F
:1001D000E3010008E3010008E3010008E30100086F
:1001E00002E000F000F8FEE772B6394880F30888B4
:1001F000384880F3098838484EF60851CEF200019D
:10020000086040F20000CCF200004EF63471CEF2ED
:1002100000010860BFF34F8FBFF36F8F40F2000003
:10022000C0F2F0004EF68851CEF200010860BFF334
:100230004F8FBFF36F8F4FF00000E1EE100A4EF6C4
:100240003C71CEF200010860062080F31488BFF3F1
:100250006F8F01F0E3FE02F005FE4FF055301F49AD
:100260001B4A91423CBF41F8040BFAE71C49194A6A
:1002700091423CBF41F8040BFAE71A491A4A1B4B5A
:100280009A423EBF51F8040B42F8040BF8E70020F5
:100290001749184A91423CBF41F8040BFAE701F0B4
:1002A000C1FE02F03BFE144C144DAC4203DA54F88C
:1002B000041B8847F9E700F03FF8114C114DAC42A0
:1002C00003DA54F8041B8847F9E701F0A9BE0000DF
:1002D000000400200024002000000008000000208E
:1002E00000040020F036000800240020282400200C
:1002F0002824002018300020E0010008E001000858
:10030000E0010008E00100082DE9F04F2DED108A12
:10031000C1F80CD0C3689D46BDEC108ABDE8F08FD3
:10032000002383F311882846A047002001F0FAFA41
:1003300001F0AAFA00DFFEE71A4B6FF0790270B500
:1003400000241A700F225C709C70DC701C715C7150
:100350009C71DC711C725C729A72DC7201F030FE6E
:10036000064601F055FE054650B90F4B9E4217D088
:1003700001339E4241F2883412BF05460024012514
:10038000002001F027FE0DB100F0B4F800F010FDE0
:1003900000F0F4FB204600F00BF900F0ABF8F9E7B1
:1003A0000446EDE728240020010007B008B500F05E
:1003B00087FBA0F120035842584108BD07B5054B03
:1003C00002211B88ADF8043001A800F0C7FB03B080
:1003D0005DF804FBC0330008064991F8243033B1BE
:1003E00000230822086A81F8243000F0E9BB0120CC
:1003F000704700BF482400202DE9F84F234C94F8A3
:1004000024300546884617468BBB2E46DFF87C9085
:10041000002F38D094F824A0BAF1000F05D1202283
:10042000FF214846266200F0B1FCCAF10805BD4232
:1004300028BF3D465FFA85FBAD0041462A4604EBE6
:100440008A0000F079FC94F82430A7EB0B079B445A
:100450005FFA8BFBBBF1080F2E44A844FFB284F86F
:1004600024B0D5D1FFF7B8FF0028D1D108E0266A23
:1004700006EB8306B042C9D0FFF7AEFF0028C4D117
:100480000020BDE8F88F0120BDE8F88F4824002047
:1004900010B5202383F311881248C3680BB101F013
:1004A000C7FA0023104A0F484FF47A7101F084FA1A
:1004B000002383F311880D4C236813B12368013B9B
:1004C0002360636813B16368013B6360084B1B786A
:1004D00033B9636823B9022000F024FC322363603F
:1004E00010BD00BF342400209104000878250020AE
:1004F0007024002010B5254B254953F8042F0132F4
:1005000000D110BD8B42F8D1224C234B22689A4275
:100510003AD9224B9B6803F1006303F580339A427A
:1005200032D2002000F044FB1D4B0220187000F076
:10053000F1FB1C4B1A6C00221A64196E1A66196EB4
:10054000596C5A64596E5A665A6E5A6942F0800262
:100550005A615A6922F080025A615A691A6942F056
:1005600000521A611A6922F000521A611B6972B6B0
:100570000D4A0E4B13601B682268202181F31188FD
:100580009D4683F30888104710BD00BFFCFF00089C
:100590001C00010804000108FFFF000828240020B7
:1005A000702400200038024008ED00E0000001083F
:1005B0002DE9F04F99B0B34C01902022FF2110A8F3
:1005C000A66800F0E3FBB04A1378A346A3B9AF488E
:1005D0000121C3601170202383F31188C3680BB11C
:1005E00001F026FA0023AA4AA8484FF47A7101F0D4
:1005F000E3F9002383F31188019B13B1A54B019A02
:100600001A60A54AA349019F0292002313704B6010
:1006100099461C461D469846012000F07BFB002FA2
:1006200000F012829B4B1B68002B40F00D8219B02A
:10063000BDE8F08F0220FFF7B9FE002840F0FB81F3
:10064000019BB9F1000F08BF1F46944B1B88ADF802
:100650002C3002210BA800F081FADDE74FF47A700C
:1006600000F02EFA031E0393EADB0220FFF79EFE42
:1006700082460028E4D0039B581E042800F2DD8146
:10068000DFE800F0030E1114170018A8052340F846
:10069000343D042100F062FA54464FF0000856E061
:1006A00004217848F6E704217D48F3E704217D48DA
:1006B000F0E71C24204600F07DFA04340B9004215E
:1006C0000BA800F04BFA2C2CF4D1E5E7002DB7D0A5
:1006D000002CB5D00220FFF769FE0546002800F087
:1006E000AF8101206C4C00F063FA0220207000F012
:1006F00011FB4FF000095FFA89FA504600F068FAE2
:10070000074658B1504600F073FA09F10109002874
:10071000F1D12C46A9460027634B97E7012302201D
:10072000237000F0EDFA3E46DBF808309E4206D218
:10073000304600F03FFA0130EBD10436F4E7029B7B
:1007400000261E70534BA9465E602C46374600F0CB
:1007500025FB15B1002C18BF0027FFF72FFE5BE724
:10076000002D3FF46DAF002C3FF46AAF029B0220D6
:10077000187000F0CFFA322000F0A2F9B0F1000AB0
:10078000C0F25E811AF0030540F05A81DBF80820C0
:1007900006EB0A03934200F25381BAF5807F00F220
:1007A0004F8155450DDA4FF47A7000F089F90490C5
:1007B000049B002BC0F244813C4A049BAB5401359E
:1007C000EFE7C820FFF7F2FD0546002800F038816A
:1007D0001F2E11D8C6F12004544528BF544610AB33
:1007E00026F0030022463149184400F0A5FA2246BB
:1007F000FF212E4800F0CAFA4FEAAA0A5FFA8AF2ED
:100800002A493046FFF7F8FD0446002800F01A8117
:1008100006EB8A0605469AE70220FFF7C7FD002887
:100820003FF40EAFFFF7D8FD00283FF409AF4FF0BB
:10083000000A5346DBF8082092451CD2BAF11F0F7C
:1008400012D8109A01320FD02AF0030218A90A44D4
:1008500052F8202C0B92184604220BA900F014FB2E
:100860000AF1040A0346E5E75046039300F0A2F9B3
:10087000039B0B90EFE718A8042140F84C3D00F0D3
:100880006DF964E72824002074250020342400201A
:10089000910400087825002070240020C23300084D
:1008A0002C24002030240020C433000874240020AD
:1008B00018A8002340F8343D642100F02BF90028EB
:1008C0007FF4BEAE0220FFF771FD00283FF4B8AE02
:1008D0000B9800F09FF918AB43F8480D0421184617
:1008E000CDE718A8002340F8343D642100F012F948
:1008F00000287FF4A5AE0220FFF758FD00283FF442
:100900009FAE0B9800F094F918AB43F8440DE5E75F
:100910000220FFF74BFD00283FF492AE00F08EF965
:1009200018AB43F8400DD9E70220FFF73FFD002840
:100930003FF486AE0BA9142000F086F9824618A871
:10094000042140F83CAD00F009F951460BA896E7A8
:10095000322000F0B5F8B0F1000AFFF671AE1AF0DF
:10096000030F7FF46DAEDBF808200AEB0803934217
:100970003FF666AE0220FFF719FD00283FF460AE97
:100980002AF0030AC244D0453FF4E1AE404600F0ED
:1009900011F904210A900AA800F0E0F808F104080F
:1009A000F1E74FF47A70FFF701FD00283FF448AEFD
:1009B000FFF712FD00283FF4AFAE109B01330CD0BF
:1009C000082210A90020FFF717FD00283FF4A4AE6D
:1009D0002022FF2110A800F0D9F9FFF7EFFC3748DB
:1009E00000F0A6FF23E6002D3FF42AAE002C3FF4D2
:1009F00027AE18A8002340F8343D642100F08AF89F
:100A0000824600287FF41CAE0220FFF7CFFC0028AE
:100A10003FF416AE0390FFF7D1FC41F2883000F0AE
:100A200087FF0B9800F0EEF900F0B8F9039B5746EA
:100A30001C461D46F0E5054689E64FF00008FFE537
:100A40002546FDE52C4667E6002000F039F80490C5
:100A5000049B002BFFF6E3AD012000F051F9049B4D
:100A6000213B122B3FF6D8AD01A252F823F000BF74
:100A7000350600085D060008CD06000819060008C6
:100A80001906000819060008610700085109000846
:100A900019080008B1080008E30800081109000857
:100AA000190600082909000819060008A30900080A
:100AB0004F07000819060008E7090008A086010092
:100AC00037B5114B1A780132D2B20024012A0146FF
:100AD0008DF8074011D80D4803681D6A4FF47A73EA
:100AE0004B4301220DF10701A847012805D1084B0E
:100AF0009DF807001C7003B030BD4FF4FA7000F091
:100B000017FF4FF0FF30F6E70024002048260020B2
:100B10008425002038B50E4B1A780132D2B2012A52
:100B200005460ED80B4803681C6A4FF47A734B4392
:100B300004222946A047042803D1074B002018703F
:100B400038BD4FF4FA7000F0F3FE4FF0FF3038BDBF
:100B500000240020482600208425002030B4054CC5
:100B60002368DD69044B0A46AC460146204630BC8A
:100B7000604700BF48260020A086010070B501F044
:100B800023F9094C094E20700025306823788342F0
:100B900008D901F013F9336805440133B5F5803FF6
:100BA0003360F2D370BD00BF852500208025002072
:100BB00001F0B8B900F1006000F5803000687047BE
:100BC00000F10060920000F5803001F043B90000B0
:100BD000054B1A68054B1B789B1A834202D91044B7
:100BE00001F0ECB80020704780250020852500200A
:100BF00038B5074D04462868204401F0E7F828B9C5
:100C000028682044BDE8384001F0F8B838BD00BF7E
:100C10008025002010F0030308D1B0F5007F05D82F
:100C200000F10050A0F508400068704700207047B0
:100C3000014BC058704700BF107AFF1F014B186866
:100C4000704700BF002004E070B52A4B1C68C4F355
:100C50000B03240C63B140F21342934231D040F2B3
:100C6000194293422FD040F2214293422DD10323C7
:100C7000214A0C2505FB03235D6893F9082042F205
:100C800001039C4224D0B4F5805F23D041F20103DC
:100C90009C4221D041F203039C421FD041F2070342
:100CA0009C4208BF3122441E0C44013D0B46A34226
:100CB0001ED215F9016F581C96B1034600F8016C5D
:100CC000F5E70123D4E70223D2E73F220B4DD6E715
:100CD0003322E3E74122E1E75A22E4E75922E2E73F
:100CE0002C2584421D7001D9981C5A70401A70BD81
:100CF0001846FBE7002004E0D4330008C83300089E
:100D0000022802BF024B4FF400129A61704700BFE5
:100D100000040240022802BF014B20229A61704762
:100D200000040240022801BF024A536983F02003F5
:100D3000536170470004024010B50023934203D072
:100D4000CC5CC4540133F9E710BD000030B5441E3B
:100D500014F9010F0B4660B193F90050854201F17F
:100D6000010106D11AB993F90020801A30BD013A69
:100D7000EEE7002AF7D1104630BD000002460346D8
:100D8000981A13F9011B0029FAD17047024403464F
:100D9000934202D003F8011BFAE77047024B1A781E
:100DA000024B1A70704700BF8425002000240020E9
:100DB00038B5104D104C284600F002F9214628465F
:100DC00000F02AF924680D48626DD2F8043843F027
:100DD0000203C2F8043800F0ABFD0949204600F0D8
:100DE00027FA626DD2F8043823F00203C2F80438FF
:100DF00038BD00BF48260020A034000840420F0044
:100E0000C834000870470000FEE7000000B59BB042
:100E1000EFF3098168226846FFF78EFFEFF3058341
:100E2000034B9A6B9A6A9A6A9A6A9A6A9B6AFEE775
:100E300000ED00E000B59BB0EFF309816822684641
:100E4000FFF77AFFEFF30583044B9A6B9A6A9A6A6D
:100E50009A6A9A6A9A6A9B6AFEE700BF00ED00E010
:100E600000B59BB0EFF3098168226846FFF764FF85
:100E7000EFF30583034B5A6B9A6A9A6A9A6A9A6AE5
:100E80009B6AFEE700ED00E030B5084D0A44914250
:100E90000BD011F8013B09245840013CF7D040F336
:100EA00000032B4083EA5000F7E730BD2083B8ED04
:100EB000002304491A465A50C8180833802B426050
:100EC000F9D170478825002002684368114301600A
:100ED00003B118477047000013B5446BD4F894343D
:100EE0001A681178042915D1217C022912D11979A7
:100EF000128901238B4013420CD101A904F14C004B
:100F000001F02AFED4F89444019B2179024620681E
:100F100000F0DAF902B010BD143001F0ADBD0000F0
:100F20004FF0FF33143001F0A7BD00004C3001F04A
:100F30007FBE00004FF0FF334C3001F079BE00005F
:100F4000143001F07BBD00004FF0FF31143001F090
:100F500075BD00004C3001F04BBE00004FF0FF3279
:100F60004C3001F045BE0000D0F8942438B5136829
:100F700019780429054601D0012038BD017C0229D9
:100F8000FAD112795C89012090400440F4D105F136
:100F9000140001F00DFD02460028EDD0D5F8945460
:100FA0004FF480732868697900F07CF9204638BDD9
:100FB000406BFFF7D9BF000000207047704700006A
:100FC0007FB5124B0360002343608360C36001253B
:100FD00002260F4B057404460290019300F184022F
:100FE000294600964FF48073143001F0BDFC094B84
:100FF0000193029400964FF4807304F523722946FE
:1010000004F14C0001F084FD04B070BD24340008EC
:10101000B10F0008D90E00080B68202282F3118856
:101020000A7903EB820290614A79093243F822007F
:101030008A7912B103EB8203986102230374C0F82A
:101040009414002383F311887047000038B5037FA0
:10105000044613B190F85430ABB9201D012502218C
:10106000FFF732FF04F1140025776FF0010100F063
:1010700087FC84F8545004F14C006FF00101BDE886
:10108000384000F07DBC38BD10B501210446043065
:10109000FFF71AFF0023237784F8543010BD0000B7
:1010A00038B504460025143001F076FC04F14C00FC
:1010B000257701F045FD201D84F854500121FFF7EC
:1010C00003FF2046BDE83840FFF74EBF90F844309C
:1010D00003F06003202B19D190F84520212A0AD073
:1010E000222A4FF000030ED0202A0FD1084A826333
:1010F0000722C26304E0064B83630723C363002314
:101100000364012070478363C363F9E700207047DD
:1011100001240020D0F8943437B51A6811780429D6
:1011200004461AD1017C022917D1197912890123A9
:101130008B40134211D100F14C05284601F0C0FD4F
:1011400058B101A9284601F007FDD4F89444019B49
:1011500021790246206800F0B7F803B030BD0000E6
:1011600000EB8103F7B59C6905460E46F4B12023D8
:1011700083F3118805EB8607201D0821FFF7A4FEE5
:10118000FB685B691B684C3413B1204601F0F2FC2C
:1011900001A9204601F0E0FC024648B1019B31461E
:1011A000284600F091F8002383F3118803B0F0BDC6
:1011B000FB685A691268002AF5D01B8A013B13406C
:1011C000F1D105F14402EAE7093138B550F8214080
:1011D000DCB1202383F31188D4F894241368527966
:1011E00003EB8203DB689B695D6845B104216018ED
:1011F000FFF76AFE294604F1140001F0E3FB2046E4
:10120000FFF7B2FE002383F3118838BD704700005A
:1012100000F08EBF0123037000234360C36183622B
:101220000362C3624362036303814381704700002A
:1012300038B50446202383F3118800254160C5603A
:1012400005614561856100F083FF0223237085F30A
:10125000118838BD70B500EB810305465069DA602E
:101260000E46144618B110220021FFF78FFDA06929
:1012700018B110220021FFF789FD31462846BDE84C
:10128000704001F02FB80000028902F001020281D3
:10129000428902F0010242810022026142618261C0
:1012A00001F0B4B8F0B400EB81044789E46801258B
:1012B000A4698D403D43458123600023A2606360A3
:1012C000F0BC01F0CFB80000F0B400EB8104078956
:1012D000E468012564698D403D4305812360002356
:1012E000A2606360F0BC01F049B9000070B5022350
:1012F000002504460370A0F84C5080F84E5080F84A
:101300004F5005814581C56005614561856180F863
:10131000345000F083FF63681B6823B129462046E0
:10132000BDE87040184770BD436802781B6880F8BC
:101330005020052202700BB10421184770470000AD
:10134000436890F850201B6802700BB105211847C4
:101350007047000090F8343070B5044613B1002394
:1013600080F8343004F14402204601F071F86368DB
:101370009B6863BB94F8445015F0600615D194F84F
:10138000453005F07F0545EA032540F202339D42D2
:1013900000F00E815BD8022D00F0DC803FD8002DDC
:1013A00000F08780012D00F0CF800021204601F061
:1013B000A7FA0021204601F099FA63681B6813B16F
:1013C000062120469847062384F8343070BD204615
:1013D00098470028CED094F84B2094F84A3043EA3E
:1013E0000223E26B934238BFE36394F94430E56B28
:1013F000002B4FF0200380F2FD80002D00F0EC80E8
:10140000092284F8342083F311880021E36BA26B56
:101410002046FFF759FF002383F3118870BDB5F50F
:10142000817F00F0B180B5F5407F49D0B5F5807F70
:10143000BBD194F84630012BB7D1B4F84C3023F02F
:101440000203A4F84C30A663E6632664C3E740F2C7
:1014500001639D421ED8B5F5C06F3BD2B5F5A06FB4
:10146000A3D1B4F84430B3F5A06F0ED194F8463050
:1014700084F84E30204600F029FF63681B6813B1E2
:10148000012120469847032323700023A363E363CD
:101490002364A0E7B5F5106F32D040F602439D42B9
:1014A00052D0B5F5006F80D104F14F03A36301233F
:1014B00024E004F14C03A3630223E36325648AE779
:1014C00094F84630012B7FF470AFB4F84C3043F001
:1014D0000203B6E794F84920616894F848304D68F3
:1014E00094F8471043EA0223204694F84620A84780
:1014F00000283FF45AAF4368A3630368E363A4E79B
:101500002378042B10D1202383F311882046FFF782
:10151000BBFE86F31188636884F84F601B68032163
:1015200021700BB12046984794F84630002BACD080
:1015300084F84F300423237063681B68002BA4D009
:10154000022120469847A0E7374BA3630223E363B9
:1015500000239DE794F8481011F0800F204601F019
:101560000F010ED000F066FF012806D002287FF49C
:101570001CAF2E4BA363E06367E72D4BA363E563CA
:1015800063E700F049FFEFE794F84630002B7FF463
:101590000CAF94F8483013F00F013FF476AF1A0601
:1015A000204602D501F0C0F96FE701F0B3F96CE70E
:1015B00094F84630002B7FF4F8AE94F8483013F0DE
:1015C0000F013FF462AF1B06204602D501F098F9E7
:1015D0005BE701F08BF958E7142284F8342083F399
:1015E00011882B462A4629462046FFF75BFE85F3E5
:1015F000118870BD5DB1152284F8342083F3118801
:101600000021E36BA26B2046FFF74CFE03E70B22A1
:1016100084F8342083F311882B462A462946204635
:10162000FFF752FEE3E700BF543400084C340008D3
:101630005034000838B590F834300446152B29D8BA
:10164000DFE803F03E28282828283E28280B2939DF
:1016500028282828282828283E3E90F84B1090F863
:101660004A20C36B42EA01229A4214D9C268128A04
:10167000B3FBF2F502FB15356DB9202383F3118816
:101680002B462A462946FFF71FFE85F311880A23B9
:1016900084F8343038BD142384F83430202383F3A5
:1016A000118800231A4619462046FFF7FBFD002348
:1016B00083F3118838BD036C03B198470023E7E733
:1016C000002101F01DF90021204601F00FF96368A7
:1016D0001B6813B10621204698470623D8E700006F
:1016E00090F83420152A38B5044622D801239340B7
:1016F00040F6416213421DD113F480150FD19B02B5
:1017000017D50B2380F83430202383F311882B4620
:101710002A462946FFF7D8FD85F3118838BDC368EE
:101720009B695B682BB9036C03B19847002384F86D
:10173000343038BD002101F0E3F80021204601F0EB
:10174000D5F863681B6813B1062120469847062325
:10175000EDE70000024B00221B605B609A6070475F
:1017600008260020002303748268054B1B689968D3
:101770009142FBD25A680360426010605860704723
:101780000826002008B5202383F31188037C032B4F
:1017900005D0042B0DD02BB983F3118808BD436904
:1017A00000221A604FF0FF334361FFF7DBFF002395
:1017B000F2E790E80C001A6002685360F2E700005C
:1017C000002303748268054B1B6899689142FBD81B
:1017D0005A68036042601060586070470826002015
:1017E000054B19690874186802681A60536018611B
:1017F00001230374FEF788BD0826002030B54B1C7A
:1018000087B005460A4C10D023690A4A01A800F0A7
:10181000D3F82846FFF7E4FF049B13B101A800F0BA
:1018200007F92369586907B030BDFFF7D9FFF8E71A
:10183000082600208517000838B50C4D41612B693A
:1018400081689A689142044603D8BDE83840FFF7A2
:1018500089BF1846FFF786FF01232C6101462374D8
:101860002046BDE83840FEF74FBD00BF08260020E7
:10187000044B1A681B6990689B68984294BF0020CB
:10188000012070470826002010B5084C2368206905
:101890001A6822605460012223611A74FFF790FFD6
:1018A00001462069BDE81040FEF72EBD0826002045
:1018B0008260022202740022427470478368A3F19E
:1018C0007C0243F80C2C026943F83C2C426943F833
:1018D000382C074A43F81C2CC26843F8102C02220B
:1018E00003F8082C002203F8072CA3F11800704716
:1018F0002103000810B5202383F31188FFF7DEFFD2
:1019000000210446FFF798FF002383F31188204647
:1019100010BD0000024B1B6958610F20FFF760BF2C
:1019200008260020202383F31188FFF7F3BF00006F
:1019300008B50146202383F311880820FFF75EFFD6
:10194000002383F3118808BD49B1064B42681B6927
:1019500018605A60136043600420FFF74FBF4FF0D8
:10196000FF307047082600200368984206D01A68A6
:101970000260506059611846FFF7F4BE70470000DE
:1019800038B504460D462068844200D138BD03684E
:1019900023605C604561FFF7E5FEF4E7054B03F16A
:1019A00014025A619A614FF0FF32DA6100221A6222
:1019B000704700BF08260020F8B503614FF0804350
:1019C000C2605C6A194B1A46022952F8145F38BF8C
:1019D0000221954206461F460AD1586198611C6251
:1019E0000560456081600819BDE8F84001F08AB9DA
:1019F000186AAB68241A0C1902D3E41A2D6804E0A3
:101A00009C4202D2204401F08BF9AB689C42F4D88E
:101A10006B68736035601E606E60B460A9684FF0DB
:101A2000FF33091BA960FB61F8BD00BF0826002039
:101A300010B41B4C234653F8141F814210D0416848
:101A400002680A60026851609A424FF00001C1606A
:101A500003D0936881680B4493605DF8044B704732
:101A60000A68626100209A425360C86003D15DF841
:101A7000044B01F04FB993688868034493604FF0BA
:101A80008042206A526A121A9342E6D9991A0129B1
:101A900098BF931C18445DF8044B01F041B900BF96
:101AA0000826002000207047FEE700007047000075
:101AB0004FF0FF3070470000022906D0032906D0FE
:101AC0000129064818BF0020704705487047032ABF
:101AD0009ABF044800EBC20000207047243500087C
:101AE000D83400080824002070B59AB001AD06462D
:101AF00008462946144600F095F82846FFF73EF9B7
:101B0000C0B2431C5B0086E8180023700323637097
:101B1000002302341946DAB2904204F1020401D8DB
:101B20001AB070BDEA5C04F8022C04F8011C013301
:101B3000F1E7000008B5202383F311880348FFF77D
:101B4000E9FA002383F3118808BD00BF482600206E
:101B500010B50446052916D8DFE801F0161503165E
:101B6000161D202383F311880E4A0121FFF772FB13
:101B700020460D4A0221FFF76DFB0C48FFF790FA53
:101B8000002383F3118810BD202383F311880748B5
:101B9000FFF75CFAF4E7202383F311880348FFF78B
:101BA00073FAEDE7583400087C340008482600201A
:101BB00038B50C4D0C4C0D492A4604F10800FFF7CE
:101BC00093FF05F1CA0204F110000949FFF78CFFE9
:101BD00005F5CA7204F118000649BDE83840FFF760
:101BE00083BF00BF102B002008240020A834000869
:101BF000B2340008BD34000870B5044608460D46EE
:101C0000FFF7BCF8C6B22046013403780BB918467A
:101C100070BD32462946FFF799F80028F3D101201C
:101C200070BD00002DE9F84F05460C46FFF7A6F8F9
:101C30002C49C6B22846FFF7DFFF08B10436F6B2DA
:101C400029492846FFF7D8FF08B11036F6B2632EAF
:101C50000DD8DFF89090DFF890A0DFF89880DFF8DB
:101C600098B0224F2E7846B92670BDE8F88F2946E5
:101C70002046BDE8F84F01F09BBB252E2DD1072251
:101C800049462846FFF762F850B93B6823607B68F5
:101C900063603B892381BB7AA37207350B34E1E78C
:101CA000082251462846FFF751F8B0B9104BA21C44
:101CB00013F8011F09095B4511F8081002F8021C0E
:101CC000197801F00F0102F1020211F8081002F870
:101CD000031CEDD118340835C4E7267001350134F2
:101CE000C0E700BF44350008BD3400084C3500088B
:101CF0000F7AFF1F583500081B7AFF1FBFF34F8F65
:101D0000024AD368DB03FCD4704700BF003C0240AA
:101D100008B5094B1B7873B9FFF7F0FF074B1A6939
:101D2000002ABFBF064A5A6002F188325A601A6818
:101D300022F480621A6008BD6E2D0020003C024033
:101D40002301674508B50B4B1B7893B9FFF7D6FF06
:101D5000094B1A6942F000421A611A6842F4805233
:101D60001A601A6822F480521A601A6842F480627B
:101D70001A6008BD6E2D0020003C02400B2870B593
:101D800013D80B4A0B4C137863B90B4E4FF000611C
:101D900044F8231056F8235001330C2B2944F7D173
:101DA0000123137054F8200070BD002070BD00BFE7
:101DB000A02D0020702D00206C350008014B53F839
:101DC000200070476C3500080C2070470B2810B5B8
:101DD000044601D9002010BDFFF7D0FF064B53F891
:101DE00024301844C21A0BB9012010BD1268013208
:101DF000F0D1043BF6E700BF6C3500080B2810B5A6
:101E0000044621D8FFF77AFFFFF782FF0F4AF3233A
:101E1000D360C300DBB243F4007343F002031361E9
:101E2000136943F480331361FFF768FFFFF7A6FFE0
:101E3000074B53F8241000F0DDF8FFF783FF20462E
:101E4000BDE81040FFF7C2BF002010BD003C0240BB
:101E50006C3500082DE9F84312F00103154640D116
:101E60008218B2F1016F3CD22C4B1B6813F00103B6
:101E700037D02B4CFFF74CFFF323E360FFF73EFF17
:101E800040F20127032D01D9830713D0244C0F46BC
:101E9000401A40F20118EB1B0B44012B00EB070624
:101EA000236924D823F001032361FFF74BFF0120AE
:101EB000BDE8F883236923F44073236123693B431E
:101EC000236151F8046B0660BFF34F8FFFF716FFD5
:101ED00003689E4208D0236923F001032361FFF7C2
:101EE00031FF0020BDE8F883043D0430CAE723F445
:101EF00040732361236943EA08032361B94637F835
:101F0000023B3380BFF34F8FFFF7F8FE3688B9F8F6
:101F10000030B6B2B342BED0DDE700BF00380240A9
:101F2000003C0240084908B50B7828B153B9FFF7C7
:101F3000EFFE01230B7008BD23B1BDE80840087017
:101F4000FFF700BF08BD00BF6E2D002010B5024492
:101F5000064B0439D2B2904200D110BD441C00B2ED
:101F600053F8200041F8040FE0B2F4E75028004095
:101F7000104B30B51C6F240407D41C6F44F400745C
:101F80001C671C6F44F400441C670B4C236843F42B
:101F9000807323600244094B0439D2B2904200D1CD
:101FA00030BD441C00B251F8045F43F82050E0B249
:101FB000F4E700BF003802400070004050280040A5
:101FC00007B5012201A90020FFF7C0FF019803B067
:101FD0005DF804FB13B50446FFF7F2FFA04206D0FC
:101FE00002A9012241F8044D0020FFF7C1FF02B011
:101FF00010BD000070470000034B1B689B0042BFF0
:10200000024B01221A70704774380240A12D002043
:10201000014B1878704700BFA12D002070470000C9
:10202000FEE70000084A094B09498B4204D3094ADC
:102030000021934205D3704752F8040F43F8040B74
:10204000F3E743F8041BF4E71437000818300020C6
:102050001830002018300020836D30B500229D68B4
:10206000446D11464FF0FF3004EB421301329542AC
:10207000C3F80019C3F81019C3F80809C3F8001B06
:10208000C3F8101BC3F8080BEED24FF00113C4F8CD
:102090001C3830BD890141F02001016103699B06B4
:1020A000FCD4122000F0C4BE204B03EB80022DE9CB
:1020B000F047D2F80CE05D6DDEF81420461CD2F833
:1020C00000C005EB063605EB4018516861450BD39F
:1020D000D5F83428012303FA00F022EA0000C5F8FD
:1020E00034081846BDE8F087BEF81040ACEB010399
:1020F000A34228BF2346D8F81849A4B2B3EB840FF3
:1021000010D894681F46A4F1040959F804AFC6F822
:1021100000A0042F01D9043FF7E71C440B4494604E
:102120005360D2E70020BDE8F08700BFA42D002057
:1021300010B5054C2046FFF76DF84FF0A0436365DE
:10214000024BA36510BD00BFA42D0020C0350008C0
:102150000378012B70B5054650D12A4B446D984247
:102160001BD1294B5A6B42F080025A635A6D42F0E0
:1021700080025A655A6D5A6942F080025A615A6962
:1021800022F080025A610E2143205B6900F0D6FBE9
:102190001E4BE3601E4BC4F800380023C4F8003E19
:1021A000C02323606E6D4FF40413A3633369002BC7
:1021B000FCDA012333610C2000F03AFE3369DB07BF
:1021C000FCD4122000F034FE3369002BFCDA002628
:1021D000A6602846FFF740FF6B68C4F81068DB680C
:1021E000C4F81468C4F81C684BB90A4BA3614FF0DB
:1021F000FF336361A36843F00103A36070BD064B26
:10220000F4E700BFA42D0020003802404014004035
:1022100003002002003C30C0083C30C0F8B5446DDB
:10222000054600212046FFF735FFA96D00234FF03A
:1022300001128F68C4F834384FF00066C4F81C28C7
:102240004FF0FF3004EB431201339F42C2F80069A4
:10225000C2F8006BC2F80809C2F8080BF2D20B688A
:102260006A6DEB65636210231361166916F0100640
:10227000FBD1122000F0DCFDD4F8003823F4FE631B
:10228000C4F80038A36943F4402343F01003A3616A
:102290000923C4F81038C4F814380A4BEB604FF027
:1022A000C043C4F8103B084BC4F8003BC4F81069A5
:1022B000C4F80039EB6D03F1100243F48013EA65B2
:1022C000A362F8BD9C35000840800010426D90F874
:1022D0004E10D2F8003823F4FE6343EA0113C2F82B
:1022E000003870472DE9F0410EB200EB86080D462C
:1022F000D8F80C100F6807F00303022B50D0032B03
:1023000050D03D4A3D4F012B18BF1746446D4FEA50
:10231000451E04EB0E030022C3F8102B8A6905F159
:10232000100C002A40D04A8A05F158035B013A4359
:10233000E2500123D4F81C2803FA0CF31343A644FB
:102340004A69C4F81C380023CEF8103905F13F0360
:10235000002A39D00A8A898B9208012988BF4A430A
:10236000C16D04EB8303561841EA0242C665294653
:102370005A602046FFF78EFED8F80C301B8A43EADD
:1023800085531F4305F148035B01E7500123D4F84F
:102390001C2803FA05F51543C4F81C58BDE8F08164
:1023A000174FB3E7174FB1E704EB4613D3F8002BF1
:1023B00022F40042C3F8002BD4F81C28012303FAAE
:1023C0000CF322EA0303BAE704EB83030E4A5A60D4
:1023D00004EB461629462046FFF75CFED6F8003986
:1023E00023F40043C6F80039D4F81C38012202FA5D
:1023F00005F523EA0505CFE70080001000800410F2
:102400000080081000800C1000040002826D126829
:10241000C265FFF721BE00005831436D49015B588A
:1024200013F4004004D013F4001F14BF0120022055
:10243000704700004831436D49015B5813F4004078
:1024400004D013F4001F14BF0120022070470000C5
:1024500000EB8101CB68196A0B6813604B6853600D
:102460007047000000EB810330B5DD68AA6913688E
:10247000D36019B9402B84BF402313606B8A146862
:10248000426D1C44013CB4FBF3F46343033323F07B
:10249000030302EB411043EAC44343F0C043C0F8D6
:1024A000103B2B6803F00303012B09B20ED1D2F8C5
:1024B000083802EB411013F4807FD0F8003B14BFC2
:1024C00043F0805343F00053C0F8003B02EB41124D
:1024D000D2F8003B43F00443C2F8003B30BD00009B
:1024E0002DE9F041244D6E6D06EB40130446D3F800
:1024F000087BC3F8087B38070AD5D6F814381907C3
:1025000006D505EB84032146DB6828465B689847BF
:10251000FA072FD5D6F81438DB072BD505EB840343
:10252000D968CCB98B69488A5E68B6FBF0F200FBCB
:1025300012628AB91868DA6890420DD2121A83E8DA
:102540001400202383F311880B482146FFF78AFFEC
:1025500084F31188BDE8F081012303FA04F26B894A
:1025600023EA02036B81CB6823B121460248BDE810
:10257000F0411847BDE8F081A42D002000EB810355
:1025800070B5DD68436D6C692668E6604A0156BB2C
:102590001A444FF40020C2F810092A6802F003021E
:1025A000012A0AB20ED1D3F8080803EB421410F442
:1025B000807FD4F8000914BF40F0805040F00050F4
:1025C000C4F8000903EB4212D2F8000940F00440BD
:1025D000C2F80009D3F83408012202FA01F10143DC
:1025E000C3F8341870BD19B9402E84BF4020206054
:1025F00020682E8A841940F00050013C1A44B4FB34
:10260000F6F440EAC440C6E7F8B504461E48456DF6
:1026100005EB4413D3F80869C3F80869F10717D527
:10262000D5F81038DA0713D500EB8403D9684B6965
:102630001F68DA68974218D2D21B00271A605F60C1
:10264000202383F311882146FFF798FF87F3118831
:10265000330617D5D5F834280123A340134211D0EF
:102660002046BDE8F840FFF71FBD012303FA04F23E
:10267000038923EA020303818B68002BE8D02146FB
:102680009847E5E7F8BD00BFA42D002096482DE946
:10269000F84F456D6E69AB691E4016F4805F6E6140
:1026A000044605D0FEF722FEBDE8F84F00F054BC0A
:1026B000002E12DAD5F8003E8B489B071EBFD5F8D6
:1026C000003E23F00303C5F8003ED5F8043823F09C
:1026D0000103C5F80438FEF733FE370502D58248FA
:1026E000FEF722FEB0040CD5D5F8083813F0060F1B
:1026F000EB6823F470530CBF43F4105343F4A0531E
:10270000EB60310704D56368DB680BB17648984706
:10271000F2025AD4B3020CD5D4F85480DFF8C8A121
:1027200000274FF00109A36D9B68F9B28B4280F03E
:102730008780F70619D5616D0A6AC2F30A1702F09D
:102740000F0302F4F012B2F5802F00F0A180B2F571
:10275000402F0AD104EB830301F58051DB68186A2E
:1027600000231A469F4240F087803003D5F818486E
:1027700013D5E10302D50020FFF7B2FEA20302D574
:102780000120FFF7ADFE630302D50220FFF7A8FE8C
:10279000270302D50320FFF7A3FE750384D5E007C6
:1027A00002D50020FFF730FFA10702D50120FFF777
:1027B0002BFF620702D50220FFF726FF23077FF5D4
:1027C00073AF0320FFF720FF6EE7D4F85480DFF8E3
:1027D00018A100274FF00109A36D9B685FFA87FBE2
:1027E0005B4597D308EB4B13D3F8002902F4402242
:1027F000B2F5802F22D1D3F80029002A1EDAD3F8AF
:10280000002942F09042C3F80029D3F80029002A99
:10281000FBDB5946606DFFF73DFC228909FA0BF39B
:1028200022EA0303238104EB8B03DB689B6813B16B
:102830005946504698475846FFF736FC0137CBE7D4
:1028400008EB4112D2F8003B03F44023B3F5802F8C
:1028500010D1D2F8003B002B0CDA628909FA01F39F
:1028600022EA0303638104EB8103DB68DB680BB1BD
:1028700050469847013756E79C0708BF0A68072B60
:1028800098BF027003F101039CBF120A013069E78F
:10289000023304EB830201F58051526890690268AB
:1028A000D0F808C04068A2EB000E00221046974204
:1028B0000AD104EB830463689B699A683A449A607E
:1028C0005A6817445F6050E712F0030F08BF0868AA
:1028D000964588BF8CF8000002F1010284BF000A0F
:1028E0000CF1010CE3E700BFA42D0020436D03EBC6
:1028F0004111D1F8003B43F40013C1F8003B70478D
:10290000436D03EB4111D1F8003943F40013C1F8D2
:1029100000397047436D03EB4111D1F8003B23F4BC
:102920000013C1F8003B7047436D03EB4111D1F830
:10293000003923F40013C1F80039704700F16043F7
:1029400000F01F02400903F5614309018000C9B28C
:1029500000F1604083F8001300F5614001239340CB
:10296000C0F880310360704730B5039C01720433B6
:1029700004FB0325C361049B03630021059B0060E6
:102980004060C160426102618561046242628162AD
:10299000C162436330BD00000022416A41610161B0
:1029A000C2608262C2626FF00101FEF7E9BF0000FF
:1029B00003694269934203D1C2680AB1002070479B
:1029C000181D704703691960C2680132C260C2698C
:1029D000134482690361934224BF436A0361002167
:1029E000FEF7C2BF38B504460D46E3683BB16269E5
:1029F000131D1268A3621344E362002038BD237ADA
:102A000033B929462046FEF79FFF0028EDDA38BD8E
:102A10006FF00100FBE70000C368C269013BC360BF
:102A20004369134482694361934224BF436A43610B
:102A300000238362036B03B11847704770B52023EE
:102A4000044683F31188866A3EB9FFF7CBFF05463B
:102A500018B186F31188284670BDA36AE26A13F89C
:102A6000015BA362934202D32046FFF7D5FF002308
:102A700083F31188EFE700002DE9F84F04460E4676
:102A800090469946202787F311880025AA46D4F856
:102A900028B0BBF1000F09D149462046FFF7A2FF3D
:102AA00020B18BF311882846BDE8F88FA16AE36A4C
:102AB000A8EB050B5B1A9B4528BF9B46BBF1400F5B
:102AC0001BD9334601F1400251F8040B43F8040BC3
:102AD0009142F9D1A36A40334036A3624035A26ADD
:102AE000E36A9A4202D32046FFF796FF8AF31188E1
:102AF0004545D8D287F31188C9E730465A46FEF7D4
:102B00001BF9A36A5B445E44A3625D44E7E70000EF
:102B100010B5029C0172043303FB0421C36100233E
:102B20008362C362039B0363049B00604060C460D4
:102B300042610261816104624262436310BD000030
:102B4000026AC260426A4261026100228262C2621B
:102B50006FF00101FEF714BF436902699A4203D185
:102B6000C2680AB100207047184650F8043B0B6059
:102B700070470000C368C2690133C36043691344EE
:102B800082694361934224BF436A43610021FEF797
:102B9000EBBE000038B504460D46E3683BB123693F
:102BA0001A1DA262E2691344E362002038BD237A51
:102BB00033B929462046FEF7C7FE0028EDDA38BDB6
:102BC0006FF00100FBE7000003691960C268013A79
:102BD000C260C269134482690361934224BF436A9D
:102BE000036100238362036B03B118477047000041
:102BF00070B5202304460E4683F31188856A35B9E3
:102C00001146FFF7C7FF10B185F3118870BDA36AA5
:102C10001E70A36AE26A01339342A36204D3E1699E
:102C200020460439FFF7D0FF002080F3118870BDE3
:102C30002DE9F84F04460D4691469A464FF020087C
:102C400088F311880026B346A76A4FB9514620463B
:102C5000FFF7A0FF20B187F311883046BDE8F88F59
:102C6000A06AE76AA9EB06033F1A9F4228BF1F46E6
:102C7000402F1BD905F1400355F8042B40F8042BD5
:102C80009D42F9D1A36A4033A3624036A26AE36A47
:102C90009A4204D3E16920460439FFF795FF8BF38C
:102CA00011884E45D9D288F31188CDE729463A4696
:102CB000FEF742F8A36A3B443D44A3623E44E5E785
:102CC000026943699A4203D1C3681BB91846704729
:102CD0000023FBE7836A002BF8D0043B9B1AF5D056
:102CE0001360C368013BC360C3691A44836902610E
:102CF0009A4224BF436A0361002383620123E5E70C
:102D000000F06CB94FF08043002258631A61022230
:102D1000DA6070474FF080430022DA6070470000AD
:102D20004FF0804358637047FEE7000010B5174C22
:102D3000FEF710FDFEF732FE802215492046FEF711
:102D4000B7FD012344F8180C0374124B124AD968DA
:102D500021F4E0610904090C0A431049DA60CA68E9
:102D600042F08072CA600E490A6842F001020A60AD
:102D70001022DA77202283F82220002383F311889F
:102D800062B60848BDE81040FEF7B4BD302600200A
:102D9000CC35000800ED00E00003FA05F0ED00E09E
:102DA000001000E0D43500082DE9F84F1F4C4FF01B
:102DB0000008656904F11407C1464FF08043266A94
:102DC0005B6AAA689E1B96421DD34FF0200AAA6830
:102DD000236AD5F80CB0134423622B68BB425F60B2
:102DE000A6EB02066361C5F80C8001D1FFF792FFE4
:102DF00089F311882869D8478AF311886569AB6817
:102E00009E42E4D2D9E76269BA420CD0916823624B
:102E10008E1B9660A86802282CBF1818981CBDE865
:102E2000F84FFFF77DBFBDE8F88F00BF08260020F0
:102E3000034B59685A68521A9042FBD8704700BF3A
:102E4000001000E04B6843608B688360CB68C36010
:102E50000B6943614B6903628B6943620B680360D2
:102E60007047000008B5224B22481A6940F2FF1152
:102E70000A431A611A6922F4FF7222F001021A61F0
:102E80001A691A6B0A431A631A6D0A431A651A4AB9
:102E90001B6D1146FFF7D6FF184802F11C01FFF722
:102EA000D1FF174802F13801FFF7CCFF154802F1B6
:102EB0005401FFF7C7FF144802F17001FFF7C2FF8A
:102EC000124802F18C01FFF7BDFF114802F1A80181
:102ED000FFF7B8FF0F4802F1C401FFF7B3FF0E4838
:102EE00002F1E001FFF7AEFFBDE8084000F0E0B8F6
:102EF0000038024000000240F4350008000402409F
:102F000000080240000C0240001002400014024081
:102F100000180240001C02400020024008B500F0EA
:102F200037FAFFF703FFFFF767F8BDE80840FEF741
:102F30003FBE000070470000064A536823F00103BB
:102F40005360EFF30983683383F30988002383F325
:102F50001188704730EF00E010B5202383F311880B
:102F6000104B5B6813F4006318D0F1EE103AEFF3E6
:102F700009844FF0807344F84C3C0B4BDB6844F8F9
:102F8000083CA4F1680383F30988FEF771FC18B1CB
:102F9000064B44F8503C10BD054BFAE783F311880B
:102FA00010BD00BF00ED00E030EF00E0310300088D
:102FB000340300084FF0804310B51A69920708D512
:102FC00000241C61202383F31188FFF7EDFE84F3B6
:102FD0001188BDE81040FFF7BFBF0000104B1A6C0E
:102FE00042F001021A641A6E42F001021A660D4A9A
:102FF0001B6E936843F0010393604FF080435322AC
:103000009A624FF0FF32DA6200229A615A63DA6004
:103010005A6001225A6108211A601C20FFF78EBCF9
:1030200000380240002004E01F4B1A696FEAC252C8
:103030006FEAD2521A611A69C2F308021A614FF09C
:10304000FF301A695A69586100215A6959615A69F1
:103050001A6A62F080521A621A6A02F080521A6288
:103060001A6A5A6A58625A6A59625A6A1A6C42F063
:1030700080521A641A6E42F080521A661A6E0B4A17
:10308000106840F480701060186F00F44070B0F564
:10309000007F1EBF4FF4803018671967536823F410
:1030A0000073536000F054B90038024000700040D3
:1030B000304B4FF080521A642F4A4FF44041116058
:1030C0001A6842F001021A601A689207FCD59A68E1
:1030D00022F003029A60274B19469A6812F00C02FC
:1030E000FBD1186800F0F90018609A601A6842F481
:1030F00080321A600B689B03FCD54B6F43F00103D1
:103100004B671C4B5A6F9007FCD51C4A5A601A68D3
:1031100042F080721A60184A53685904FCD5154B66
:103120001A689201FCD5164A9A60164B1A68164B1B
:103130009A42164B1BD1164A1168164A914216D173
:1031400040F205121A600B4B9A6842F002029A6034
:103150009A6802F00C02082AFAD15A6C42F48042B2
:103160005A645A6E42F480425A665B6E704740F26F
:103170000572E7E70038024000700040085440073D
:1031800000948838002004E011640020003C0240D4
:1031900000ED00E041C20F41084A08B553691168CB
:1031A0000B4003F00103536123B1054A13680BB1CF
:1031B00050689847BDE80840FFF7CEBE003C01408C
:1031C00088250020084A08B5536911680B4003F0B0
:1031D0000203536123B1054A93680BB1D068984745
:1031E000BDE80840FFF7B8BE003C0140882500203C
:1031F000084A08B5536911680B4003F00403536192
:1032000023B1054A13690BB150699847BDE80840DE
:10321000FFF7A2BE003C014088250020084A08B5FF
:10322000536911680B4003F00803536123B1054A49
:1032300093690BB1D0699847BDE80840FFF78CBE91
:10324000003C014088250020084A08B553691168F0
:103250000B4003F01003536123B1054A136A0BB10D
:10326000506A9847BDE80840FFF776BE003C014031
:1032700088250020174B10B55C691A68144004F4C7
:1032800078725A61A30604D5134A936A0BB1D06AC7
:103290009847600604D5104A136B0BB1506B9847E2
:1032A000210604D50C4A936B0BB1D06B9847E2050D
:1032B00004D5094A136C0BB1506C9847A30504D58B
:1032C000054A936C0BB1D06C9847BDE81040FFF7EE
:1032D00043BE00BF003C0140882500201A4B10B5BA
:1032E0005C691A68144004F47C425A61620504D592
:1032F000164A136D0BB1506D9847230504D5134A38
:10330000936D0BB1D06D9847E00404D50F4A136E4E
:103310000BB1506E9847A10404D50C4A936E0BB1C3
:10332000D06E9847620404D5084A136F0BB1506FF2
:103330009847230404D5054A936F0BB1D06F984783
:10334000BDE81040FFF708BE003C01408825002082
:10335000062108B50846FFF7F1FA06210720FFF716
:10336000EDFA06210820FFF7E9FA06210920FFF708
:10337000E5FA06210A20FFF7E1FA06211720FFF7F8
:10338000DDFA06212820BDE80840FFF7D7BA000083
:1033900008B5FFF749FEFDF78BFDFDF739FFFDF797
:1033A0000DFEFFF7C7FDBDE80840FFF7A9BC000010
:1033B000034611F8012B03F8012B002AF9D17047BD
:1033C000121012131211000053544D3332463F3F76
:1033D0003F00000000000000C83300083F0000006C
:1033E00013040000043400083F000000190400002A
:1033F0000E3400083F0000002104000018340008CB
:103400003F00000053544D3332463430780053545B
:103410004D3332463432780053544D3332463434CF
:103420003658580000000000350F0008210F000832
:103430005D0F0008490F0008550F0008410F0008F4
:103440002D0F0008190F0008B90F00080000000038
:103450000100000000000000020000000000000069
:1034600061110008C911000840004000E02A002056
:10347000F02A00200200000000000000030000000D
:10348000000000000D120008000000001000000005
:10349000002B0020000000000100000000000000E0
:1034A000A42D0020010102004172647550696C6F07
:1034B000740025424F415244252D424C002553456E
:1034C0005249414C25000000511B0008B91A000860
:1034D000CD100008351B000843000000E034000850
:1034E00009024300020100C0320904000001020287
:1034F000010005240010010524010001042402023A
:103500000524060001070582030800FF09040100E5
:10351000020A0000000705010240000007058102C1
:1035200040000000120000002C35000812011001BC
:10353000020000400912415700020102030100008D
:103540000403090425424F41524425007370656508
:10355000647962656566340030313233343536372C
:103560003839414243444546000000000040000015
:10357000004000000040000000400000000001008A
:103580000000020000000200000002000000020033
:103590000000020000000200000002000000000025
:1035A0005513000835160008E116000840004000D9
:1035B000042E0020042E002001000000142E002004
:1035C0008000000040010000030000006D61696E92
:1035D00000000000EC350008202E002018300020EC
:1035E00001000000292D00080000000069646C65DE
:1035F000000000000000800200000000AAAAAAAAA1
:1036000000000000FFFF00000000000000A00A0012
:103610000004500000000000AAAAAAAA000050005E
:10362000DFFF0000000000000000000001000000BB
:1036300000000000AAAAAAAA01000000FFFF0000E3
:10364000000000000000000000000000000000007A
:10365000AAAAAAAA00000000FFFF000000000000C4
:10366000000000000000000000000000AAAAAAAAB2
:1036700000000000FFFF000000000000000000004C
:103680000000000000000000AAAAAAAA0000000092
:10369000FFFF00000000000000000000000000002C
:1036A00000000000AAAAAAAA00000000FFFF000074
:1036B000000000000000000000000000000000000A
:1036C0000A000000000000000300000000000000ED
:1036D00000000000000000000000000000000000EA
:1036E00000000000000000000000000000000000DA
:1036F000FF009600000000080400000040350008AC
:1037000000000000000000000000000000000000B9
:103710000000000000000000FFFFFFFFFFFFFFFFB1
:10372000FFFFFFFFFFFFFFFFFFFFFFFFFFFFFFFFA9
:10373000FFFFFFFFFFFFFFFFFFFFFFFFFFFFFFFF99
:10374000FFFFFFFFFFFFFFFFFFFFFFFFFFFFFFFF89
:10375000FFFFFFFFFFFFFFFFFFFFFFFFFFFFFFFF79
:020000040801F1
:100000000006002089120108291E0A08851D0A0819
:10001000F11D0A08851D0A08BD1D0A088B1201087A
:100020008B1201088B1201088B120108D5490C08AC
:100030008B1201088B1201088B1201088B12010828
:100040008B1201088B1201088B1201088B12010818
:100050008B1201088B120108F15B0C08195C0C086B
:10006000415C0C08695C0C08915C0C08F5050C08F7
:100070001D060C0849060C0875060C08A1060C089C
:10008000C9060C08F5060C0879050C088B12010846
:100090008B1201088B1201088B120108B95C0C0845
:1000A000DD5D0C08F15D0C08055E0C08095E0C08AE
:1000B0000D5E0C088B1201088B120108810C0C08D4
:1000C000290E0C088B1201088B1201088B120108F3
:1000D0008B1201088D5D0C088B120108A15D0C08C4
:1000E0001D5D0C088B1201088B120108315E0C0893
:1000F000355E0C08495E0C084D5E0C0821070C08A3
:100100008B1201088B120108215E0C088B1201086A
:10011000B55D0C08C95D0C088B1201088B12010833
:100120004D070C0875070C08A1070C08CD070C0833
:10013000F9070C088B1201088B1201088B120108B9
:100140008B1201088B1201088B12010801510C0857
:1001500021080C084D080C0879080C088B120108BE
:100160008B1201088B1201088B1201088B120108F7
:100170008B1201088B1201088B1201088B120108E7
:100180008B1201088B1201088B1201088B120108D7
:100190008B1201088B1201088B1201088B120108C7
:1001A0008B1201088B1201088B1201088B120108B7
:1001B0008B1201088B1201088B1201088B120108A7
:1001C0008B1201088B1201088B1201088B12010897
:1001D0008B1201088B1201088B1201088B12010887
:1001E00005650108693603081DAA0408392D0608AB
:1001F0005D330608719E0608FDEE0608C1F6060886
:10020000F9F90608055A07084D7F0708211708085D
:1002100065680808F5160A087D160B08DD820B08CC
:1002200035A90B08B5B30B0875E10B083DE70B08C2
:1002300081F0004102E000BF83F0004330B54FEA97
:1002400041044FEA430594EA050F08BF90EA020F04
:100250001FBF54EA000C55EA020C7FEA645C7FEA97
:10026000655C00F0E2804FEA5454D4EB5555B8BFBA
:100270006D420CDD2C4480EA020281EA030382EA2B
:10028000000083EA010180EA020281EA0303362DBD
:1002900088BF30BD11F0004F4FEA01314FF4801C90
:1002A0004CEA113102D0404261EB410113F0004FA2
:1002B0004FEA03334CEA133302D0524263EB430359
:1002C00094EA050F00F0A780A4F10104D5F1200EF7
:1002D0000DDB02FA0EFC22FA05F2801841F1000152
:1002E00003FA0EF2801843FA05F359410EE0A5F126
:1002F00020050EF1200E012A03FA0EFC28BF4CF057
:10030000020C43FA05F3C01851EBE37101F000450C
:1003100007D54FF0000EDCF1000C7EEB00006EEB19
:100320000101B1F5801F1BD3B1F5001F0CD34908A3
:100330005FEA30004FEA3C0C04F101044FEA4452FA
:1003400012F5800F80F09A80BCF1004F08BF5FEA81
:10035000500C50F1000041EB045141EA050130BD61
:100360005FEA4C0C404141EB0101013C28BFB1F573
:10037000801FE9D291F0000F04BF01460020B1FABE
:1003800081F308BF2033A3F10B03B3F120020CDA91
:100390000C3208DD02F1140CC2F10C0201FA0CF06F
:1003A00021FA02F10CE002F11402D8BFC2F1200CD4
:1003B00001FA02F120FA0CFCDCBF41EA0C0190408A
:1003C000E41AA2BF01EB0451294330BD6FEA0404D3
:1003D0001F3C1CDA0C340EDC04F11404C4F12002BE
:1003E00020FA04F001FA02F340EA030021FA04F3D0
:1003F00045EA030130BDC4F10C04C4F1200220FA27
:1004000002F001FA04F340EA0300294630BD21FA64
:1004100004F0294630BD94F0000F83F4801306BF2A
:1004200081F480110134013D4EE77FEA645C18BF1E
:100430007FEA655C29D094EA050F08BF90EA020FB5
:1004400005D054EA000C04BF1946104630BD91EAAD
:10045000030F1EBF0021002030BD5FEA545C05D1B0
:100460004000494128BF41F0004130BD14F58004EF
:100470003CBF01F5801130BD01F0004545F0FE4163
:1004800041F470014FF0000030BD7FEA645C1ABF98
:10049000194610467FEA655C1CBF0B46024650EACF
:1004A000013406BF52EA033591EA030F41F40021FB
:1004B00030BD00BF90F0000F04BF0021704730B581
:1004C0004FF4806404F132044FF000054FF0000156
:1004D00050E700BF90F0000F04BF0021704730B517
:1004E0004FF4806404F1320410F0004548BF4042EC
:1004F0004FF000013EE700BF42004FEAE2014FEA41
:1005000031014FEA02701FBF12F07F4393F07F4F1B
:1005100081F06051704732F07F4208BF704793F01E
:100520007F4F04BF41F40021704730B54FF4607431
:1005300001F0004521F000411CE700BF50EA010234
:1005400008BF704730B54FF000050AE050EA0102DD
:1005500008BF704730B511F0004502D5404261EB4D
:1005600041014FF4806404F132045FEA915C3FF48E
:10057000D8AE4FF003025FEADC0C18BF03325FEA2B
:10058000DC0C18BF033202EBDC02C2F1200300FADC
:1005900003FC20FA02F001FA03FE40EA0E0021FA01
:1005A00002F11444BDE600BF70B54FF0FF0C4CF4EF
:1005B000E06C1CEA11541DBF1CEA135594EA0C0FA1
:1005C00095EA0C0F00F0DEF82C4481EA030621EADC
:1005D0004C5123EA4C5350EA013518BF52EA033517
:1005E00041F4801143F4801338D0A0FB02CE4FF0C9
:1005F0000005E1FB02E506F00042E0FB03E54FF0F9
:100600000006E1FB03569CF0000F18BF4EF0010EF0
:10061000A4F1FF04B6F5007F64F5407404D25FEAEC
:100620004E0E6D4146EB060642EAC62141EA55519F
:100630004FEAC52040EA5E504FEACE2EB4F1FD0CE1
:1006400088BFBCF5E06F1ED8BEF1004F08BF5FEA5F
:10065000500E50F1000041EB045170BD06F0004611
:1006600046EA010140EA020081EA0301B4EB5C04BE
:10067000C2BFD4EB0C0541EA045170BD41F48011B6
:100680004FF0000E013C00F3AB8014F1360FDEBFDB
:10069000002001F0004170BDC4F10004203C35DAB7
:1006A0000C341BDC04F11404C4F1200500FA05F33A
:1006B00020FA04F001FA05F240EA020001F00042DB
:1006C00021F0004110EBD37021FA04F642EB060151
:1006D0005EEA430E08BF20EAD37070BDC4F10C047B
:1006E000C4F1200500FA04F320FA05F001FA04F23F
:1006F00040EA020001F0004110EBD37041F100012B
:100700005EEA430E08BF20EAD37070BDC4F1200535
:1007100000FA05F24EEA020E20FA04F301FA05F29D
:1007200043EA020321FA04F001F0004121FA04F245
:1007300020EA020000EBD3705EEA430E08BF20EA15
:10074000D37070BD94F0000F0FD101F0004640004F
:1007500041EB010111F4801F08BF013CF7D041EAD1
:10076000060195F0000F18BF704703F000465200D5
:1007700043EB030313F4801F08BF013DF7D043EAA6
:100780000603704794EA0C0F0CEA135518BF95EA5C
:100790000C0F0CD050EA410618BF52EA4306D1D1E3
:1007A00081EA030101F000414FF0000070BD50EA02
:1007B000410606BF1046194652EA430619D094EA8C
:1007C0000C0F02D150EA013613D195EA0C0F05D176
:1007D00052EA03361CBF104619460AD181EA0301CA
:1007E00001F0004141F0FE4141F470014FF0000082
:1007F00070BD41F0FE4141F4780170BD70B54FF01D
:10080000FF0C4CF4E06C1CEA11541DBF1CEA13559C
:1008100094EA0C0F95EA0C0F00F0A7F8A4EB05047E
:1008200081EA030E52EA03354FEA013100F0888075
:100830004FEA03334FF0805545EA131343EA12633E
:100840004FEA022245EA111545EA10654FEA0026F3
:100850000EF000419D4208BF964244F1FD0404F5AC
:10086000407402D25B084FEA3202B61A65EB030508
:100870005B084FEA32024FF480104FF4002CB6EBC5
:10088000020E75EB030E22BFB61A754640EA0C0045
:100890005B084FEA3202B6EB020E75EB030E22BF85
:1008A000B61A754640EA5C005B084FEA3202B6EBC6
:1008B000020E75EB030E22BFB61A754640EA9C0085
:1008C0005B084FEA3202B6EB020E75EB030E22BF55
:1008D000B61A754640EADC0055EA060E18D04FEA13
:1008E000051545EA16754FEA06164FEAC30343EAB3
:1008F00052734FEAC2025FEA1C1CC0D111F4801F80
:100900000BD141EA00014FF000004FF0004CB6E778
:1009100011F4801F04BF01430020B4F1FD0C88BF17
:10092000BCF5E06F3FF6AFAEB5EB030C04BFB6EB22
:10093000020C5FEA500C50F1000041EB045170BD15
:100940000EF0004E4EEA113114EB5C04C2BFD4EB42
:100950000C0541EA045170BD41F480114FF0000EC6
:10096000013C90E645EA060E8DE60CEA135594EA42
:100970000C0F08BF95EA0C0F3FF43BAF94EA0C0F45
:100980000AD150EA01347FF434AF95EA0C0F7FF4BA
:1009900025AF104619462CE795EA0C0F06D152EA0E
:1009A00003353FF4FDAE1046194622E750EA4106F2
:1009B00018BF52EA43067FF4C5AE50EA41047FF403
:1009C0000DAF52EA43057FF4EBAE12E74FF0FF3C68
:1009D00006E000BF4FF0010C02E000BF4FF0010C39
:1009E0004DF804CD4FEA410C7FEA6C5C4FEA430CB2
:1009F00018BF7FEA6C5C1BD001B050EA410C0CBF01
:100A000052EA430C91EA030F02BF90EA020F002062
:100A1000704710F1000F91EA030F58BF994208BFC9
:100A200090422CBFD8176FEAE37040F00100704786
:100A30004FEA410C7FEA6C5C02D150EA013C07D1DD
:100A40004FEA430C7FEA6C5CD6D152EA033CD3D028
:100A50005DF8040B704700BF8446104662468C4622
:100A60001946634600E000BF01B5FFF7B7FF002855
:100A700048BF10F1000F01BD4DF808EDFFF7F4FF7E
:100A80000CBF012000205DF808FB00BF4DF808ED09
:100A9000FFF7EAFF34BF012000205DF808FB00BF2C
:100AA0004DF808EDFFF7E0FF94BF012000205DF84E
:100AB00008FB00BF4DF808EDFFF7CEFF94BF012003
:100AC00000205DF808FB00BF4DF808EDFFF7C4FFFC
:100AD00034BF012000205DF808FB00BF4FEA410C45
:100AE0007FEA6C5C02D150EA013C0AD14FEA430C28
:100AF0007FEA6C5C02D152EA033C02D14FF0000065
:100B000070474FF0010070474FEA410212F50012A2
:100B100015D211D56FF47873B3EB625212D94FEA44
:100B2000C12343F0004343EA505311F0004F23FA2E
:100B300002F018BF404270474FF00000704750EA83
:100B4000013005D111F0004008BF6FF00040704740
:100B50004FF00000704700BF4A0011D212F500129A
:100B600011D20DD56FF47873B3EB62520ED44FEA05
:100B7000C12343F0004343EA505323FA02F0704785
:100B80004FF00000704750EA013002D14FF0FF30C3
:100B900070474FF0000070474FEA4102B2F1E04366
:100BA00024BFB3F5001CDCF1FE5C0DD901F0004C54
:100BB0004FEAC0024CEA5070B2F1004F40EB8300A4
:100BC00008BF20F00100704711F0804F21D113F1D0
:100BD0003872BCBF01F00040704741F480114FEA09
:100BE0005252C2F11802C2F1200C10FA0CF320FA92
:100BF00002F018BF40F001004FEAC1234FEAD323AF
:100C000003FA0CFC40EA0C0023FA02F34FEA430318
:100C1000CCE77FEA625307D150EA01331EBF4FF0A1
:100C2000FE4040F44000704701F0004040F0FE40BC
:100C300040F40000704700BF80F0004002E000BFB9
:100C400081F0004142001FBF5FEA410392EA030FB7
:100C50007FEA226C7FEA236C6AD04FEA1262D2EB01
:100C60001363C1BFD218414048404140B8BF5B4206
:100C7000192B88BF704710F0004F40F4000020F09F
:100C80007F4018BF404211F0004F41F4000121F0B5
:100C90007F4118BF494292EA030F3FD0A2F10102FF
:100CA00041FA03FC10EB0C00C3F1200301FA03F13D
:100CB00000F0004302D5494260EB4000B0F5000F60
:100CC00013D3B0F1807F06D340084FEA310102F11F
:100CD0000102FE2A51D2B1F1004F40EBC25008BFD1
:100CE00020F0010040EA03007047490040EB00009B
:100CF000013A28BFB0F5000FEDD2B0FA80FCACF19C
:100D0000080CB2EB0C0200FA0CF0AABF00EBC250C8
:100D100052421843BCBFD0401843704792F0000FB6
:100D200081F4000106BF80F400000132013BB5E709
:100D30004FEA41037FEA226C18BF7FEA236C21D07F
:100D400092EA030F04D092F0000F08BF08467047E4
:100D500090EA010F1CBF0020704712F07F4F04D1B2
:100D6000400028BF40F00040704712F100723CBFC5
:100D700000F50000704700F0004343F0FE4040F4EF
:100D8000000070477FEA226216BF08467FEA2363AD
:100D90000146420206BF5FEA412390EA010F40F498
:100DA000800070474FF0000304E000BF10F00043E4
:100DB00048BF40425FEA000C08BF704743F09643CB
:100DC00001464FF000001CE050EA010208BF7047E6
:100DD0004FF000030AE000BF50EA010208BF70476D
:100DE00011F0004302D5404261EB41015FEA010C82
:100DF00002BF84460146002043F0B64308BFA3F17A
:100E00008053A3F50003BCFA8CF2083AA3EBC2535B
:100E100010DB01FA02FC634400FA02FCC2F120027A
:100E2000BCF1004F20FA02F243EB020008BF20F0B1
:100E30000100704702F1200201FA02FCC2F1200217
:100E400050EA4C0021FA02F243EB020008BF20EA0C
:100E5000DC7070477BB972B90029BEBF00204FF02B
:100E6000004106E008BF00281CBF6FF000414FF0B2
:100E7000FF3000F007BAADF1080C6DE904CE00298F
:100E800009DB002B1ADB00F095F8DDF804E0DDE962
:100E9000022304B07047404261EB4101002B1BDB91
:100EA00000F088F8DDF804E0DDE9022304B04042F8
:100EB00061EB4101524263EB43037047524263EBE3
:100EC000430300F077F8DDF804E0DDE9022304B025
:100ED000404261EB41017047524263EB430300F033
:100EE00069F8DDF804E0DDE9022304B0524263EB67
:100EF0004303704753B94AB9002908BF00281CBFF3
:100F00004FF0FF314FF0FF3000F0BCB9ADF1080CED
:100F10006DE904CE00F04EF8DDF804E0DDE90223CF
:100F200004B07047430803F05533C01A830803F038
:100F3000333300F03330184400EB101000F00F3062
:100F400000EB002000EB0040000E704707EE900A17
:100F5000F5EEC07AF1EE10FA01D400F00BB8F1EE24
:100F6000677A08B517EE900A00F004F8404261EB8A
:100F7000410108BDD0B5FFF7BFFA0C4B0022064671
:100F80000F46FFF711FBFFF7E7FD0446FFF792FA64
:100F9000074B0022FFF708FB02460B463046394656
:100FA000FFF74AF9FFF7D8FD2146D0BD0000F03D1C
:100FB0000000F0412DE9F047089D04468E46002BC5
:100FC0004DD18A42944669D9B2FA82F252B101FAFD
:100FD00002F3C2F1200120FA01F10CFA02FC41EA0D
:100FE000030E94404FEA1C48210CBEFBF8F61FFA92
:100FF0008CF708FB16E341EA034306FB07F199422D
:101000000AD91CEB030306F1FF3080F01F819942DF
:1010100040F21C81023E63445B1AA4B2B3FBF8F0B9
:1010200008FB103344EA034400FB07F7A7420AD940
:101030001CEB040400F1FF3380F00A81A74240F268
:1010400007816444023840EA0640E41B00261DB1D3
:10105000D4400023C5E900433146BDE8F0878B4208
:1010600009D9002D00F0EF800026C5E900013046C7
:101070003146BDE8F087B3FA83F6002E4AD18B42A1
:1010800002D3824200F2F980841A61EB030301204B
:101090009E46002DE0D0C5E9004EDDE702B9FFDE37
:1010A000B2FA82F2002A40F09280A1EB0C014FEAE2
:1010B0001C471FFA8CFE0126200CB1FBF7F307FB3F
:1010C000131140EA01410EFB03F0884208D91CEBE2
:1010D000010103F1FF3802D2884200F2CB8043467F
:1010E000091AA4B2B1FBF7F007FB101144EA01445E
:1010F0000EFB00FEA64508D91CEB040400F1FF31ED
:1011000002D2A64500F2BB800846A4EB0E0440EADA
:1011100003409CE7C6F12007B34022FA07FC4CEAE3
:10112000030C20FA07F401FA06F31C43F9404FEAD6
:101130001C4900FA06F3B1FBF9F8200C1FFA8CFEEB
:1011400009FB181140EA014108FB0EF0884202FA3F
:1011500006F20BD91CEB010108F1FF3A80F0888000
:10116000884240F28580A8F102086144091AA4B2BD
:10117000B1FBF9F009FB101144EA014100FB0EFE3E
:101180008E4508D91CEB010100F1FF346CD28E456D
:101190006AD90238614440EA0840A0FB0294A1EBFE
:1011A0000E01A142C846A64656D353D05DB1B3EB5B
:1011B000080261EB0E0101FA07F722FA06F3F1408B
:1011C0001F43C5E9007100263146BDE8F087C2F132
:1011D0002003D8400CFA02FC21FA03F391400143AA
:1011E0004FEA1C471FFA8CFEB3FBF7F007FB1036E3
:1011F0000B0C43EA064300FB0EF69E4204FA02F48F
:1012000008D91CEB030300F1FF382FD29E422DD9E1
:10121000023863449B1B89B2B3FBF7F607FB163316
:1012200041EA034106FB0EF38B4208D91CEB010196
:1012300006F1FF3816D28B4214D9023E6144C91A16
:1012400046EA004638E72E46284605E70646E3E626
:101250001846F8E64B45A9D2B9EB020864EB0C0E30
:101260000138A3E74646EAE7204694E74046D1E73F
:10127000D0467BE7023B614432E7304609E76444ED
:10128000023842E7704700BF02E000F000F8FEE7D6
:1012900072B6374880F30888364880F309883648A4
:1012A0003649086040F20000CCF200004EF634717E
:1012B000CEF200010860BFF34F8FBFF36F8F40F293
:1012C0000000C0F2F0004EF68851CEF20001086036
:1012D000BFF34F8FBFF36F8F4FF00000E1EE100AA6
:1012E0004EF63C71CEF200010860062080F31488AF
:1012F000BFF36F8FB3F0CCFBB4F016FB4FF055305B
:101300001F491B4A91423CBF41F8040BFAE71D49B3
:10131000184A91423CBF41F8040BFAE71A491B4AAC
:101320001B4B9A423EBF51F8040B42F8040BF8E7FE
:1013300000201849184A91423CBF41F8040BFAE7D3
:10134000B3F0AAFBB4F044FB144C154DAC4203DAE5
:1013500054F8041B8847F9E701F082FB114C124D49
:10136000AC4203DA54F8041B8847F9E7B3F092BBA8
:1013700000060020002200200000010808ED00E027
:101380000000002000060020B8F20E080022002015
:101390005C2B0020602B002060470120E001010849
:1013A0003002010830020108300201082DE9F04F37
:1013B0002DED108AC1F80CD0C3689D46BDEC108A93
:1013C000BDE8F08F002383F311882846A047002052
:1013D000B2F0E2FAFEE7B2F03FF900DFFEE700000C
:1013E00001F0FF01102A2BDB10F0070F08D010F8D6
:1013F000013B013A8B422DD010F0070F42B3F6D1DA
:10140000F0B441EA012141EA014122F007047FF0F2
:1014100000070023F0E80256083C85EA010586EA49
:10142000010685FA47F5A3FA87F586FA47F6A5FA85
:1014300087F68EB9EED1F0BC01F0FF0102F0070291
:1014400032B110F8013B013A83EA010313B1F8D13C
:101450000020704701387047002D06BF354603381D
:10146000073815F0010F07D1013015F4807F02BF56
:10147000013015F4C03F0130F0BC0138704700BFA7
:1014800010F8012B11F8013B012A28BF9A42F7D02E
:10149000D01A7047034613F8012B002AFBD1181A03
:1014A0000138704738B50022002304460D46FFF787
:1014B000EDFA28B920462946BDE8384000F00AB8C0
:1014C000204605F1004100F005F8404261EB410182
:1014D00038BD00BFD0B50C4B002206460F46FFF7C3
:1014E00063F8FFF739FB0446FEF7E4FF074B0022E1
:1014F000FFF75AF802460B4630463946FEF79CFE87
:10150000FFF72AFB2146D0BD0000F03D0000F0416E
:10151000036800221B68184710B503685B6804461F
:10152000984708B194F84D0010BD00002DE9F04136
:10153000674B03F5A04490B094F99C2806460F46EB
:10154000002A00F0C28094F8E45835B9614A7FF06F
:10155000CFF8284610B0BDE8F081B3F9A4201AB93D
:10156000B3F8A220A3F8A420B3F8A430632B05D8C5
:10157000594A394630467FF0BBF8002500212E221B
:1015800004A80391B7F01AFAD4F8FC07036803AA79
:101590001B6832219847804630B9504A03AB394620
:1015A00030467FF0A5F84546B4F8D837A3F57A73EE
:1015B0009BB241F65832934206D9494B3A46202114
:1015C00030467EF0B3FE002594F90C3A002B6BDD1B
:1015D00094F9C439002B5BDD424B3A46202130465A
:1015E0007EF0A4FE00254049D4F80808322303AA5F
:1015F0008AF02AF8804640B903AB00933A463B4B49
:10160000202130467EF092FE45463949D4F8040840
:10161000322303AA87F04AF8804640B903AB00930F
:101620003A46324B202130467EF080FE454620214E
:1016300030467EF073FEC8B104F65803D3ED007A4D
:101640009FED2C7AF0EEE77AF4EEC77AF1EE10FA1D
:101650000CD594F90C3A002B02DD94F8703A2BB9B2
:10166000254A394630467FF043F8002594F90C3A74
:10167000002B7FF76EAF94F9C938002B3FF469AFA8
:101680001E4B3A46202130467EF050FE002560E792
:1016900094F8708AB8F1000F06D1194B3A46202110
:1016A00030467EF043FE454694F9C439002B9ADD5E
:1016B00094F8F589B8F1000F95D1124B3A462021E4
:1016C00030467EF033FE45468DE7012541E700BFF9
:1016D000702B0020B4CD0C08D6CD0C08FDCD0C0825
:1016E00008CE0C081ACE0C088BCE0C088FCE0C0836
:1016F000A1CE0C0800000034A5CE0C08BFCE0C080B
:1017000040CE0C0866CE0C0838B504467EF0EAFDE3
:10171000114B93F8A819114B1D68EB6A1A68002940
:1017200008BF01461268184690475AF0C9F9EB6A9B
:1017300093F89C1059F0FEFA94F837305BB190F0B2
:10174000A9FBEB6AD3F8A030C01AB0F5FA6F24BF3A
:10175000002384F8373038BD707B00206C2B0020CC
:1017600008B5FFF7D1FF054B05481B68DB6A93F806
:101770009C10BDE8084010F0D3BF00BF6C2B0020C8
:101780004083002070B50E46054664F05BFB64F0B4
:101790001DFB10B90124204670BD0A4B93F9B231EC
:1017A000012BF7D164F04EFB437A002BF2D164F0A9
:1017B00049FB847A002CEDD1034A314628467EF05D
:1017C00097FFE8E7704B0020D8CE0C087EF040BDB4
:1017D0002DE9F0472DED028BC47F90B006460F46F1
:1017E0008CB990F90430002B00F00581834B1D6803
:1017F000A86A03685B6B9847044650B9804A39462B
:1018000030467EF075FF204610B0BDEC028BBDE87F
:10181000F087B3684BB933685B6B3946304610B01C
:10182000BDEC028BBDE8F0471847E86AFFF774FE8D
:1018300004460028E7D1394630467FF0CDFDDFF879
:10184000F4810546394630467EF07AFF98ED717A8C
:10185000D8ED707AB4EEE77A2840F1EE10FAC5B20E
:1018600009D598F9BC31032B05D0664A3946304674
:101870007EF03EFF2546D8ED597AB0EE088AF4EEA8
:10188000C87AF1EE10FA0BD517EE900AFEF734FE87
:101890005D4ACDE90001394630467EF029FF00253A
:1018A000D8ED5A7AF4EEC87AF1EE10FA0BD517EEAD
:1018B000900AFEF721FE554ACDE90001394630462F
:1018C0007EF016FF0025D8ED5B7AB8EE087AF4EECC
:1018D000C77AF1EE10FA0BDD17EE900AFEF70CFE58
:1018E0004B4ACDE90001394630467EF001FF002524
:1018F000B8F95031042B07DC052200923946454ADD
:1019000030467EF0F5FE0025D8F8D00B64F0F6FAEC
:1019100080B198F9B2316BB1D8F8D03BB8F9B421A5
:10192000B3F90E309A4205DA3B4A394630467EF02A
:10193000DFFE002539463046FFF724FFDFF8F8A028
:10194000814639463046FFF7F1FD9AF8D53E002B27
:101950004AD109EA050500EA050430484FF48061E0
:1019600001F062F878B1D8F8D03BB3F90C30A3F2AB
:10197000E24292B2B2F5FA7F05D9294A3946304699
:101980007EF0B6FE0024274890F828355BB100F5BC
:10199000A46038F0C3F8054628B9234A39463046D2
:1019A0007EF0A6FE2C4600212E2204A80DF10C0884
:1019B0000391B7F003F8DAF8C00E4246322109F07D
:1019C0004FFB054600287FF41EAFDAF8C00E03680F
:1019D0009B689847154ACDF8008003463946304643
:1019E0007EF086FE2C460EE7114A394630467EF0E0
:1019F0007FFE0024B1E7012405E700BF6C2B002027
:101A0000E8CE0C08FFCE0C0822CF0C0842CF0C0801
:101A100064CF0C0886CF0C08A5CF0C08702B0020D3
:101A2000E0CF0C08707B002008D00C08609D0D08EA
:101A3000CBCF0C08704B0020706B002070B50546B2
:101A40000E46FFF79FFE3146044628467FF07CFB9A
:101A50002040C0B270BD0000F0B591B005460E4602
:101A60007EF00EFF0446D8B1102128467EF056FCC9
:101A7000B0B100212E2204A803AF0391B6F09EFF5F
:101A80001BF074FD32233A4601211BF02FF8044667
:101A900030B9054B00973246102128467EF046FCAF
:101AA000204611B0F0BD00BF1CD00C0870B5054633
:101AB0000E46B1B990F910408CB1164813F05AFD9A
:101AC000DFED157AB0EEC00AB4EEE70AF1EE10FAD7
:101AD00007D4124A012128467EF00AFE34462046E9
:101AE00070BDAB689BB10E4B1B68D86AFFF714FD45
:101AF000044630B162F004FF0A4A04215CF0A4F805
:101B0000EDE731462846BDE870407FF085B90124F5
:101B1000E5E700BF702B00200000003428D00C083F
:101B20006C2B00203AD00C0838B504467FF00EFD2F
:101B30000546A8B10B4806F043F938B10A490B48ED
:101B40001BF02CF910B1074800F040FF2046FFF7CA
:101B500007FE0123064984F8373020467FF00CFC4D
:101B6000284638BD702B002078820020D83D002008
:101B70005CD00C08F8B505460E461746C2B12329BD
:101B800001D0012914D8244808F030FD044668B17A
:101B900000242046F8BD95F91030022B08D062F0E1
:101BA000AFFE1E4A06215CF04FF8F2E7002EF2D09D
:101BB0003A46314628467FF075FD04460028E7D0B6
:101BC000174ED6F8C02E06F542639A4203D006F5AA
:101BD000A95038F0D9FBD6F8C00E124F03689B6BA2
:101BE0009847D7F8203887F8F804012B07D164F01C
:101BF00029F9542165F0EAF808B9C7F82008284601
:101C0000FFF7AEFD4FF0FF330749C6F8F83E284610
:101C10007FF0B2FBBDE700BF702B00206CD00C083A
:101C2000706B0020707B002084D00C082DE9F04FF1
:101C30002DED028BDFF8449191B0074688467EF087
:101C4000F3FB99F987510446CDB94548BD2138F0D9
:101C500031FB38B1434B42464FF4804138467EF069
:101C600065FB2C463E48BC2138F024FB38B13E4B86
:101C700042464FF4804138467EF058FB00243B4EEC
:101C800096F8E438002B64D01C22002102A8B6F894
:101C900054A5DFED378AB6F091FE04A821F0EAF8EA
:101CA00006F5A46B0125A6F5A046554551D20BA813
:101CB00021F0E0F809AA2946584635F0B7FF002878
:101CC00047D0BDF82610304607F09CFD80B3BDF824
:101CD0000A30102B2CD104A90BA821F0FBFB09F62C
:101CE000E843B0EE408A93ED000A2248B4EEE80AD9
:101CF000F1EE10FAB8BF99ED550A20EE000A0EF089
:101D00001BFEF6EE087A60EE277AB4EEE78AF1EE73
:101D100010FA0DD517EE900AFEF7EEFB164BCDE943
:101D2000000142464FF4804138467EF0FFFA00241D
:101D30000DF1240CBCE80F000DF1080EAEE80F0009
:101D40009CE80700AEE8030001358EF80020ADB234
:101D5000ABE7204611B0BDEC028BBDE8F08F00BFB1
:101D60009080002098D00C08C4D00C08707B002014
:101D70000000003440830020F7D00C08704B002096
:101D800000207047014800F0A1BD00BF702B00206B
:101D900003685B681847000067F096BA63F0A0BF5D
:101DA0002FF012BF59F044B908F074BD0DF0E4B93A
:101DB00014F03EBE03F0E8BA57F022B81FF070BA34
:101DC00066F028BE14F09ABE13F052BC1EF0EEBDB1
:101DD00068F0FABF63F09EBC61F062BE07F0FABE25
:101DE00005F014BA0CF0B6BC0DF024B914F05CBCCC
:101DF00014F032BF13F06EBA14F094BD01F096BB2C
:101E000000F2545022F0CEB808F07EBA90F8C432F6
:101E1000B02202FB030390F8082393F8A13012B11B
:101E2000012B28BF012318467047000090F8143199
:101E30000BB190F841311846704700000348086024
:101E40002921117008221A60704700BF28D40C089D
:101E5000F8B5044604F5935600F5AF40083008364F
:101E6000FFF752FC002130461BF0F2FA8021204699
:101E700015F060F918B131F09BFA2FF033FB04F53F
:101E80000055D5ED597A9FED317A67EE877A05F6E0
:101E9000E437FDEEE77A04F5B44017EE903AC5F862
:101EA000E03BD5F86C313B60083015F045FBF8B9E4
:101EB000D5F8E03B07EE903A04F5805303F2B442C4
:101EC00092ED007AF8EEE77A03F5966367EE877A8B
:101ED000FDEEE77A17EE902AC5F8E02BD3ED007AF5
:101EE00097ED007AF0EEE77A67EE877AC7ED007A31
:101EF00004F5AD5106F5457035F016F904F5A84521
:101F000094ED467AD5ED1E7AE7EE007AC5ED1E7A9D
:101F1000B0EE670A31F074FF04F5AF4085ED1E0A9C
:101F200050300DF011FE04F5AF4000215C3083F01D
:101F3000F9FA4FF40011204615F0FCF820B13046B4
:101F4000BDE8F84019F0AEBBF8BD00BF0000C842C4
:101F5000FFF77EBF70B500F580430546D3F8C00E8D
:101F600003689B6B984705F5AF44503406462046FE
:101F700010F098FB05F5A043002893F8B73418BF7C
:101F800000262BB926B105F53150383083F02EFAF2
:101F9000204610F01DF818B92046FFF747FF20B182
:101FA0002046BDE8704010F0CBBD70BDFFF7D2BF3A
:101FB00038B54FF48011054615F0BCF8044620B939
:101FC0000121284615F0B6F804460221284615F0EE
:101FD000B1F850B114B9284603F0FCF805F5935058
:101FE0000830BDE8384019F05BBA002CF6D138BD96
:101FF000FFF7DEBF38B54FF48011044615F09AF8AC
:1020000001210546204615F095F818B115B920466E
:1020100003F0E0F81021204615F08CF860B120465E
:1020200003F0CAF94FF48001204615F083F818B97F
:1020300031F0BEF92FF048FB2021204615F07AF848
:1020400028B1204603F02EFA204603F047FB4FF458
:102050000051204615F06EF810B1204603F026FB23
:102060008021204615F066F828B131F0A1F9BDE8CD
:1020700038402FF05BBA38BDFFF7BCBF10B504463F
:1020800022F080F890F921308BB190F8403373B191
:1020900094F978355BB1064B1B68DB6A93F89C308A
:1020A0002BB904F25450BDE8104021F093BD10BD8F
:1020B0006C2B0020FFF7E2BF2DE9F041424B1B687B
:1020C000DB6A93F89C300446002B7AD000F58056EA
:1020D00096F87135002B74D008F088FA002870D07B
:1020E00004F5F455103596F8DE1F284618F07CFDEF
:1020F000002866D004F590773846FFF787FE02285F
:102100005FD994F8E4334FF0B00808FB034393ED34
:10211000777AF1EE007AB4EEE77AF1EE10FA50D465
:1021200096F8DE1F284619F00FF804F50053B3F9AE
:10213000502107EE902AB8EEE77AB4EEC07AF1EEBD
:1021400010FA0CDD94F8E42308FB0242F8EE677AFB
:1021500092ED777AF4EEC77AF1EE10FA31DCD6F828
:102160006024D3F8E01B002AB8BF52428A4228DC20
:1021700006F26442D2ED007AD3ED5A6A9FED136AFB
:10218000F8EEE77A66EE866AF4EEE67AF1EE10FA99
:1021900017DC03F6E43292ED007A27EE067AF4EECD
:1021A000C77AF1EE10FA0CD494F8E413B02202FBD3
:1021B00001712846B3F95221BDE8F041D43118F03D
:1021C00091BBBDE8F08100BF6C2B00200000C8422D
:1021D000FFF772BF2DE9F04190F8E4332D4D00EB8D
:1021E00003132F68D3F8948100F5907604463046A7
:1021F000FFF70CFE474514D0022814D904F5804798
:10220000C5F8008097F8F03E012B15D817D104F5DA
:10221000A045D5F81037E3B9D5F81437CBB9052365
:102220000BE0022810D804F5804393F8F02E5AB141
:10223000052283F8F02E07E0013B87F8F03E04F515
:10224000B55004301CF046FB2046BDE8F0410CF0D0
:102250006DBC114B1B68D86A03685B689847804661
:102260000028ECD194F8E413B02303FB0161AC31F6
:10227000204605F017FED5F8F4360FCB05F5DF66DE
:1022800005F5E36586E80F0085E80F0087F8F08E16
:10229000D5E700BF602B00206C2B0020FFF79ABF12
:1022A000F8B500F5A047044697F8E43800F58056E5
:1022B000BBB100F5B440083015F044FC18B101235F
:1022C00086F87135F8BD04F5AF45503528460FF056
:1022D0007FFE08B10023F3E72846FFF7A7FD00289B
:1022E000F8D197F8B734002BF4D1D7F8FC34042B8D
:1022F000E5D104F5AC4038308CF08AFA86F87105E7
:10230000E0E7000010B500F5804400F59843D4F8EC
:10231000C01E2033994200F5A04308D000F59B422F
:10232000283291421CBF4FF0FF32C3F8702403F5EE
:102330008C620749116003F26443064A1A60FFF792
:10234000AFFFD4F8C00E0368BDE810401B69184702
:102350000000C8420000C8C2FFF7D4BFF7B500F5BF
:10236000A0470446D7F8FC348B420D4624D00B1FFF
:1023700000F5AC46594206F1380659413046019104
:102380008CF036F9019930468CF032F9072D0BD1DB
:1023900004F54E50D7F880246423052192FBF3F313
:1023A0000830064A5BF050FC2046C7F8FC5403B0E6
:1023B000BDE8F04003F0E0B803B0F0BD88D10C08F0
:1023C00070B500F580460446D6F8C00E03689B6BD6
:1023D0009847B8B104F5A04595F8F83493B9D6F804
:1023E000C02E04F5984320339A424CD104F5AF46F1
:1023F000503630460FF002F860B995F8B0347BB92A
:10240000012108E004F5AF45503528460FF0E0FD06
:1024100000283ED002212046BDE87040FFF79EBF55
:10242000B5F85E35152B27D195F83C1611F0010152
:1024300020D1D5F8FC34072B1CD095F9B2360BB956
:102440000421E8E7204613F095F8DFED137AB4EEA7
:10245000E70AF1EE10FAF3DB04F5AC4038308CF00B
:1024600017F90028ECD004F54E500C4A062108302C
:102470005BF0EAFB0721CEE73046FFF7D7FC0028E8
:10248000C8D10321C7E704F59B4328339A42F8D10A
:1024900070BD2846F1E700BF0000B442ACD10C0883
:1024A00038B52F4DD5F8C02E05F542639A422DED73
:1024B000028B0446B0EE408A03D00020BDEC028BB4
:1024C00038BD28480EF09AFF40B1BDEC028B04F5F0
:1024D000AF405030BDE8384010F0B2B805F5805438
:1024E000D4F8FC34042B32D195F8F13E33B11E49B7
:1024F000A1F5F47038F0C0F90028DFD194F8E43881
:102500004BB118480EF07AFF0028D6D115480EF0CE
:1025100035FF0028D1D19FED157AF0EEC87AF4EEA0
:10252000C77AF1EE10FA09D49FED110A28EE008A5D
:10253000BDEEC88A18EE103AC4F880340D488CF00D
:10254000A7F80028B9D0002384F8B334B6E7B4F86C
:102550005E15A5F5804007F055F90028C4D1ACE719
:10256000706B00204083002078820020000000343F
:102570000000C842A881002010B52DED028B00F5A7
:10258000A0430446D3F8FC24042A0BD105F0D6F866
:102590002046B0EE408A05F043F938EE400ABDEC23
:1025A000028B10BD03F5E76393ED000AF7E7000027
:1025B0002DE9F0412DED028B00F586658AB00446C9
:1025C00028461DF03FFB04F59350002307A908306F
:1025D0000793089309931AF0C7FD002800F08E8036
:1025E0009DED090ADFED5C7A04F5A04505F59263DF
:1025F00093ED007A20EE270ADFED587AA7EE270A3E
:1026000004F5AC40183004F5804783ED000A68F00B
:102610002FFD2046FFF7D4FED7F8C00E03689B6B52
:102620009847064604F5AF40503010F03BF895F857
:10263000B734002818BF0026002B5AD1002E58D0DE
:1026400095F8F834002B54D1D5F8FC34042B6CD019
:102650009FED438A204605F005F9C5F8340BD7F8FD
:10266000C02E04F598434C339A4204F500581AD111
:1026700095F88037BBB9B8F9AC3B002B04DC394A7C
:10268000D2F88C2BD2060ED5D5F8F416D5F8FC2648
:1026900049680A33521A64214B438242ACBF9B18EB
:1026A0001B18C5F8343BD5F8341BD5F8FC34D7F8E3
:1026B000F42E059120460492039316F03FFAB7F9E1
:1026C000027F06462046FFF757FFCDE9006705F574
:1026D000A36504F53150F0EE400ADDE90332D8ED90
:1026E0007B1A95ED001A0599B0EE480A383082F051
:1026F00021FB0AB0BDEC028BBDE8F08104F59070BF
:10270000FFF784FB02280AD994F8E433B02202FBD5
:10271000034393F8102212B193ED7F0A62E7284633
:102720001DF02AF9B1EE400A5CE704F5AE4604F567
:10273000AE48083608F1180804F5AD414246783134
:10274000304620F033FE002882D04146304620F04B
:10275000C1FEB0EE408A7DE7CDCC4C3ECDCC4C3FA7
:1027600000000000704B0020FFF722BFF8B500F515
:10277000804200F59943D2F8C02E40339A42044675
:102780000E4623D000F5AF47503738460FF020FCF7
:102790000546A8B138460EF097F870B104F5A0448C
:1027A000D4F80C0803689B689847DFED097A20EE9F
:1027B000270A86ED000A2846F8BD9FED060AF8E7CD
:1027C00004F5A9440125A3693360F4E70025F2E785
:1027D0000AD7233C00000000F8B500F5804200F560
:1027E0009943D2F8C02E40339A4204460E4630D068
:1027F00000F5AF47503738460FF0EAFB0546A8B161
:1028000038460EF061F870B104F5A044D4F80C0815
:102810000368DB68984707EE900AF8EEE77AC6EDA2
:10282000007A2846F8BDDFED0C7AF8E704F540544D
:102830000125D4F8A40503681B69984707EE900AA0
:102840009FED067AF8EEE77A67EE877AC6ED007AB2
:10285000E7E70025E5E700BF000000000AD7233CBA
:10286000F8B500F5804200F59943D2F8C02E403308
:102870009A4204460E4624D000F5AF4750373846FA
:102880000FF0A6FB054688B138460EF01DF850B192
:1028900004F5A044D4F80C38186987F03FFE86EDA3
:1028A000000A2846F8BD9FED080AF8E704F54054F1
:1028B0000125D4F8A40503685B69984786ED000AF2
:1028C000EFE70025EDE700BF0000000030B505464A
:1028D0000FC985B06C4684E80F0040F2793221467A
:1028E000284605F071F90C4B03F68442D3F8C03E3C
:1028F00093420ED19DF8001011F0040102D1204640
:1029000020F050FB0548214605F018FA012005B0DB
:1029100030BD0020FBE700BF706B0020702B002053
:1029200010B5044606480FF087F940B904F5804415
:10293000D4F8C00E0368BDE810409B6C184710BD6A
:102940004083002010B5044606480EF0C5FD40B98E
:1029500004F58044D4F8C00E0368BDE81040DB6C79
:10296000184710BD4083002070B5044600F5AF4005
:1029700050300E4615460EF009F950B104F5A0444A
:10298000D4F8843A9B682B60D4F8843A5B6833604F
:1029900070BD04F5805303F58E6203F26C43126838
:1029A0002A601B68336004F50054D4F88C3B9B0507
:1029B000EED4D4ED7B6AD5ED007A9FED037AE6EE96
:1029C000C77AC5ED007AE3E735FA8E3C38B50D4D90
:1029D000044629460C481AF0F3FA04F5804305F141
:1029E000300183F8F10E04F5935008301AF080F9A5
:1029F00004F5AE40D0ED0E7AF1EE677AC0ED0E7AB6
:102A000038BD00BF78820020D83D002010B50446B4
:102A100000F5907029F038FF2046BDE81040FFF720
:102A2000D5BF0000FFF7F2BF00F50050D0F88C3B97
:102A3000194214BF012000207047000010B500F5B6
:102A400080430446D3F8C00E03689B6D9847014647
:102A500004F59C40BDE810408EF088B8FFF7EEBF4B
:102A600038B5054B1C6823680A461D68034B0146B0
:102A70002046A847002038BD6C2B0020702B00207A
:102A800070B52DED028B0446036804F500559B6D6F
:102A90009847D5F88C3B1B0618D5B5F95031B5F9D8
:102AA0005211CA1A0B4402EBD27203EBD3735210C9
:102AB0005B1000EE902A00EE103A04F59350F8EE09
:102AC000E00AB8EEC00A083019F098FE5A4BB5F883
:102AD00082211A7004F5AF4565F032FA083564F0CA
:102AE000C1FE00212846FEF773FE544E0123B0714B
:102AF0002846F3717DF0F6FB28B928467EF050FC9D
:102B0000B0FA80F04009307128467DF0EBFB04F507
:102B1000A045D8B994F8E43304EB031341F28832AA
:102B2000D3F89461D5F88437F31A93420ED904F59B
:102B30009070FFF76BF9022808D9C5F88467204622
:102B400005F03EF905F5C76300221A60B4F9A43018
:102B50001BB9B4F8A230A4F8A430B4F8A430DFED67
:102B6000388A07EE903AF8EEE77AB7EE008A88EEF8
:102B7000270AD4ED2B7AF0EEE77AF4EEE87AF1EE5C
:102B800010FA09D5B4F9A23007EE903AF8EEE77AD8
:102B900088EE277A84ED2B7AD4ED2B0A31F032F8C7
:102BA00070BB57F0D1FA40F27D124FF4801157F00C
:102BB00083FA56F0DBF955F043FE95F8E438B0EEB1
:102BC000408A23B1D5F8040803681B6F984704F5C1
:102BD0003C50B0EE480A343075F07EFB04F54250AC
:102BE000B0EE480A103075F077FBB0EE480ABDEC45
:102BF000028B04F547500430BDE8704075F06CBBA3
:102C0000D4ED2B7A94ED460AF0EEE77AF4EEE87A0A
:102C1000F1EE10FA09D5B4F9A23007EE903AF8EEC9
:102C2000E77A88EE277A84ED2B7AD4ED2B0A30F000
:102C3000E9FF0028B5D0BCE77123002055870020AC
:102C400000000034FFF71CBF70B500F5A046044635
:102C500096F9B036002B28DD07F0C8FC28BB04F538
:102C6000AF45083528467EF09BFBF0B128467DF045
:102C700039FBD0B18FF00EF9D6F8A034C01A96F90E
:102C8000B0364FF47A72534398420ED301221C217E
:102C90002846FEF76FFF40B104F54E50034ABDE8E9
:102CA0007040062108305AF0CFBF70BDCCD10C085F
:102CB00000B52DED028B9FED0B8AD0ED4E7A67EEBD
:102CC000887A83B0C0ED4E7A3830019075F062FB9F
:102CD000019820EE080A03B0BDEC028B5DF804EB0E
:102CE00075F070BC52B87E3F00B52DED028B9FEDA4
:102CF0000B8AD0ED4F7A67EE887A83B0C0ED4F7AB9
:102D00003C30019075F046FB019820EE080A03B0B4
:102D1000BDEC028B5DF804EB75F054BC52B87E3FFD
:102D200070B52DED048B044682B000F5935001A9D7
:102D300008301AF0EBF9002800F0B78004F5A0463F
:102D400006F5916595ED007ADDED017AB4EEE77A4E
:102D5000F1EE10FA07D504F5AF4008307DF0CCFA5B
:102D600008B1019B2B6004F5005595ED697AB5F922
:102D70005031DFED5F6A052BB8BF052307EE903AAF
:102D8000B5F95231F8EEE78A07EE903AF8EEE77AB5
:102D9000B6EE009A77EEA77A1820C7EE270ADFED85
:102DA000557A68EEA77AF4EE490A87EE271AF0EE14
:102DB000007AF1EE10FAB4EE671AC8BFF0EE490AD5
:102DC000F1EE10FA48BFB0EE671ADDED017AF4EECD
:102DD000E67AF1EE10FACCBF87EE270AB0EE410A90
:102DE00031F022F804F5AF405030B0EE408A0FF0D9
:102DF000EFF828B996F8E438D3B396F81139BBB395
:102E000004F5AF4008307DF077FA88B328EE892AC0
:102E10009DED011AB4EEC21AF1EE10FA28D5D5EDE7
:102E2000690ADFED351A9FED350AC0EE820A30F0EF
:102E30002DFF04F53B503C30B4EE408AF0EE408A62
:102E4000F1EE10FA48BFF0EE488AFFF731FF04F5C3
:102E50004150143004F54054FFF746FFD4EDC17AD9
:102E60009FED277A67EE877AB0EE688AC4EDC17A63
:102E7000244819F0F9F890B923484021FFF7D4FD10
:102E800068B1224BD3F8FC34012B08D1F7EE007A5D
:102E9000B4EEE78AF1EE10FA58BFB0EE678AB0EEF2
:102EA000480A02B0BDEC048B70BD04F5AF40083099
:102EB0007DF022FAB7EE008A0028D9D0462064F0CF
:102EC000E7FAB4EEC80ADFED127AF1EE10FAD8BFD5
:102ED000B0EE480A87EE800AB3F0C0FC2F209FEDC9
:102EE0000D1ADFED0D0A30F09FFFB0EE408ABFE70C
:102EF00017B7D1383333333F000000006F12833AE5
:102F000052B87E3FD83D0020702B0020707B0020FF
:102F1000000034428FC2D53F9A99193FF8B5044654
:102F200062F090FF0368DB689847054610B90025FA
:102F30002846F8BD04F58046204607F0D3F9D6F8B8
:102F4000C02E04F59A4350339A42074605D104F542
:102F5000A04393F8A439022BE9D804F5AF405030D0
:102F60000FF05CFA0028E2D1D6F8C00E03689B6B24
:102F7000984758B996F8D43E002BD9D004F50054A0
:102F800094F9BC51023D18BF0125D1E7084BD3F895
:102F9000C00E03685B6B98470028EBD004F5005423
:102FA00094F9F931002BC2D0032BC0D03D46BFE7C6
:102FB000706B0020F0B52DED028B044600F58046C5
:102FC00000F5AF4006F5716383B0503093ED008A91
:102FD0000FF038F904F53B5504F5A0473C350028BF
:102FE00040D1D7F8040803689B689847D7F8943A0B
:102FF0005B0221D5D7F8043893ED437AD3ED097AF3
:1030000067EE877A9FED2F7AF4EEC77AF1EE10FA29
:1030100012DB04F53C5393ED007A67EE877AF7EE06
:10302000006A86EEA77AB4EE667AF1EE10FAC8BFAF
:10303000B0EE667A85ED497ADFED237A90ED250AC8
:10304000F0EE480A20EE270A28467FF043F828468B
:103050008DED010AFFF72CFE9DED010A03B0BDECDA
:10306000028BF0BDD6F8C02E04F5964330339A4259
:1030700026D104F50053D3F8C83BB3F90860003EED
:1030800018BF012604F58054D7F81035D4F86044F1
:103090001C1B97F80C353BB10C484FF40061FFF74F
:1030A000C3FC80F00100C3B23246B0EE480A2146AC
:1030B000284603B0BDEC028BBDE8F0407FF00EB8AF
:1030C0000026DFE700000034E02E6542702B002070
:1030D00010B5044606F0BEFC98B104F5A042D2F843
:1030E000103503F58C415031C2F8101504F58051AC
:1030F000D1F860140029BEBFA3F58C43503BC2F841
:1031000010352046FFF756FFBDE81040042064F05C
:10311000ABB900002DE9F04700F5AF442DED048B6D
:1031200000F580495034054609F571632046D3ED1A
:10313000008A0FF087F805F5415605F5A0481436CA
:10314000002842D1D8F804080368DB689847D8F80B
:10315000943A5B0221D5D8F8043893ED447AD3ED44
:103160000B7A67EE877A9FED4F7AF4EEC77AF1EE2D
:1031700010FA12DB05F5405595ED167A67EE877A61
:10318000F7EE006A86EEA77AB4EE667AF1EE10FAF0
:10319000C8BFB0EE667A85ED5F7A90ED250ADFED67
:1031A000427AF0EE680A20EE270A30467EF0ECFB09
:1031B0003046B0EE408AFFF797FDBDEEC80ABDEC81
:1031C000048BB8EEC00ABDE8F087204605F500572D
:1031D0000DF0A8FB9FED359A97ED7B8AD8F8143552
:1031E00028EE098A8246BDEEC88A462018EE102ACB
:1031F0001A4408EE102A64F04BF9B8EEC88AD7EDED
:10320000657AD9F8C00EA0EE278A05F596433033CB
:103210009842FDEEC87A17EE904A41D1D7F8CC3BE0
:10322000B3F90870003F18BF0127BAF1000F1CD195
:1032300003685B699847C0B9D9F8C00E03689B6BF7
:10324000984790B9D8F82C3B022B0ED1284611F0A4
:10325000DFFF50B108F5D263D3ED007A67EE897ACB
:10326000FDEEE77A17EE903A1CB205F58055D5F8D9
:103270006434E41A98F80C353BB10D484FF4006102
:10328000FFF7D2FB80F00100C3B2B0EE680ABDECDC
:10329000048B3A4621463046BDE8F0477EF05ABCE2
:1032A0000027C2E700000034E02E65420000C8425B
:1032B000702B002010B5044615F088FD68B100B2EF
:1032C00000EB4000C0EB001300EE103AB8EEC00A6D
:1032D000BDE81040132064F0C7B82046FFF71AFF7E
:1032E000F6E7000010B51048FFF718FED0B10F4800
:1032F0000FF0CEF9B0B10E4C042064F0C9F8D4F848
:10330000C80B63F00FF8042064F0AEF8132064F0EB
:10331000BFF8D4F8CC0B63F005F8BDE810401320DB
:1033200064F0A2B810BD00BF702B002040830020C5
:10333000704B0020F8B52DED028B0446FFF7EEFD33
:10334000002800F0AB8004F5804704F59642D7F8DA
:10335000C03E6832934200F0A18004F597422432C7
:10336000934200F09B8004F598420432934200F0AF
:10337000958004F597424032934200F08F8004F527
:1033800097425C32934200F0898004F599425C32A6
:10339000934200F0838004F59942783293427DD0C5
:1033A00004F59A421432934278D004F59A423432AA
:1033B000934273D004F59A42703293426ED004F572
:1033C000AF4050300FF064F9002867D0D7F8C02E16
:1033D00004F596434C339A4260D004F50055F6EE5E
:1033E000008AD5F8C80B62F05DFEB4EEE80AF1EE93
:1033F00010FA40DDB0EE087AFFEE007AE0EE077AD0
:10340000B0EE670AD5F8E02B04F5A04607EE902A47
:10341000D6F81035B8EEE77A07EE903AF8EEE77A8C
:103420005142E7EE007AFDEEE77A17EE900AC6F811
:10343000100530F099FDC6F81005D7F8C02E04F538
:10344000984368339A4222D0D5F8CC0B62F02AFE1A
:10345000B4EEE80AF1EE10FAB0EE408A21DCFEEE9E
:10346000007AB4EEE70AF1EE10FA22D5B0EE087A4F
:10347000F7EE007A19E0FEEE007AB4EEE70AF1EE1C
:1034800010FABFD5B0EE087AF7EE007AB6E7254815
:103490004FF48051FFF7C8FA0028D5D0BDEC028B5D
:1034A000F8BDB0EE087AFFEE007AE8EE077AB0EEEB
:1034B000678A204606F0CEFA08B1B1EE488AD6F8FF
:1034C0001435D5ED5A6A9FED186A05F6E43595ED89
:1034D000007AB5EEC08A07EE903AF1EE10FACCBF52
:1034E00028EE268A27EE488AF8EEE77A66EE866AA4
:1034F000E8EE067A27EE067AFDEEE77AFDEEE66A5A
:1035000017EE903ABDEEC77A16EE902A17EE101A13
:1035100017EE900AC6F8143530F026FDC6F81405EB
:10352000BCE700BF702B00200000C842F8B504467D
:1035300004F5A0458EF0AEFC95F8E438074653B18B
:10354000D5F80C09036804F5AA4204F5AA411B6AE0
:1035500010321431984704F58046D6F8D03EFB1A55
:10356000B3F5FA6F03D9D6F8C00E07F093FD2E4BD2
:10357000C6F8D07ED3F8C00E0268136898470021C1
:10358000204611F0F7FFDFED297AB0EEC00AB4EE65
:10359000E70AF1EE10FA45D505F5E765D5ED007AB5
:1035A000B1EE047AF0EEE77AF4EEC77AF1EE10FAB3
:1035B00038D504F586601CF0DFF9F6EE007AB0EE3F
:1035C000C00AB4EEE70AF1EE10FA2BD504F5B355B4
:1035D00095ED037AF0EE087AB4EEE77AF1EE10FAA0
:1035E00005F10C051ED504F53B503C307EF0E6FDA0
:1035F00004F5415014307EF05DFB04F546502C304C
:103600007FF08AFA95ED007AF7EE007AB4EEE77A69
:10361000F1EE10FA06D504F54C502030BDE8F84024
:103620007EF0D0BFF8BD00BF706B002000000034FA
:1036300000F5005090F94731012BC3BF00F67840E8
:1036400090ED290ADFED047A9FED040AC8BF20EE51
:10365000270A462063F008BF0000C84200000000AF
:103660002DE9F8432DED028B00F5804909F57163D2
:10367000D3ED008A054611F0CFFB0746D9F8C00EFE
:1036800003681B6A984705F546562C3698B14D4C91
:10369000D4F8DC34002B0EDD8EF0FCFBD4F8DC34E7
:1036A000C01A40F6B733984205D8B4F9D044304632
:1036B0007FF03EFA78E005F5A04805F5005498F84B
:1036C000213B43B1B4F9D831002B04DD05F540535B
:1036D00093F9C23103BBD9F8C03E05F596453035A4
:1036E000AB426BD00021B0EE680A30467EF0B8FFE6
:1036F0000546042063F0CCFE2BB207EE903A94ED21
:10370000637AF8EEE77AE0EE077AFDEEE77A17EEF5
:10371000904A3C4424B2CAE70121284611F06EFDCC
:103720009FED297AB4F9D831C0EE077A08F21C5817
:1037300008EE103A58F80C3C9FED240AB8EEC88AFF
:1037400028EE278A07EE903AF8EEE77A67EE807A5D
:103750009FED1F0A27EE800AB2F0A4FEB4F95031A3
:10376000DFED1C7A98ED007A20EE270A07EE903AFA
:10377000F8EEE77A0021B4EEE77AF1EE10FA58BFDE
:10378000F0EE477A80EE277A3046DFED137AB0EE1E
:10379000480AA7EE270AF0EE680A7FF0BDF8BDEEF2
:1037A000C00A10EE103A1CB2BDEC028B20460B4949
:1037B000BDE8F84341F2941230F0E6BB391E18BF61
:1037C000012190E7707B002000A08C450AD7233CA4
:1037D00035FA8E3C0AE81C41E02E65426CEEFFFF94
:1037E00038B500F540530546D3F8A4050368DB68F7
:1037F0009847014605F54C5020307EF0C5FE04B2D6
:103800002846FFF78BFB70B107EE904A05F500558F
:10381000B8EEE70AD5F8D40B62F084FDBDEEC00A1D
:1038200010EE103A1CB220460349BDE8384041F280
:10383000941230F0A9BB00BF6CEEFFFF38B590F8D2
:10384000E433B02202FB030393ED777AF7EE007ABC
:10385000B4EEE77AF1EE10FA054600F5A0441DD566
:10386000002111F087FEDFED427AB0EEC00AB4EE1F
:10387000E70AF1EE10FA11D5D4F8FC34012B0DD083
:10388000072B0BD0002384F8743404F58F640023D5
:1038900023602846BDE8384011F0BEBA8EF0FAFA2F
:1038A000D4F87C34C4F87C04C31AB3F57A7F84BF9F
:1038B000002384F87434284611F0AEFAD4F8FC34AE
:1038C000012B07EE100A2DD0072B2BD0B8EEC77AAC
:1038D000DFED286AC7EE267A05F50052B2F99C2181
:1038E00000EE102AB8EEC00A27EE800ADFED207A3B
:1038F000B0EEC07AB4EEE77AF1EE10FA14D40023F9
:1039000084F8743494F8743405F54C502030DBB9E5
:103910007EF022FDBDE83840174900B241F2941212
:1039200030F032BB9FED150A94F87424002AE9D1D7
:103930000122934284F87424E4D0072B1EBF04F5BF
:103940008F6300221A60DDE704F58F6494ED007A3E
:10395000DFED0B7A67EEC77A9FED0A7A67EE877A1A
:10396000FDEEE77A17EE901A7EF00EFED2E700BF6A
:103970000000003400A08C456CEEFFFF000000004A
:10398000E02E65420000C84270B52DED028B00F5B7
:10399000AC46383682B0044630468AF0A9FD05466A
:1039A000D8B904F50052D2F8C83BB3F9083073B95E
:1039B00004F5AE43D3ED0E7A92ED667AF0EEE77A37
:1039C000F4EEC77AF1EE10FA4CBF0125002530461F
:1039D0008AF0A2FD002808BF002530468AF088FD45
:1039E00050BB04F5A043D3F8703401331ED01DBB87
:1039F0009FED1C8A2046FFF733FE07EE900AB8EED3
:103A0000E70A8DED010AFDB9152063F02DFD9DED4E
:103A1000010A1A2063F028FD04F5B040583002B0C6
:103A2000BDEC028BBDE8704003F0C2BB002DDFD0BF
:103A30002046FFF703FF02E02046FFF7D1FE07EE26
:103A4000900AB8EEE78AD5E71A2063F0B9FF9DED3A
:103A5000010A08B9B0EE480A152063F005FDB0EE82
:103A6000480AD6E70000000010B500F5005303F641
:103A7000E432D3ED5A6ADFED127A92ED007A9FEDCF
:103A8000116A03F6784366EEA76A27EE277AD3ED2C
:103A90002A7A67EE867AFDEEE66ABDEEC77AFDEE1B
:103AA000E77A044616EE902A17EE101A17EE900ADF
:103AB00030F05AFA04F5A044C4F8140510BD00BF54
:103AC0000000C842A00CB34510B5044613F036FB05
:103AD000031E2ADB04F5005191F947219A4224DDA7
:103AE00004F5A040D0F8FC44022C1ED0D1ED687A39
:103AF000DFED0E6AD31A66EEE76A07EE102A07EECC
:103B0000903AB8EEC77AF8EEE77AD0F8143587EE37
:103B1000876A07EE903AF8EEE77AE6EE867AFDEEEF
:103B2000E77A17EE903AC0F8143510BD0000C8428D
:103B300070B52DED028B00F5A0449FED540AD4F82A
:103B400010359FED537A07EE903AF8EEE77A054686
:103B500067EE807A9FED4F0AF0EEE76AF4EE476A6F
:103B6000F1EE10FAC8BFF0EE477A27EE800AB2F005
:103B700009FB30F07BF8B7EE008AC8EE007A04F556
:103B8000A36305F50056C3ED007A94F8E438A3B1B9
:103B9000D4F80C09036805F52F515B6A203198476A
:103BA00058B1D6F8E02BD4F81005514230F0DCF9CA
:103BB000C4F81005BDEC028B70BD96F97831002B6E
:103BC000F8D0284605F046FF0028F3D105F5B440AB
:103BD000083013F0B1FC0028ECD1B6F95031012BBC
:103BE000B8BF012307EE903A04F21C52F8EEE77AD0
:103BF000D2ED006A86EEA77AB4EEC87AF1EE10FA3A
:103C000013D840F6C4122449D4F8100530F0ACF9AA
:103C1000C4F81005D6F8E02B40F6C4139A42D4BF7E
:103C2000C6F8E02BC6F8E03BC4E704F5A363D3ED88
:103C3000007AF4EEC77AF1EE10FABBDD88EE070ADF
:103C400020EE000AB2F058FCDFED147AD4F810052B
:103C500020EE270ADFED127A20EE270A40F6C41381
:103C6000FDEEC07A17EE905A9D42B8BF1D462A4617
:103C7000694230F079F9C4F81005D6F8E03BAB4260
:103C8000D4BFC6F8E03BC6F8E05B93E70AD7233C15
:103C90000000AA4235FA8E3C3CF6FFFFE02E65425A
:103CA0000000C84210B500F540530446D3F8A405FF
:103CB00003681B68984704F50053D3F8E02B514282
:103CC00030F052F904F5A043C3F810052046BDE8D2
:103CD0001040FFF72DBF0000704700000120704723
:103CE0000820704701207047014B93F8840170470A
:103CF000704B0020034B93F98409003818BF012052
:103D0000704700BF704B0020014B93F9860170474C
:103D1000704B002013B5064BD3F8C00E4B690468F6
:103D2000009308310EC9646CA04702B010BD00BFFB
:103D3000706B0020704700007047000038B5254DBB
:103D4000D5F8C00E03685B68984719283BD8DFE8B0
:103D500000F00D38360D0D363636363A38383838EC
:103D600038383A36363636383A0D383840241A4B19
:103D700093F8812312B193F880330BB944F0100407
:103D8000164BD5F8C02E9A42A3F11C0303D09A42D9
:103D900018BF44F01004124991F9F911A9B19A42DF
:103DA00015D0032902D10F4B9A4201D144F04004AF
:103DB0000D487CF097FA50B144F0800407E01024DD
:103DC000D5E71824D3E70124D1E79A42F0D144F093
:103DD000010038BD706B0020705B0020307800203F
:103DE000704B002090770020F882002008B504482E
:103DF00006F0FCFB00280CBF0120022008BD00BF1C
:103E0000702B0020F0B52DED028B8BB0054619F01C
:103E1000ADFB4FF48071D0F8047290ED828AD0F837
:103E20000C6204461948FEF7FFFD30B9184BDFED70
:103E3000197A93ED7B7AA7EE678A17480CF0A6FEF5
:103E400030B1164BD3F8843A5F6893ED028ADE688E
:103E50002D7C8EF01FF8D4F81823D4F81C33D4F836
:103E600014130892099327221C23CDE900320390F2
:103E7000079103AA1E21284604978DED058A069610
:103E80005AF000FF0BB0BDEC028BF0BD702B002090
:103E9000704B002035FA8E3C40830020707B002060
:103EA00038B5C5780B46352D044628BF3525352253
:103EB00000211846B4F082FD2A4604F10C01BDE849
:103EC0003840B4F031BD000008B5024813F036F9AF
:103ED00000B208BD702B002037B50D46134840F2E4
:103EE000EF2203F071FE2C7814F004040AD0696804
:103EF00003220F481EF0C4FF0C4803B0BDE8304059
:103F000003F07ABA01AA214628461FF05BF8002880
:103F1000F2D0DDED017A9FED077A67EE877A2246CF
:103F2000FDEEE77A17EE901AE3E700BF702B002052
:103F3000888200200000C84210B5054C012384F897
:103F400083335CF021FB002384F8833310BD00BF72
:103F5000705B00205FF052BC2DE9F0412DED028B2B
:103F60004FF0000882B0CDE900281E4F9FED1E8A59
:103F70000C461546B0EE480AB1F90220D7F8C81B26
:103F80004FF47A7306465FF013FF0123CDE9005327
:103F9000B4F90020D7F8CC1BB0EE480A30464FF4F5
:103FA0007A735FF005FFB4F90420D7F8D01B9FEDBA
:103FB0000F0A43463046CDE900585FF0F9FECDE9DF
:103FC0000058B4F90620D7F8D41BB0EE480A4FF4D5
:103FD0007A7330465FF0ECFE02B0BDEC028BBDE8B8
:103FE000F08100BF704B00200000FA4400007A44CA
:103FF00008B55CF0C1F840F4A67040F0010008BDBF
:1040000010B504461FF03EFB204610BD10B50C4C09
:10401000002384F8B3345CF0B1FFA4F58052A4F51A
:104020007873D2F8C02E9A4208D194F824352BB96F
:1040300004F5A460BDE8104036F078BB10BD00BFA9
:10404000707B002013B5124C94F8DE1F04F56960F4
:1040500016F0CAFD78B194F8DE1F04F5696017F018
:1040600031F840B194F8DE1F04F5696002B0BDE894
:10407000104017F069B819F079FA01A919F046F85B
:1040800018B19DED010A02B010BD9FED020AFAE7DA
:10409000703B002000000000044B93F8E40820B1BE
:1040A000D3F80C0903681B6B18477047707B00201E
:1040B00008B5084BD3F8702B002A03DCBDE8084094
:1040C0005CF09EB803F5296059F02CF990ED000AD8
:1040D00008BD00BF704B002008B51248D0F8C02EB4
:1040E00000F6A4439A4216D0B0F9D83EABB900F519
:1040F000805393F83D2482B990F8D52E6AB993F88D
:10410000E93463B9A0F5804006F070FA00280CBFCE
:104110000320042008BD0220FCE70520FAE7062062
:10412000F8E700BF706B002010B5224B03F54C621E
:10413000D3F8C03E934290B0044639D0002302F633
:10414000582002931EF086FE014618B91A4802AAAA
:104150001EF0CCFE247C8DF09DFE184BDDED027A26
:10416000D3F82027D3F8243705930023F8EEE77A15
:104170009FED137A0793089309930A930B930C937B
:104180000D930E934FF6F853ADF83C300023CDE974
:10419000030267EE877A96228DF83E303323CDE90D
:1041A0000032572103AA2046CDED067A5AF06AFD67
:1041B00010B010BD706B002088820020707B002042
:1041C0000AD7233CF0B58DB004468DF063FE184A43
:1041D000D2F80839C31A642B28D8D2F804380290D0
:1041E000D3F88C10D3F89020D3F88460D3F888509B
:1041F000D3F8DC70D3F894E0D3F898C0D3F89C30AF
:10420000099300238DF82C30069225231622CDE940
:1042100000320591207CCDF81CE002AA5321CDF894
:1042200020C00A97039604955AF02CFD0DB0F0BDFE
:10423000707B002010B55CF0E9F9044688B90A48A3
:10424000A0F58052A0F57873D2F8C02E80F8B34460
:104250009A4206D190F824351BB900F5A46036F0D7
:1042600065FA204610BD00BF707B00202DE9F047A5
:104270002DED088B8D4CD4F8C02E04F54C639A427A
:1042800090B0054600F0EB8003F531600CF07EFC49
:10429000DFED878ADFED879A9FED879A04F58057D7
:1042A000002867D007F5FA600CF00EFB002861D0FB
:1042B000D7F804089FED810A6C3032F0B9FE07F29E
:1042C000DC70B0EE60AAB0EE418ACDED070A8DED4C
:1042D000081AF0EE40AA8DED060A81F077F9D7F8BA
:1042E00008380146D3F85C23D3F85833059204A864
:1042F000049332F09DFC09A88DED090AB0EE680A1E
:10430000CDED0A0A32F0A4FC28EE288A02A8BDEE00
:10431000C88A95F81090CDED030A18EE103A8DED8D
:10432000020A1EB232F008FDDFED657A20EE270AA0
:1043300002A8BDEEC00A6AEEA8AA10EE103A0FFA63
:1043400083F832F043FDB4EEE90AF1EE10FA58BFFB
:10435000B0EE690ABCEEC00AD4F8C02E10EE103AD6
:104360009DB204F6DC439A422AEE28AA7CD1DFED06
:10437000558A7FE0D7F81035DFF84CA195F81090FA
:10438000DAF8A48507EE903AD7F81435B8EEE7BA14
:1043900007EE903AD8F8003040469B68F8EEE7AA5E
:1043A000984707EE900AF8EEE77A404667EEA87A5B
:1043B00007F59367FDEEE77A04F6FC6417EE903A92
:1043C0001EB2D8F800301B69984707EE900AF8EE45
:1043D000E77A97ED00AA67EEA87AB4EEE9AAFDEEB7
:1043E000E77AF1EE10FA17EE903ADFED327AAAF59D
:1043F000405058BFB0EE67AA1DB203F0A1F8D8F83C
:104400000030D4ED007A5B6908EE100A404627EED2
:10441000899A9847B8EEC88ABCEECAAA2BEE28BA89
:104420006AEEA8AA1AEE103A68EE288A8DED09BA4B
:10443000CDED0AAACDED0B8A8DED0C9A8DED0D0A0E
:10444000ADF83860ADF83A50ADF83C30B7221A23D9
:10445000CDE900323E2109AA48465AF013FC10B0BB
:10446000BDEC088BBDE8F087D7F80838D3ED0F7A9C
:1044700067EEA88AD7F80C3804F6FC64D4ED007A0D
:10448000186927EE899A86F049F8CDED09AA8DEDD5
:104490000AAACDED0B8A8DED0C9A8DED0D0AADF8C3
:1044A0003860ADF83A80ADF83C50CFE7706B002033
:1044B0000AD7233C00FF7F470000C8429F0CB3454A
:1044C000E02E654200000000705B002001480CF007
:1044D0000DBA00BF4083002008B5034BD3F8C00ECF
:1044E00003685B68984708BD706B002030B587B0E3
:1044F000054619F03BF804462D7C8DF0BFFCD4F83E
:104500008422D4F888320492059300211023CD220E
:10451000CDE900320290039102AA42F60C312846FE
:104520005AF0B0FB07B030BD30B52DED028B89B02D
:10453000054619F01BF800F55A7393E8070002AC22
:1045400084E80700DDED020A9DED030A2D7CF1EE03
:10455000600AB1EE400AB2F037F82046B0EE408A69
:1045600033F0EAF9DFED0B7A049B079328EE278AF4
:104570000C230122CDE90032A82105AA28468DEDA1
:10458000058A8DED060A5AF07DFB09B0BDEC028B61
:1045900030BD00BFE02E6542422938B505461BD02C
:1045A0000AD824290CD0402924D01B2922D02846FF
:1045B000BDE838405FF02EBF432917D05329F5E7F7
:1045C0000C2159F05DFD044610B90024204638BD89
:1045D0002846FFF7A9FFF9E7102159F051FD0446DD
:1045E0000028F2D02846FFF781FFEFE7017C024860
:1045F00089F07CFF0124E9E7A8810020F0B52DEDCA
:10460000028B05468DB01646B0EE408A0C46002956
:1046100030D0007C5AF0CCFA0746287C5BF0CCF90D
:1046200000F121039F4207D2287C0DB0BDEC028B24
:10463000BDE8F04059F012BD63690893636A2269CE
:10464000CDF82530236AA069E1680792CDF82930BA
:104650006222212327680590CDE900320691287C4B
:104660000397192303AAC2218DED048A8DF82460D3
:104670005AF008FB0DB0BDEC028BF0BDF8B54B4C09
:10468000D4F8C02E04F54C639A42054600F08C80A5
:10469000A4F50056B6F82232DF0713D544480DF0D2
:1046A00097FC002879D004F58054D4F804080368F6
:1046B0009B68984700F1940191ED010A0122284678
:1046C000FFF79CFFB6F822329C0712D538480DF050
:1046D0007FFC002864D0374BD3F804080368DB68FC
:1046E000984700F1940191ED010A02222846FFF754
:1046F00085FFB6F82232580712D52D480DF068FC18
:1047000000284FD02B4BD3F8040803681B69984747
:1047100000F1940191ED010A03222846FFF76EFF94
:10472000B6F82232190708D52349052291EDD50A9A
:10473000284601F55471FFF761FFB6F82232DA0618
:1047400016D51C4FD7F8FC34042B11D118F00EFFEE
:10475000044607F5C76089F0F9FE94EDC70ADFED5E
:10476000177A014620EE270A06222846FFF746FF61
:10477000B6F822329B0617D50D480DF029FC98B1EA
:104780000C4BD3F80818284691EDAB0ABDE8F84069
:10479000042201F52A71FFF731BFA4F6DC718BE723
:1047A0000749A0E70749B5E7F8BD00BF706B0020D7
:1047B00040830020707B0020705B0020E02E65426B
:1047C000F05C0020645E002070B504460E4628F0C0
:1047D00099F890F8C412B02303FB0101AC312046D4
:1047E00003F060FB0546C0B13EB118F0BFFE90F883
:1047F0007C3243F0020380F87C3204F58043D3F826
:10480000C00E04F598434C33984204D004F59A4402
:104810005034A04201D106F065FB284670BD00006F
:1048200073B516460191044618F0A0FE019918F0E0
:10483000B5FA0546C0B13EB118F098FE90F87C324A
:1048400043F0020380F87C3204F58043D3F8C00EB5
:1048500004F598434C33984204D004F59A445034FC
:10486000A04201D106F03EFB284602B070BD000018
:1048700030B5054685B00C46D1E9040130F0CEFBD9
:1048800040B168461EF0F6FA6A46214628465FF0B7
:10489000FFF908B9022067E0344840F24F32694618
:1048A00003F092F9D4ED037AF4EE677AF1EE10FAA0
:1048B00022D69FED2F7AF0EEE77AF4EEC77AF1EE8A
:1048C00010FA54BF012200229DF80030294962F3FA
:1048D000410368468DF800301EF004FC0028D9D151
:1048E000254869466BF09AFB40B957F0E9F8052274
:1048F000162157F041F8CDE70022E5E7D4ED017A23
:10490000FDEEE77A17EE903ADB0706D41B4B03F671
:104910008442D3F8C03E934225D11949134802225C
:1049200012F01CFA9DF8001011F0040102D1684643
:104930001EF038FB0D48694603F000FA94ED020AB8
:10494000B4EE400AF1EE10FA0BD6B5EEC00AF1EE65
:1049500010FA06DD9DF800100948C1F3400107F088
:104960009DFC002000E0042005B030BD702B00202D
:104970000000003478820020B84B0020706B0020CB
:10498000F477002010B52DED028BD1ED017A91ED79
:10499000008AFCEEE77A8AB0CDED037A9DF80C1020
:1049A00005AA04465FF05EF9C8B1DFED0E7A059BFB
:1049B000009368EE277A0022FDEEE77A114617EEA3
:1049C000903A06A81EF076FA23682046D3F8C43041
:1049D00006A9984700200AB0BDEC028B10BD02204A
:1049E000F9E700BF0000C84237B5124DD5F8C00E38
:1049F00003681B6A0C46984740B9D5F8C02E05F5E8
:104A000042639A4202D0042003B030BDD4ED007A54
:104A1000D4ED020A94ED010A0748FCEEE77ACDEDE9
:104A2000017A9DF8041003F0EBFE0028EBD0002083
:104A3000EAE700BF706B0020702B0020134610B512
:104A400024220C4618460021B3F0B8FFA27F8277DB
:104A5000E27FC277072280F82020A28B8283D4EDE8
:104A6000067AF1EE677AC0ED067A10BD10B48C8B31
:104A7000162C03D15DF8044BFFF7E0BF5DF8044B43
:104A80005EF02EBB08B591F82030072B0ED10948F7
:104A900090F8E43843B191ED060A00F5FA60B1EE02
:104AA000400A0DF05BF818B9042008BD0220FCE7AD
:104AB0000020FAE7707B002008B5D1ED007A9FED69
:104AC000087A0848F0EEE77AF4EEC77AF1EE10FAC9
:104AD00054BF0121002104F0B7FF002008BD00BF32
:104AE00000000034702B002010B5D1ED007AFCEEF0
:104AF000E77A17EE903A9CB2012C02D0022C06D035
:104B000084B91148214666F021FA002010BD0F48F3
:104B100090F82C365B0707D55FF0F2FE0C4A0521B2
:104B200059F092F80420F1E790F918361BB95FF0BC
:104B3000E7FE084AF3E7A0F5A0400AF049FB002889
:104B400014BF00200420E1E788810020707B002052
:104B500064D70C087FD70C081FB5D1ED017AFCEEA5
:104B6000E77A0B46CDED027AD1ED007A1A7C017C12
:104B70000192FCEEE77A0B48CDED037AD3ED027A91
:104B8000FCEEE77A17EE902A92B2009293ED030AB8
:104B90009DF80C209DF8083009F084FC05B05DF804
:104BA00004FB00BF4083002007B5D1ED007A084820
:104BB000FCEEE77ACDED017A9DF804100BF096FA41
:104BC00000280CBF0420002003B05DF804FB00BFE8
:104BD0004083002070B58B8BC02B05460C4633D824
:104BE000B12B0DD8142B00F0AE80162B59D0112B01
:104BF00000F0A68021462846BDE8704060F0A2BAC9
:104C0000B23B0E2BF6D801A151F823F0914C0108CC
:104C1000F54B0108F54B0108F54B0108F54B010870
:104C2000F54B0108F54B0108F54B0108874C0108CD
:104C3000F54B0108BB4C0108F74C0108F54B010886
:104C4000AB4C01087D4C0108D42B13D007D8D02BD6
:104C500023D0D12BCED1BDE87040FFF77DBFB3F597
:104C6000967F53D040F6B836B342C3D1BDE870400A
:104C7000FFF79ABFBDE87040FFF71EBF2146BDE8B1
:104C80007040FFF7F5BD2146BDE87040FFF77ABEE2
:104C90002146BDE87040FFF7A7BEBDE87040FFF7B2
:104CA00023BFBDE87040FFF7EDBE94ED000A284831
:104CB000FDF7F6FBE8B100201CE0264C94F8F13E2D
:104CC000BBB1254904F5A95035F02EFE88B104F595
:104CD0008053012283F8592504F542610222A4F58C
:104CE000804012F03BF80028E5D11C4B002283F8ED
:104CF0005925042070BD174C94F8F13E002BF8D0D4
:104D0000154904F5A95035F093FDDFE7D1ED007AA0
:104D10009FED137AF0EEE77AF4EEC77AF1EE10FA2F
:104D200014D5D1ED017AF0EEE77AF4EEC77AF1EE20
:104D300010FA0BD50B490222054812F00FF8BAE71A
:104D400009490222F8E709490222F5E70220D1E7E2
:104D5000702B0020706B002078820020707B002078
:104D60000000003490770020D8770020BC77002026
:104D700070B5434B03F68442D3F8C03E93428EB0E5
:104D80000C467BD1CD78272D28BF2725272200214F
:104D900004A8B3F013FE2A4604F10C0104A8B3F0F2
:104DA000C3FD059B9DF836400093069B0193E443A9
:104DB000079B0293E4B2089B03938DF836408DF075
:104DC00069F814F0810F04F08705064601D1802DA3
:104DD00013D1684631F096FCDFED2A7A2A4B20EE9B
:104DE000270ADFED2A7AC3F8D46420EE270ABDEE45
:104DF000C00A10EE102AC3F8C82414F0820F01D1A3
:104E0000802D13D1684631F097FCDFED1E7A1E4BE2
:104E100020EE270ADFED1D7AC3F8D86420EE270ABA
:104E2000BDEEC00A10EE102AC3F8CC2414F0840F93
:104E300001D1802D13D1684631F08EFCDFED117A5F
:104E4000114B20EE270ADFED117AC3F8DC6420EE67
:104E5000270ABDEEC00A10EE102AC3F8D02463065C
:104E60000CD5DDED0C7A9FED097A074B67EE877A5A
:104E700003F59C62C2ED007AC3F8E4640EB070BD25
:104E8000706B0020E02E6542707B00200000C8425D
:104E900030B5214C91B0084602A9FFF701F8D4F8CB
:104EA000C02E04F684439A4233D19DF83C30072B40
:104EB0002FD104F58054DDED056AD4F81C379FED41
:104EC000177A07EE903AF8EEE77AE6EEC77AFDEE4B
:104ED000E77A17EE903AC4F81C375FF011FDD4F86A
:104EE000F426D4F81C3752689FED0D7A9B1A07EE12
:104EF000903AF8EEE77A054667EE877A17EE900A61
:104F0000FBF7FAFA074ACDE900010621284658F0D6
:104F10009BFE11B030BD00BF706B00200000C84286
:104F20000AD7233C98D70C0810B51D4B03F68442D2
:104F3000D3F8C03E9342044696B008460FD108A964
:104F4000FEF7AEFF9DF8541003AA20465EF08AFEDD
:104F500038B95FF0D5FC134A042158F075FE16B03D
:104F600010BDBDF8503023F004039BB2002BF6D0E7
:104F7000DDED0B7A9FED0C7A039B009367EE877A49
:104F80000022FDEEE77A114617EE903A04A81DF0D4
:104F900091FF236804A9D3F8C43020469847DEE780
:104FA000706B0020ACD70C080000C84230B48D7A7A
:104FB0004B7A43EA0523CD7A43EA0543562B044650
:104FC0000A4618D008D8522B0FD0542B10D02046A8
:104FD000114630BC5EF04EBF03F18073863B23F078
:104FE0007F43012BF3D830BC704730BCFFF7C0BE05
:104FF00030BCFFF74DBF30BCFFF796BF00207047B5
:10500000C82070470120704700207047002070477B
:1050100090F890308B4286BF00EB8100D0F894006E
:105020000020704790F890308B4286BF00EB8100E3
:10503000D0F894000020704703207047014B93F88C
:1050400082017047704B002070B504463E4810F056
:105050008BFA18B1236A43F4000323623A4810F034
:1050600083FA88B1462062F013FADFED387AB4EEA5
:10507000E70AF1EE10FA07D8636A43F400036362AB
:10508000A36A43F40003A362236A43F4F843236250
:105090002F4BD3F8C00E03685B6898470138182877
:1050A00015D8DFE800F0343C0D3E3C3C3C3C143469
:1050B0003434343434143C3C3C3C34143E343400FA
:1050C000244A92F8803353B392F8812352B3224B8F
:1050D0001D68DDB1214E284696F8BA1B4EF088FBBC
:1050E000A0B1236A43F48073236296F920321BB186
:1050F000636A43F48073636296F8BA1B28464EF0E5
:10510000AFFB18B1A36A43F48073A36270BDD4E906
:10511000092342F4E04243F4E0436262A3620123C4
:1051200000E00023616A41F480626262A26A42F494
:105130008060A062002BCAD041F4406142F440621A
:105140006162A262C3E700BF702B0020000000B4C0
:10515000706B0020705B0020FC870020704B0020EB
:1051600013B54FF44470CDE900211EF083FA0446D4
:1051700028B1DDE900215FF0E1FB024B236020460E
:1051800002B010BDA8D90C0800207047002070475D
:10519000002070470020704700F50750243070470A
:1051A00000487047F4FF0C0800F58040D0F8C00EAE
:1051B00003685B681847000000F5804300F59840DD
:1051C000D3F8C03E20301B1A5842584170470000A7
:1051D000A22070472DE9F04100F5A045DFED686A97
:1051E000D5F8103507EE903AD5F81435B8EEE77AD1
:1051F00007EE903AF8EEE77A00F5AF4890B027EE68
:10520000267A67EEA67A08F1500804460023404645
:105210008DED017ACDED027A03930BF0B7FC0028F7
:1052200000F0A680D5F8043884330FCB0CAF87E8A4
:105230000F0008AE04AF87E80F0086E80F0001A951
:10524000384603AB02AA31F0A1FA9FED4E0AD5F819
:10525000847A01A831F0ECFE314638468DED080A1B
:10526000CDED090A8DED0A1A16F07AFA8CF012FECD
:10527000D5F80839C01A632804F57C662DD8D5F80E
:10528000040803689B689847042100F194023046A3
:1052900055F038FCD5F804080368DB689847052109
:1052A00000F19402304655F02DFCD5F8040803684F
:1052B0001B699847062100F19402304655F022FC04
:1052C000D5F80828304602F52A72072155F01AFC55
:1052D00004F5B440083013F097F940460CF078FE1E
:1052E00090B1D5F8080884F0F5FD68B1D5F8082824
:1052F0006E219032304655F005FCD5F808286F2114
:10530000BC32304655F0FEFB04F540522432692190
:10531000304655F0F7FB04F546526A21304655F009
:10532000F1FB04F5405393F9C22132B9D3ED6E7A03
:10533000F5EEC07AF1EE10FA06DD04F54B52343288
:105340006B21304655F0DEFB04F54C5420342046EA
:105350007DF03CF928B104F130026D21304655F062
:10536000D1FB18F003F917F015FE10B0BDE8F0817D
:1053700004F5935001A9083016F0BAF876E700BF9B
:105380000AD7233CE02E654210B54FF48011044645
:1053900011F0D0FE10B12046FFF71CFF4FF4800142
:1053A000204611F0C7FE28B12EF002F8BDE81040EB
:1053B0002CF08AB910BD000030B500F5935591B0BE
:1053C00000230835029302A9002304460DF10702C9
:1053D00028468DF8073017F09FFE03A9284616F0DF
:1053E00093FE08B92D4B03933022002104A8B3F09B
:1053F000E5FAA3238DF8103095238DF811308CF049
:1054000051FD04F5A042CDF81300D2F81035ADF8E7
:105410001B3004F58053D2F81425CDF81710462020
:10542000D3F86014D3F86434ADF81D10ADF81F2024
:10543000ADF8213062F02CF810EE103A1520CDF8BE
:10544000233062F025F810EE103ACDF8273004F53D
:1054500031539FED137AD3ED377A67EE877A28467A
:1054600017EE903ACDF82B30029BCDF82F309DF8F7
:1054700007308DF83330039B0D9318F053F804F583
:1054800080433022D3F8043F8DED0E0A04A904F5C1
:105490007C600F9355F066FC11B030BD2292CA7F3C
:1054A0000000C84270B58EB035220446002168461F
:1054B000B3F084FAA3238DF8003095238DF80130E2
:1054C000012304F5A0458DF802308CF0EBFC04F5C7
:1054D000405605F59363CDF803001B68D6F8A40584
:1054E000CDF80710CDF80B3003681B699847ADF86D
:1054F0000F00D6F8A40503689B689847ADF8110023
:105500001C4802F01DF8ADF81300D6F8A405036896
:105510005B69984710EE103AD6F8A405CDF815301F
:1055200003689B69984710EE103ACDF8193004F5DE
:10553000804303F6FC6135220968CDF81D10D5F8CB
:105540002017CDF82110D5F82417CDF82510D5F85F
:105550001C17CDF82910D5F8341BD3F8F43ECDF83C
:105560002D1004F57C606946CDF8313055F0FAFB1A
:105570000EB070BD702B002030B587B016220446E7
:1055800000216846B3F01AFAA3238DF80030952362
:105590008DF8013002238DF802308CF083FCCDF8B9
:1055A00003002046CDF8071005F020F804F5AA43C3
:1055B0008DF80B001B680393134B1B68D86A90F897
:1055C0009C308DF810300368DB69984704F5A045DE
:1055D0008DF8110095F8E9348DF812302DF0E8FEC1
:1055E0002DF036F8D5F8FC348DF813008DF8143012
:1055F000162295F8EA348DF81530694604F57C607A
:1056000055F0B0FB07B030BD6C2B002010B58AB050
:105610002722044600216846B3F0D0F9A3238DF871
:10562000003095238DF8013009238DF802308CF07D
:1056300039FCCDF803000420CDF8071061F028FFF5
:1056400010EE103A1320CDF80B3061F021FF10EE70
:10565000103A4620CDF80F3061F01AFF10EE103AE4
:105660001520CDF8133061F013FF10EE103A03202F
:10567000CDF8173061F01CFF10EE103A1A20CDF86B
:105680001B3061F005FF10EE103ACDF81F3004F525
:105690009E43103327221B68CDF82330694604F55A
:1056A0007C6055F05FFB0AB010BD000013B50446E6
:1056B00000F57C60019054F093FE019854F02AFFAD
:1056C00004F58053019893F978300BB154F0CAFF78
:1056D000204602B0BDE81040FFF798BF70470000B9
:1056E00030B500F5A04389B093F8E428044600F5EE
:1056F0007C6552B1D3F8FC071E22694686F01AFD7C
:105700000F496A46284655F0C9FC04F58043D3F892
:10571000C00E03685B68984704F50053014693F890
:105720000421284655F0DEFC04F59350083018F0AB
:1057300097F904F5907009B0BDE8304026F04CB9F7
:10574000B4DA0C089FED020A00224CF033BB00BF14
:105750000AD7233C134B70B5044640F8043B60F075
:10576000F1F9114E114B63605425601960F0A0FBF4
:1057700066513035B5F5557FF7D104F5557062F0B7
:105780007DFA0B4A04F5EC6002F6343189F03AFDFB
:1057900001232046074984F891394CF01BFD20462F
:1057A00070BD00BFB0370020D42A0D08E82A0D08CC
:1057B000B44C0020E41A0D082DE9F04100F5065123
:1057C0009AB00D22044653F0F5FE0022BD48272171
:1057D0004CF068FA0421002062F0DAF9132101206C
:1057E00062F0D6F94621022062F0D2F91521032099
:1057F00062F0CEF961F09CFF04F5A04393F99C3868
:1058000023B19FEDB10AB1484DF084F84CF0E8FEA9
:10581000AF4AB04E138843F0040313804FF00008E2
:105820000AAF002110223846B3F0C8F801238DF8E2
:1058300030303388ADF8283005A973680B933846AB
:105840004CF038F9C8B19DF91430002B15DD60F02B
:10585000F9FA9DF81410036801391B68C9B298471A
:1058600058B1051D28464CF06FF830B9B368ADF853
:10587000183006A928464DF067FB08F10608B8F174
:105880002A0F06F10C06CCD1934800220DF10B0132
:105890004BF042FE06AD064620B34CF055F808BB6F
:1058A0008E4B0FCB85E80F0004A928464CF002F977
:1058B000002840F033814FF00408894B0FCB87E874
:1058C0000F0005A938464CF0F5F828B105A84CF0B2
:1058D0003BF808B148F0010803A930468DF80C8068
:1058E0004DF0E0FA7F4B0FCB85E80F0003A9284667
:1058F0004CF0E0F8002846D00998002204A94BF0AB
:105900000BFE064600283ED04CF01EF80546002847
:1059100039D19DF80C30013BDBB2032B96BF724AA4
:105920000346D35C8DF82830304639464DF0BAFA3C
:105930006E48002205A94BF0EFFD06466AF0B0FD67
:1059400078B16AF0ABFD90F8302090F8281090F80C
:105950004830114490F840200A44D34214BF012536
:10596000002586B130469DF90C804BF0EDFF50B913
:105970001DB1B8F1000518BF0125394630468DF834
:1059800028504DF08FFA04F506500022B7EE000AB9
:10599000022138304CF00EFA012304F5F451009343
:1059A000534A002310318E204CF080F994F974C9C9
:1059B000BCF1000F1AD14F4E0FCE3D460FC50FCE92
:1059C0000FC50FCE0FC596E80F0085E80F006246A1
:1059D000042138464CF066F99FED470A47484CF0E1
:1059E00099FF4748B7EE000A4CF094FF012504F5F3
:1059F0000151444A00950023083140F205104CF053
:105A000055F904F5075002212C30FFF79BFE04F5F1
:105A1000055003211430FFF795FE04F505500321CE
:105A20001C30FFF78FFE04F5075003212830FFF7E5
:105A300089FE04F5075002213030FFF783FE04F59C
:105A4000055002212830FFF77DFE04F505500221A4
:105A50002C30FFF777FE04F5055002212430FFF7C4
:105A600071FE04F5AC40383088F0D4FE264A136845
:105A7000D90705D42549156004F5FF5310330B6091
:105A800004F5085021490122283001254CF060F925
:105A90001F4A0095002304F57C61FD204CF006F9B7
:105AA0001C4B1A68D20705D41B4A1D6004F58C54A0
:105AB0000C341460184801214CF066F91AB0BDE8A6
:105AC000F08100BF20180D08000096438CFF0D08E0
:105AD000E0870020901A0D08E4170D0878CB0C0819
:105AE00088CB0C0898CB0C081C180D08EF170D0874
:105AF000E45B0D08A8CB0C0800000000FC170D08A3
:105B00000B180D0848640E08642B002000220020AA
:105B100008E80D08682B00200C22002004A84BF098
:105B200013FF00283FF4C7AE4FF00C08C5E600BFD6
:105B30007047000000207047002070470020704729
:105B40000020704700207047704700000020704719
:105B50000020704784B001A880E80E0004B0002047
:105B60007047000000207047002070477047000019
:105B70001020704700487047D0260D080048704735
:105B8000E0260D0800207047704700000120704794
:105B90000120704700207047002343608360C3608A
:105BA00003614361002303767047000010B504468B
:105BB000FFF7F2FF0023637610BD0000027E531C46
:105BC000DBB2042B037600EB820288BF002382ED58
:105BD000010A88BF0376704710B50446FFF7EEFF51
:105BE000D4ED017A9FED107A94ED020A637E77EE90
:105BF000877A042B77EE807A94ED030A94BF013301
:105C0000052377EE807A94ED040A637677EE807A46
:105C1000637E94ED050A77EE807A00EE103AB8EED6
:105C2000C00A87EE800A10BD0000000010B50446CF
:105C30001DF028FD204610BD04F0ECB902F0F0BFC5
:105C400003F0C4BD02F0FABF01F084BC01F034BB24
:105C500001F05EBC01F0F4BCFCF7F6BFFCF7B0BB92
:105C600070B51F4B036000F540530446D3F8380568
:105C70001C4AC3F8882308B11DF008FD1A4B2360A5
:105C800004F5805393F82C2E42B9D3F8285E2DB139
:105C900028462AF0A1FD28461DF0F4FC04F58B509F
:105CA000103079F065FE04F58350183063F0E6F8A3
:105CB00004F6C44504F66446B54204D0183D2846AF
:105CC0002AF0DEF9F8E7094BC4F8983804F6941086
:105CD00057F004F804F5106057F000F8204670BD46
:105CE0008C0E0D08A0000E0874E10D08C8A90D085F
:105CF00038B5484B044640F8043B63F005FC04F11A
:105D000010001AF079FF04F1680052F007FE04F564
:105D1000907025F043FA04F5866019F003FE04F252
:105D200054501DF0B5FC04F698002BF0F1FD04F57D
:105D3000446063F0C7F904F551604DF07FFC04F551
:105D40007C6054F057FF04F58350183063F07EF800
:105D500004F5855014301CF041FA04F58B501030D6
:105D600079F0F2FD04F58C500C3053F099F904F5FC
:105D70008F5064F073FD04F580530025264A83F8A4
:105D8000045204F5905004F590530433143013601A
:105D900049F07CFA04F593502946083015F096FE38
:105DA00004F5C550183072F0CBFC04F5E5501C30FA
:105DB00076F010FE04F5EE50143078F01FFF04F575
:105DC000F150183079F054FB04F5F450103014F011
:105DD0009FFD04F5FF50103073F010F904F50150E9
:105DE000083069F033FE04F5005304F5045083F8DD
:105DF00004510A4D1C307AF07BF92B6813B1084826
:105E00008CF016F8204607494CF0E4F92C60204647
:105E100038BD00BF74E10D08D0900020308800200C
:105E2000E8260D089CE00D082DE9F04F2DED028BC2
:105E300004469FB0FFF75CFFE24B236004F5085077
:105E40002830FFF787FC04F52F5004F500577BF04E
:105E500049FC04F507530A33C7F8E83B04F5305012
:105E6000062387F8EC3B143062F002FC04F5315352
:105E700038330E9304F5AC433833C7F8903C0F9396
:105E80004FF40063C7F8943C5A2387F8143D04F597
:105E9000055907F6784304F5935809F10409CA4AED
:105EA000DFEDCA8AC7F88C9C08F10808C7F8888C0F
:105EB000B7EE008AC3F8602104F53950C44AC3F82C
:105EC0006821C3F8CC2183ED578AC3ED598A143079
:105ED00057F024FA04F53950203057F01FFABD4B23
:105EE000C7F8703E0E9B002687F8886E03F5FC709D
:105EF000FFF752FEB84BB949C7F8703E87F8896E74
:105F00000E984CF067F9B64BC7F8903E0E9BC7F859
:105F1000983E07F569630022C7F8948E04F53A5558
:105F20005A63DA6304F53B50012387F8D43E1035F9
:105F300028301CF09FFF87F8F86EAA4928464CF0DD
:105F400049F904F53B5049463C307BF081FF04F5AC
:105F50004150494614307BF0DFFB04F5465049467A
:105F600004F540572C307CF03DFB2C22314607F5E0
:105F70005470B2F023FD04F54C509B49203004F5D9
:105F80004E564CF027F90836984BC7F8883306F17F
:105F900008008BF035F904F54E5A04F5505B0AF110
:105FA000340A0BF1180B50460AF1140A5BF0AAFFF1
:105FB000D345F8D10723C7F83C350023A7F840356F
:105FC0004FF4CB701DF05CFBC7F8380504F5555055
:105FD00004308BF015F904F5565008308BF010F9A9
:105FE000834B1A6802B91E60824BC7F8883304F5E8
:105FF00056504FF48051C7F8A45528301AF0D6FEF9
:1060000004F5585028304DF055F804F558503C3000
:106010006BF0C2FD04F5964004F58045143004F0A1
:1060200035FF754BC5F8143B04F59640303004F04D
:106030002DFF724BC5F8303B04F596404C3004F010
:1060400025FF6F4BC5F84C3B04F59640683004F0D3
:106050001DFF6C4BC5F8683B05F53963002204F55C
:106060009740DA609A605A6083ED008A243004F029
:106070000DFF654BC5F8A43B04F59740403004F094
:1060800005FF624BC5F8C03B04F597405C3004F057
:10609000FDFE5F4BC5F8DC3B04F59840043004F08E
:1060A000F5FE5C4BC5F8043C04F59840203004F044
:1060B000EDFE594BC5F8203C04F598404C3004F0F7
:1060C000E5FE564BC5F84C3C04F59840683004F0AA
:1060D000DDFE534BC5F8683C04F59940043004F5E7
:1060E000994604F0D3FE24364E4BC5F8843C304626
:1060F00004F0CCFE4C4BC5F8A43C04F5994040306C
:1061000004F0C4FE494BC5F8C03C04F599405C302E
:1061100004F0BCFE464BC5F8DC3C04F599407830F1
:1061200004F0B4FE434BC5F8F83C04F59A40143033
:1061300004F0ACFE404BC5F8143D04F59A403430F1
:1061400004F0A4FE3D4BC5F8343D04F59A405030B0
:1061500004F09CFE3A4BC5F8503D04F59A4070306F
:1061600004F094FE374BC5F8703D04F59B400C30AD
:1061700004F08CFE344BC5F88C3D04F59B40283070
:1061800007F0E0FE04F59B40643004F07FFE2F4BE7
:10619000C5F8E43D2E4BC5F8003E4FF4C053A5F8BA
:1061A000543E2C4904F59C404CF014F8FE2385F82D
:1061B000CC3E052385F8F03E4FF0FF3B264BC5F85B
:1061C000C06E4BE08C0E0D08000080BF0000B44292
:1061D0000000B4C220270D0830270D08E09B0E08F0
:1061E00040990E08E8980E0840970E08A0000E0887
:1061F0004C8B00207CDA0C0830320D082C390D084D
:106200004C3C0D082C300D0840330D08C8330D08E8
:10621000A8320D08B0310D082C310D08BC380D081E
:10622000B8340D0848340D0868270D0838350D08B6
:1062300044380D0838360D0828370D08A8360D08E3
:10624000C0370D08B8350D08BC2F0D08C83B0D0828
:1062500058270D08A0BC0E08395C0108C5F8C46EAB
:10626000C5F8F8BE119305F57165894B85ED008A77
:1062700004F59E4004F5A04522464FF400710093BA
:106280001430844B10941AF029F804F5A943C5F88A
:1062900070B4C3ED038A03230026C5F8FC3405F56A
:1062A000A363C5F8C864C5F8CC64C5F8D064C5F864
:1062B000D464C5F8D864C5F8DC6483ED008A764BF5
:1062C000C5F84035754BC5F8483504F5AA40744B00
:1062D000C5F85035C5F83C45C5F84445C5F84C45AA
:1062E00064301CF0C7FD04F5AB401CF0C3FD04F5A1
:1062F000AB4004F5AA4A1C301CF0BCFD0AF1200A90
:10630000684BC5F8B035A5F8B4B50AF198001CF093
:10631000B1FD654B6549C5F814B65046C3F800A0F9
:106320004BF058FF4FF6FF73A5F85C3504F5AC4011
:106330005F4B6049A5F878B5183018604BF04AFFFC
:106340005D4BD7F8A4251294CDE913345B4BCDE90E
:1063500015345B4BCDE917345A4BCDE919345A4B00
:10636000CDE91B34594B1D931EA911E903000CAB59
:1063700083E80300DDE91A010AAB83E80300DDE9E5
:10638000180108AB83E80300DDE9160106AB83E8DA
:106390000300DDE9140104AB83E80300DDE9120129
:1063A00002AB83E803005146CDE900290E9B0F980C
:1063B000424688F039F808F51B7304F5AD40C5F87E
:1063C000F43678301CF056FD04F5AE4008301CF071
:1063D00051FD04F5AE40183004F5AF471CF04AFDFE
:1063E00008371022314605F5E560B2F0E7FA384685
:1063F00079F038FF364B3749C5F8883738464BF0C7
:10640000E9FE354A3549116004F5AF43403314279E
:10641000B0B207FB00120136127C002AF8D1304AD4
:106420001080304A166816B12F488BF001FD04F534
:10643000AF404430136079F0FFFE2C4BC5F8C437F1
:1064400004F5AF404146503009F08AF8284BC5F8B2
:10645000C83A642385F8CC3A264BC5F8003B04F5CE
:10646000B540254BC5F8043B244948304BF0B2FEFB
:10647000234BC5F8C83A20460123C5F8286B85F898
:10648000306B85F8B0341FB0BDEC028BBDE8F08FE7
:106490005CD70C08395C01083D5C0108415C0108CF
:1064A000455C01080000FFFF2887002000B80D08A8
:1064B000D4900020AC0E0E08495C01084D5C010828
:1064C000515C0108555C0108595C01085D5C0108DC
:1064D00040D10C0818D10C08F0870020941C0D083E
:1064E000EC870020AC870020FC260D0880D10C082A
:1064F00040270D0838580D0890580D0888070E08D9
:10650000105A0D0810B58BF0F1F8064C064B1860C8
:106510002046FFF789FC2046044A0549BDE81040A3
:10652000AFF00ABD702B00206C2B0020ECE20020A5
:10653000615C01080069C0F3401070470F299DBFDE
:10654000302303FB0100503000207047014B93F9CA
:10655000C9017047704B0020014BD3F8D40B704732
:10656000704B002008B503689B68984730B9044B0E
:1065700093F8DA0EB0FA80F0400908BD0020FCE77D
:10658000706B002008B504480EF062FD10B9034B93
:1065900093F8D40E08BD00BF702B0020706B002054
:1065A000022A10B50C4605D1BDE810400948352235
:1065B00010F0ACBC084BD3F8C00E03685B6898477A
:1065C000A04205D15FF03EFCBDE810405FF0C4BBC7
:1065D00010BD00BF702B0020706B0020012910B58A
:1065E0000C4610D0022904D061B95EF089F9084A3E
:1065F00002E05EF085F9074A062157F025FB064BBD
:10660000C3F8684810BD5EF07BF9044AF4E700BFA8
:1066100080280D0858280D08707B00206F280D0871
:10662000012910B50C4614D0022907D0D1B90E4B60
:10663000C3F8281B5EF064F90C4A05E00A4BC3F866
:10664000281B5EF05DF90A4ABDE81040062157F0AC
:10665000FBBA5EF055F9074A062157F0F5FA024BEE
:10666000C3F8284B10BD00BF707B0020BF280D0869
:1066700094280D08A8280D08012903D0022914BF69
:1066800000210221014BC3F8741B7047704B00209E
:10669000012902D0022900D011B9024BC3F82C1BEA
:1066A000704700BF707B00206C2910B400F3A680F7
:1066B0003F290FDC162900F39980032940F39A80C3
:1066C0007E4B01248C402340002B00F093805DF82A
:1066D000044B7047A1F140032C2B00F28B8001A4E6
:1066E00054F823F09D680108F5670108F567010873
:1066F000F5670108F5670108F5670108F567010806
:10670000F5670108CF660108F5670108F56701081C
:10671000F5670108F5670108CF660108F56701080C
:10672000F5670108F5670108F56701089368010836
:10673000F567010893680108F56701089368010887
:106740009368010893680108CF660108F56701089E
:1067500093680108CF660108F5670108F56701082D
:10676000CF660108CF660108F5670108CF6601080A
:10677000F5670108F5670108F5670108F567010885
:10678000F5670108F5670108F5670108F567010875
:10679000CF660108CF660108112B2BD801A454F84D
:1067A00023F000BFCF660108F5670108F56701080F
:1067B000F5670108CF660108F5670108F56701086C
:1067C000F5670108F5670108F5670108F567010835
:1067D000F5670108CF660108CF660108F567010873
:1067E000F5670108CF660108CF660108A1F127030C
:1067F000112BD1D95DF8044B60F036B9A0291FDC0C
:106800009529F7DDA1F196030A2BF3D801A454F8DA
:1068100023F000BFCF660108F5670108F56701089E
:10682000F5670108CF660108CF660108F567010822
:10683000CF660108F5670108F5670108936801084C
:10684000B52921DCA929D5DDA1F1AA030B2BD1D8CB
:1068500001A454F823F000BFCF660108F5670108D2
:10686000F5670108CF660108F5670108F5670108BB
:10687000CF660108F5670108F5670108F5670108AB
:10688000F5670108CF660108A1F1D003022BB1D84A
:106890001DE75DF8044B002360F0B8B8084B0122F7
:1068A00083F8242BA3F54053D3F8D00B00283FF4F2
:1068B0000EAF5DF8044B64215FF00ABB100041008D
:1068C000707B00206C2938B50346154600F3A28082
:1068D0003F2912DC38290ADC26296FDC102900F058
:1068E0000581162900F08A81042900F016812A46C4
:1068F0001846BDE838405FF07FBEA1F140022C2A67
:10690000F5D801A050F822F0C56A0108EF68010827
:10691000EF680108EF680108EF680108EF680108F7
:10692000EF680108EF680108F56A0108EF680108DF
:10693000EF680108EF680108EF6801081F6B0108A4
:10694000EF680108EF680108EF680108EF680108C7
:10695000676B0108EF680108BB6B0108EF6801086D
:10696000716B0108B16B01085D6B0108F36B0108E5
:10697000EF680108DB6B0108256B0108EF6801086F
:10698000EF680108B36A01080B6C0108EF680108A1
:10699000036B0108EF680108EF680108EF68010860
:1069A000EF680108EF680108EF680108EF68010867
:1069B000EF680108936C01082B6B0108A1F1270215
:1069C000112A94D801A050F822F000BFB36A010840
:1069D000EF680108EF680108EF680108B76A01086D
:1069E000EF680108EF680108EF680108EF68010827
:1069F000EF680108EF680108EF680108156B0108EE
:106A0000FD6A0108EF680108EF6801080F6B0108D3
:106A1000096B0108A02921DC95297FF768AFA1F156
:106A200096020A2A3FF663AF01A050F822F000BF99
:106A3000156C0108EF680108EF680108EF680108AC
:106A40001B6C01086D6C0108EF6801087B6C010884
:106A5000EF680108EF6801083B6C0108B52923DCE9
:106A6000A9297FF744AFA1F1AA020B2A3FF63FAF55
:106A700001A050F822F000BF316B0108EF68010857
:106A8000EF6801085B6C0108EF680108EF68010816
:106A9000376B0108EF680108EF680108EF6801082B
:106AA000EF680108B36C0108A1F1D002022A3FF699
:106AB0001EAF01248FE0A91E864B4D424D4183F845
:106AC000CD5EF6E7AA1E5542834C554184F8235B00
:106AD0005DF016FF814A94F8231B814B002908BF03
:106AE0001346804A062157F0AFF8E2E70A21FFF784
:106AF00057FDDEE72A4601211846F8E72A46042119
:106B0000FAE72A460321F7E72A460C21F4E72A464A
:106B10000F21F1E72A460021EEE70B21E7E72A469D
:106B20000D21E9E72A460521E6E72A461521E3E794
:106B30002A461121E0E7AB1E5A425A41664B93F8B0
:106B4000C8189142B5D083F8C8285DF0D9FE664ACE
:106B5000664B022D08BF1346654AC3E7294618460F
:106B6000FFF78AFDA5E729461846FFF737FDA0E79E
:106B7000594CD5B1022D0DD1012384F8203BA4F549
:106B80008053D3F8C00E03685B6A984710B1594828
:106B900000F070FB5DF0B4FE534A94F8201B534B99
:106BA000002908BF1346544A9CE784F8205BE6E7B7
:106BB00029461846FFF734FD7BE7012445B1022D35
:106BC00009D1454BC3F82048002283F8102902E080
:106BD000414BC3F82058204638BD01242DB1022D69
:106BE000F9D1464B83F8DC4FF5E7444B83F8DC5F83
:106BF000F1E729461846FFF74BFD5AE7022A7FF4D2
:106C000058AF3C4808F0E4FA53E75FF01BF95FF037
:106C1000A3F84EE72A4607216EE7184629465FF09B
:106C20001BFC374879F05EFB044600283FF441AF77
:106C3000294B0122C3F82028C6E7274BD3F8E038B8
:106C4000002B3FF436AF012425B1022DC3D183F8C8
:106C50002C40C0E783F82C50BDE7022D7FF429AF0C
:106C60009FED280A2348FBF71BFC22E7022D7FF447
:106C700020AF20480EF0FAF81BE701242DB1022DB9
:106C8000A9D1154B83F8224BA5E7134B83F8225B60
:106C9000A1E7022D12D10F4DD5F8C00E0368DB6BB2
:106CA0009847044678B10121A5F5804002F0CCFE5A
:106CB00091E71548294689F035FCFAE60D48002190
:106CC00002F0C2FEF5E65DF01BFE104A042156F00C
:106CD000BBFFEEE6706B0020707B0020D4280D080F
:106CE0001F110D08DC280D0828FB0C0898390D0829
:106CF000EC280D08702B0020F8280D08703B0020B0
:106D0000F882002000000000707900200B290D0897
:106D100010B599B104681168416004B90160126846
:106D200001681B68521A9A4202D80021084610BD19
:106D3000017A012381F001010372F7E7037A3BB185
:106D400044682CB11368029A12681B1B9342ECD959
:106D50000023C0E90033EFE70023C0E90533C0E9B1
:106D600008338385037780F828307047F0B52DED20
:106D7000028B044687B0A148B0EE408A0F4679F0F6
:106D8000BBFA40B1236933B1206B00F50E7010F0EF
:106D9000B5FB054638B12046FFF7DEFF002007B0FF
:106DA000BDEC028BF0BD236B93F93C22002A1EDD63
:106DB00093F8A032DBB1924ED6F82C2B002AEAD100
:106DC0002369D4ED007A991E4842F5EEC07A484115
:106DD000F1EE10FA84F82C0027D8C4E90822C4E99F
:106DE000052284F82D2084F828202277D7E7854EC5
:106DF000D6F8C00E03689B6B984728B106F58056FD
:106E000096F8F834002BD6D07F4800210EF0B2FB64
:106E1000DFED7E7AB4EEE70AF1EE10FACBDA7A48CB
:106E200003F0E4FB0028C6D1B5E76FB1F4EEC87AF1
:106E3000F1EE10FA3CDD236BD3F8C432DB0403D54A
:106E4000734815F011F9074684F82D708BF022F87D
:106E5000D4ED027A9FED6F7A039067EE877AFCEEAD
:106E6000E77A17EE903A5B000593B4F90630CDED62
:106E7000047A002B1EDC0023C4E9083384F8283090
:106E800094F90430002B41DC0023C4E90533237757
:106E900094F82C00002882D194F82D0000287FF46B
:106EA0007EAF94F8280000287FF479AF207F76E742
:106EB0001746C9E70421544800F0AEFCB4F9063087
:106EC00007EE903AF8EEE77A05ABF4EEC07AF1EE11
:106ED00010FA0093CCBF0121002104AB03AA04F1F6
:106EE0002000B0EE408AFFF713FF0028C8D05DF005
:106EF00007FD074618EE100AF9F7FEFA464ACDE9F3
:106F000000010421384656F09FFEB9E7434F9FED3C
:106F1000447AD7F86024DFED436A07F58051D1ED5C
:106F2000597A82EAE270B0EE476AA0EBE270A7EE0F
:106F3000A66A07EE900AF8EEE77AF4EEC67AF1EE6A
:106F400010FA56D8D7F8640491ED5A6A07EE900A01
:106F5000A6EE267AF8EEE77AF4EEC77AF1EE10FAAA
:106F600047D591ED5B6A9FED307AA6EE267AF4EE76
:106F7000C77AF1EE10FACCBF4FF0010C4FF0000CC5
:106F8000642113FB01F1D6F81035D21A002AB8BFDC
:106F900052428A4230DAD7F86424D6F81435D31A2C
:106FA000002BB8BF5B428B42ACBF0023012304F12E
:106FB0001400BCF1000F01D183F0010505AB009373
:106FC00003AA04AB2946FFF7A3FE00283FF460AFF5
:106FD0005DF096FCD7F86014D7F86424642392FB24
:106FE000F3F291FBF3F300920421104A56F02CFEC9
:106FF0004EE74FF0000CC3E70023D8E7F8820020EB
:10700000707B0020706B0020702B0020000000348B
:10701000D83D002000007A44042B0D08703B00206E
:107020000000FA430000C8420000FAC3152B0D0807
:1070300073B58289036BD20704466CD493F93C2262
:10704000002A03DD93F8A022002A64D1524DD5F81E
:10705000C01E05F5576291425DD0A5F54055B3F9C4
:107060000860D5F8603407EE903AD5F86434B8EE8D
:10707000E77A07EE903AF8EEE77A6846CDED017AC6
:107080008DED007A2FF0A2FE730007EE903AF8EE35
:10709000E77AB0EEC00AF4EEC07AF1EE10FA42D40C
:1070A000236B93F8F1223AB307EE906AF8EEE77A91
:1070B000F4EEC07AF1EE10FA1EDB002183F8F11233
:1070C000236B586B81F002FE236B9FED347ADA6BF1
:1070D000D2ED067A05F26C6267EE877A92ED007A5D
:1070E000F4EEC77AF1EE10FA06D5986B84F04EF8FC
:1070F000236B986B83F0E4FDA389226B13F00203EA
:1071000002D192F8F11299B9002382F8F232236B7E
:1071100093F8F10205E0002083F8F102236B83F875
:10712000F20202B070BD236B012283F8F122B7E7AF
:1071300005F28451D1ED007A9FED197AF0EEE76AFD
:10714000F4EEC76AF1EE10FADFDD05F27C51D1ED05
:10715000006A9FED146AB0EEE67AB4EEC67AF1EEFC
:1071600010FAD2DD104991ED007AB0EEC77AB4EE94
:10717000C67AF1EE10FAC8DD67EEA67AF5EEC07AAF
:10718000F1EE10FAC1D5D5F8643408498B42ACBF92
:1071900000230123B9E700BF706B00200AD7233C0E
:1071A000C2B8323E920A063FF04000206CEEFFFF6C
:1071B00008B5036B93F8F2223AB1DA6A92F8A0208C
:1071C000022A03D0002283F8F22208BD0B4B9FED68
:1071D0000C0AD3ED007AF5EEC07ADFED0A7AF1EE13
:1071E00010FAD8BFB0EE670A152060F03DF9BDE88F
:1071F00008409FED050A132060F036B9F4400020E6
:1072000000A08CC500A08C450000000000F5804067
:10721000D0F8C00E03681B6C1847000000F500533F
:1072200093ED7A7A00F5A040B5EEC07AF1EE10FA4F
:107230005DBFD0F8F436DFED086AD3ED017AD0F8FF
:107240000C075FBFF8EEE77AE7EE267AFDEEE77A05
:1072500017EE900A704700BF0000C84200F50050CA
:1072600090F8200228B141F00101084214BF01202A
:107270000020704700F5A040D0F80C37C0F8283740
:107280000023C0F82C37704700F5A0404A68C0F8CA
:1072900028270B78DB0741BFD0F8F4365B689B18D2
:1072A000C0F828377047000000F5A040D0F8283714
:1072B0001944C0F82817704710B54B68516800F59D
:1072C000A0448B42D8BF0A46D4F82807CCBF1A4640
:1072D00019462CF049FEC4F8280710BD10B5044625
:1072E000414868F00FFD10F0080217BF3F4BDFED7B
:1072F000407A93ED157AD3ED177A1FBF77EE877A30
:107300009FED3C7A012267EE877A10F0010317BFE8
:10731000364B9FED377AD3ED176A93ED147A1CBF85
:1073200037EE667ADFED336A04F5005118BF27EEB9
:10733000267AD1ED7C6AF5EEC06A18BF0123F1EE22
:1073400010FA4BDD294A9FED2B6AD2ED7C6A66EE7E
:10735000866AF4EE676AF1EE10FA58BFF0EE667ACC
:10736000F3B11A4604F5A043D3F8F416D1ED016A3F
:10737000D3F82817F8EEE66A76EE876A07EE101A59
:10738000B8EEC77AF4EEC76AF1EE10FAD8BFB0EEE5
:10739000667ABDEEC77A17EE101AC3F828170AB33B
:1073A00004F5A044D4F8F43693ED017AD4F82837E4
:1073B000B8EEC77A77EE277A07EE103AB8EEC77ABA
:1073C000F4EEC77AF1EE10FA58BFB0EE677ABDEE70
:1073D000C77A17EE103AC4F8283703E0002ABFD165
:1073E000002BBFD110BD00BFB84B0020704B002058
:1073F000000000000000C84200F5A0400023C0F8D3
:107400002C37704713B500230446104601AA019398
:107410001BF0ECFD034648B1DDED017A9FED177AD4
:1074200067EE877AFDEEE77A17EE903A04F5A04111
:10743000D1F8FC24C1F82C37042A1DD004F50054DF
:10744000B4F91A22002A14DD83EAE370A0EBE3709A
:1074500007EE900A9FED0A7AF8EEE77A67EE877AF0
:1074600007EE102AB8EEC77AF4EEC77AF1EE10FAFA
:1074700002D50023C1F82C3702B010BD0000C8426D
:107480000AD7233C0B78D1ED017A00F5A04013F028
:10749000010F1CBFD0F8F43693ED017AF8EEE77ACD
:1074A00018BFB8EEC77A00F20C7318BF77EE877A70
:1074B00093ED007AB8EEC77AB4EEE77AF1EE10FAFF
:1074C000CCBF0120002070477047000000F500533A
:1074D00000F58042B3F9D231D2F8C02E00EE103A56
:1074E00000F5984320339A42B8EEC00A0ED100F559
:1074F000A040D0F8FC34042B02D090F8B1342BB16A
:1075000000F5C760D0ED007A30EE270A7047000022
:10751000014608B501F5A041FFF7D8FF01F20C7351
:10752000D3ED007A9FED057AF8EEE77AE0EE477A40
:10753000FDEEE77A17EE900A08BD00BF0000C842D2
:1075400010B5044604F5A044FFF7E2FFD4F828374D
:10755000181A10BD70B504462DED028B04F5A04538
:10756000FFF792FEDFED340A40F24310B7EE001A47
:107570000E462CF059FCD5F82C27534207EE903AD2
:10758000F8EEE77AD5F8283767EE807AB0EE408AD1
:10759000FDEEE77A17EE901A1944C5F8281704F59E
:1075A0000053D3ED876AF5EEC06AF1EE10FA3FDDC5
:1075B000002A3DDD2046FFF7C3FF9FED207A07EE4E
:1075C000900A66EE876AF8EEE77AF4EEE67AF1EE74
:1075D00010FA2DD531462046FFF756FE04F5AE4190
:1075E000324608312046FFF70DFFD5F82C275342CD
:1075F00007EE903AF8EEE77AD5F8283767EE887A02
:10760000B5EEC08AFDEEE77AF1EE10FA17EE901AA9
:107610001944C5F828170BDD07EE902AF8EEE77A33
:1076200087EE887ABDEEC77A17EE103AC5F82C3788
:10763000BDEC028B70BD00BF000000000000C8C29E
:10764000014608B5FFF742FF01F5AE40D0ED0E7AD6
:1076500037EEC00ADFED047A20EE270AFDEEC07A8D
:1076600017EE900A08BD00BF0000C8422DE9F041A6
:1076700000F5AE4800F5AE4508F108081835044697
:10768000294640461BF026FF04F5A04704F5AD4609
:1076900007F5936378362A46314683ED000A404663
:1076A0001BF04EFE07F29C43DFED220A83ED000A39
:1076B000B7EE001A76202CF0B7FB04F5315383EDBA
:1076C0007F0A2046FAF77CFE04F58043D3F8C00E0B
:1076D00003685B6898470B280BD006D80A280FD0A0
:1076E0000023C7F82C37BDE8F0810E38C0B201285E
:1076F000F6D829462046FFF7C5FE0028F0D011E055
:1077000029462046FFF7BEFE30B90B484FF48041B2
:10771000FBF78AF90028E3D12046FFF791FFB0F587
:10772000FA6FE6DD2A4631462046BDE8F041FFF714
:1077300069BE00BF00000000702B002010B500F5EE
:10774000A04300F58054D3F81C2793F818379FED19
:10775000146A13F0010F07EE902A08BFD4F8D8344A
:10776000F8EEE76A08BF07EE903A66EE866A04BF55
:10777000F8EEE77AE7EEC66AFFF7CAFE04F59B6308
:1077800093ED000A07EE900AB8EEC00AF8EEE77A29
:1077900026EE400AA7EE860A30EE660A10BD00BF4C
:1077A0000AD7233C38B50446FFF758FD78B904F5ED
:1077B000AF45503528460AF03FFA28B3284609F06D
:1077C000DDFD08BB2046BDE83840FFF7B7BF04F534
:1077D000005595F8F03BDB0704D505F60C4595ED13
:1077E000000A38BD04F5AF4050300AF04BFA0028CB
:1077F000DDD095F8BA1B04F551604BF0EFFF02287D
:10780000D5D19FED040AECE704F5AE4494ED0E0AE1
:10781000E7E700BF000000000022FFF7C3BF000041
:1078200010B504468AF036FB04F50053D3F8042C57
:10783000801A41F2883290420FD802212046FFF789
:107840000DFD50B104F5A044D4F8FC24042A04D161
:1078500003F6F83393ED000A10BD9FED010AFBE734
:107860000000000008B52DED028B00F5A043014695
:10787000D3F8F426D3F828375268DFED0D8A9B1A27
:1078800008EE103AFFF722FEB8EEC88A0846A0EECE
:10789000288AFFF7C5FFBDEEC88AB8EEC88AA0EEF9
:1078A000288AFDEEC87ABDEC028B17EE900A08BD5F
:1078B0000000C842F0B52DED048B00F5005489B0EE
:1078C00000F5516694F8BA1B0391054630464BF01B
:1078D00085FF0399074630464BF092FF042F03992A
:1078E000B0EE408A21D1002305A88DED050A06934C
:1078F00007932FF0EBFC05F5AC5005A908302DF0EF
:10790000B3FBDFED997A8DED050AB4EEE71AF1EEDF
:1079100010FACDED060A8DED071A06DB05F580534A
:1079200093F8E47417F001070CD194F8F03B0022AF
:1079300062F3000384F8082C84F8F03B09B0BDEC36
:10794000048BF0BD94F8F03B9A075FBF43F002034D
:1079500084F8F03B04F6F43383ED008A04F60C431C
:1079600083ED001A94F8083C092B79D804F541639B
:10797000D3ED000A9FED7D9AB0EE480A2CF042F953
:1079800000BB04F6F43394F8BA1BD3ED008A3046FA
:107990004BF054FF07EE900A9FED757AF8EEE77A08
:1079A00078EEC88A67EE877AF0EEE88A67EE897A21
:1079B000F4EEE78AF1EE10FAC2BF94F8083C013306
:1079C00084F8083C04F5416394F8BA1BD3ED008AAF
:1079D00030464BF033FF07EE900AF8EEE77A9FED62
:1079E000657A67EE897A78EEC88A67EE877AF0EE74
:1079F000E88AF4EEE78AF1EE10FA02DD002384F85B
:107A0000083C04F5416383ED008A94F8F03BDA0703
:107A100094D52846FFF792FE04F60C4696ED008AB0
:107A200030EE488A8AF036FAD4F8042C41F28831D4
:107A3000821A8A42034604F6F83204F6FC315AD917
:107A400082ED008A284681ED008A0221FFF706FCBC
:107A500018B105F5AC456A6C2A64C4F8043C6DE7BE
:107A600094F8F03B43F0010384F8F03B05F5A043A4
:107A7000D3F8FC6405F58043301FD3F8C02E05F51C
:107A80009A43464203F1340346419A4212D005F527
:107A90009A4350339A420DD005F5984320339A42C9
:107AA00009D1354B05F5AF40B3F85E15503009F0FC
:107AB00081FC00B13E4694F8F03B5907A1D4002E5A
:107AC0009FD002212846FFF7C9FB002899D043F038
:107AD000040384F8F03B04F60C4305F54E56186891
:107AE000F8F70AFD0836CDE90001244A06213046A0
:107AF00056F0AAF885E79FED1F0A92ED007ADFEDB8
:107B0000207A28EE008AA7EE278A82ED008AC4F840
:107B1000040CD1ED007A38EE678AF3EE0E7AB0EEFF
:107B2000C88AB4EEE78AF1EE10FA7FF707AF94F84F
:107B3000F03B5B070CD53068F8F7DEFC05F54E54DA
:107B40000834CDE900010F4A0621204656F07CF8A2
:107B500005F52F5024220021303009B0BDEC048BF4
:107B6000BDE8F040B0F02ABF000000340AD7233C43
:107B7000CDCC4C3DCDCC4C3E707B00202C2B0D0849
:107B8000CDCC4C3F492B0D0838B52DED028B0D4661
:107B90000446FFF7D3FD002320462B70B0EE408A49
:107BA000FFF73EFE0221204638EE400AFFF756FB63
:107BB00028B104F5005494F8F00B00F00100BDEC7E
:107BC000028B287038BD000070B50B7803F00503F8
:107BD000042B05460C46164615D105F5A04552F076
:107BE000B3FAB2B24FF4801152F066FAD5F8F42627
:107BF000636852689B1A13F5FA7FC8BF63602378E5
:107C000043F00103237070BDF8B500F5805300F513
:107C1000A047D3F8D864D7F8C054B542044619D069
:107C20000E4A1268D26A92F89C209AB100F5AE41D1
:107C3000751B25221831FFF7C7FF07EE905AB8EEE3
:107C4000E70ADFED077A04F5315020EE270A3830D5
:107C50007DF0FEF9C7F8C064F8BD00BF6C2B0020B2
:107C60000AD7233CF8B500F5A044054694F8B3C400
:107C70000F4604F5DF66BCF1000F53D004F5E36353
:107C80000FCB86E80F00012384F8B43497E80F0087
:107C900004F5E36686E80F00D4F8203705F5AE4614
:107CA000183693B9D4F824377BB9D4F81037D4F800
:107CB0001C27C4F82037D4F81437C4F8243722B965
:107CC000D4F80C1730461BF0DBF831462822284642
:107CD000FFF77AFF94F8181711F0040102D130462B
:107CE0001BF060F905F5AD4105F5AE40324678313F
:107CF00008301BF05BFB38B104F5DF6604F5E16486
:107D000094E80F0086E80F00284606F0D3FC2846CA
:107D1000FFF7ACFC284607F0C7F82846BDE8F84056
:107D2000FFF774BA04F5E1630FCB86E80F00012377
:107D300084F8B33484F8B4C4A8E70000F8B500F5BB
:107D400000530446B3F97A31002B0E4634DB0B782E
:107D500013F0020F14BF4FF0FF33012304F5A045C9
:107D600005F5DF6785F8D03605F5E1630FCB87E8C9
:107D70000F0096E80F0005F5E36787E80F0004F5AC
:107D8000AE41572218312046FFF71EFF2046FFF76D
:107D900071FA20460026FFF769FC204607F084F8B8
:107DA00085F8B464C5F8D46685F8B964204606F051
:107DB00081FC85F81269F8BD4FF0FF33CEE7000073
:107DC0002DE9F043364B1B6885B00546D86AF9F7B4
:107DD000A3FB002861D105F5005393F9883B5A1C99
:107DE00054D0002B05F5866711DD95F84124242138
:107DF00007EE903A01FB027292ED0B7AF8EEE77A09
:107E0000B0EEC77AB4EEE77AF1EE10FA3EDC05F593
:107E1000805305F5935693F8E43413F0010406F10A
:107E2000080629D0C3F340089B0732D495F8E41321
:107E300095F828444FF0B00909FB015191F8C13180
:107E40004CBB022B18D968461BF014F86946304623
:107E500015F0B6F8044678B195F8E43309FB0353FE
:107E60004246D3F8D01168461BF00AF815F07EFBA5
:107E7000694614F093FF0446384617F027FE304653
:107E800014F0AAFE2846FAF7A1FD204605B0BDE889
:107E9000F0830024F0E74446EEE70020F6E700BF59
:107EA0006C2B002038B50C4B1B680546D86A0C4675
:107EB000F9F732FB10B10024204638BD15F056FB0F
:107EC000214614F06BFF04460028F4D005F5AA40C3
:107ED000203030F015F8EFE76C2B0020F0B500F5FE
:107EE000A045002385F8B33485F8B43405F5E16383
:107EF000044600EE101A0FCB87B005F5DF6686E862
:107F00000F0002AE04F5AE42B8EEC00A3046174983
:107F100008324BF0D7F996E80F0005F5E36787E8DC
:107F20000F0004F5AE4140F257121831204601917E
:107F3000FFF74AFE01992046FFF7C6FA019920464D
:107F4000FFF7A2F904F500532046B3F97A31002B6C
:107F5000B4BF4FF0FF33012385F8D036FFF786FB1F
:107F6000204607B0BDE8F04006F09EBF98610020B3
:107F700010B5034904464BF0A5F9204610BD00BFDB
:107F800098610020F8B500F5A04404F5E1630546CA
:107F90000E460FCB04F5DF6787E80F0006F10801F6
:107FA0002846FFF75FFEB388D4F81C2703EB830352
:107FB00003EB83039B001BB2002BD8BF4FF4C873A5
:107FC000A4F8AE34D4F8F4365968521AC4F88024B0
:107FD0009A680A32C4F82027DB680A33C4F82437C9
:107FE0000023C4F8943484F8B03484F8C434C4F85A
:107FF000843404F58F6300221A604FF0FF33C4F815
:10800000703495F8412405F58663242101FB023381
:1080100004F59564DB6A2360F8BD000070B50E4678
:1080200008310546FFF71EFEB38805F5A04443B3AB
:10803000642213FB02F3C4F88034B4F9AE34002B8D
:10804000D8BF4FF47A7305F52F50D8BFA4F8AE34DB
:10805000242200213030B0F0B1FC04F5E76305F5CF
:10806000AC4093ED000A3146383086F0D3FAD4F8AC
:10807000FC34072B0CD128460421BDE87040FAF7E8
:108080006DB9D4F88034002BD7DC40F6B833D2E792
:1080900070BD000030B5083104460FC985B06D468B
:1080A00085E80F0004F5AE41083128461BF01AF8A8
:1080B00020462946FFF7D6FD04F580440123C4F885
:1080C000E83E05B030BD00000B7A00F5A04013F08B
:1080D000020F14BF4FF0FF33012380F8D0367047F2
:1080E0007FB501F1080305460E460FCB6C4684E8C8
:1080F0000F0005F5AE41083120461AF0F3FF214686
:108100002846FFF7AFFD31462846FFF7DDFF04B0F4
:1081100070BD00007FB501F1080304460E460FCB89
:108120006D4685E80F0004F5AE41083128461AF087
:10813000D9FF29462046FFF795FD20463146FFF737
:10814000C3FF337907EE903A337E9B0748BF9FED1C
:108150000C7AF8EE677A04F5A04448BF67EE877A98
:108160009FED087A67EE877AFCEEE77A17EE903A91
:10817000C4F8C8360123C4F8E83604B070BD00BFA7
:108180000000803B00A00C477FB501F108030446C6
:108190000E460FCB6D4685E80F0004F5AE41083161
:1081A00028461AF09FFF29462046FFF75BFD204630
:1081B0003146FFF789FFB38804F5A0444FF47A7283
:1081C0005343C4F8E0360123C4F8E83604B070BD68
:1081D0002DE9F34100F5AE450446183500F5AD40F4
:1081E0000E46783029461AF03DFF04F5A047C0B985
:1081F0004FF0FF33C7F8703406F1080840461AF014
:1082000069FE032802463AD1F16828461AF038FE82
:10821000B388C7F8E836204602B0BDE8F041FFF762
:10822000EBB824F06FFBF9F7F1FD012812D94FF0FC
:10823000FF33C7F8703424F065FB90F8C432DFEDEB
:10824000150AB02202FB030090ED300A28461BF00D
:10825000E7F9D1E704F58058D8F868042BF0B8FDA9
:1082600008F58D63C7F87004D3ED007A9FED0A0A14
:10827000DFED080AF8EEE77A27EE800AE6E701AAC2
:10828000002140461AF032FE0028C1D00199002298
:10829000BBE700BF00007A440AD7233C7FB501F159
:1082A000080304460E460FCB6D4685E80F0004F523
:1082B000AE41083128461AF015FF29462046FFF73F
:1082C000D1FC20463146FFF7FFFE04F5A044002311
:1082D000C4F8E83604B070BD37B504460D4689F0E1
:1082E000D9FD2062D5ED027AF5EEC07AF1EE10FAF2
:1082F00015DD9FED127A67EE877AFCEEE77AC4ED22
:10830000077A5CF0FDFAE2694FF47A73B2FBF3F39B
:108310000B4A062103B0BDE8304055F095BC67F02C
:108320003FFB0023009395F90D2095F90E3095F948
:108330000C1067F0D1FAE061E3E700BF00007A4477
:108340006C2B0D082DE9F0432DED028B85B0044612
:1083500015F00CF914F0F2F904F5805304F5A0457A
:1083600093F860370BB9002877D0D5F87034013313
:1083700073D1D5F89434002B4BD089F08BFDD5F810
:108380009434C01AB0F5FA6F67D394F8E423DFEDA4
:108390005F7A9FED5F8A4FF0B00808FB024292EDD2
:1083A000780A20EE270A2BF02BFD05F58F69D9ED11
:1083B000007A30EE670A2BF023FDDFED567A20EECF
:1083C000080A04F54E5720EE270A2BF0C1FCFDEEFB
:1083D000C07A083717EE906AC5F87064D9ED007A54
:1083E00067EE887A17EE900AF8F786F8CDE9020171
:1083F00094F8E43308FB0343D3F8DC01F8F77CF886
:10840000454ACDE9000133460621384655F01CFCAB
:1084100023E004F59070F9F7F9FC02281DD994F8CF
:10842000E433B02202FB034393ED777AF1EE047A52
:10843000B4EEE77AF1EE10FA0FDD384B1B68D86A1C
:108440000368DB699847012803D089F023FDC5F84C
:108450009404D5F89434002B8FD104F54053D5F80B
:108460007014D3F8A4054A1C036846D01B6B9847C8
:108470002B4810F011FD20B104F5AA40203031F056
:1084800083FF2046FFF7DCF8D5F8803483420646A8
:1084900036DA07EE906A9FED237AF8EEE77A04F574
:1084A0004E5467EE877A083417EE900AF8F724F8EE
:1084B0001D4ACDE900012046062155F0C5FB0124E7
:1084C0004FF0FF33C5F8703485F8B04405F5E1632B
:1084D0000FCB05F5DF6605F5E36786E80F0087E853
:1084E0000F00124867F0D8FB002385F8B33420460C
:1084F00005B0BDEC028BBDE8F0835B6B9847B7E736
:10850000074810F0A9FC0028C3D1F1E735FA8E3CEA
:10851000E02E65420000C8427C2B0D086C2B002029
:10852000702B00200AD7233CA02B0D08B84B00204D
:108530002DE9F04100F5AD4700F5AE457837183527
:108540000446294638461AF08DFD04F5A04604F588
:10855000405830B3D6F870144B1C22D0D8F8A4057C
:1085600003681B6B9847D6F8E836012B47D0D6F83E
:10857000E836022B06D12046FEF7CAFFD6F81C3794
:10858000984243DD2046FEF7C3FFD6F81C37C01AD9
:108590000028B8BF4042B0F5FA7FCCBF00200120D0
:1085A00035E004F5AE40294608301AF093FFDFEDC0
:1085B000197AB4EEE70AF1EE10FA16D538462946D4
:1085C0001AF058FE9FED147ADFED140AF6EE007AE9
:1085D000E0EE077A28469FED120AFDEEE77AF8EE04
:1085E000E77A27EE800A1BF01BF8D8F8A4059FED68
:1085F0000D0A03682A469B6A39469847B3E7204626
:10860000FEF786FFD6F81C379842B0DB0120BDE8A4
:10861000F08100BF00004843A00CB3450000964322
:108620000AD7233C0000000073B5394CD1ED026A33
:10863000D4F80C379FED377A07EE903AF8EEE77AE8
:108640000546D7EE876A0E46F5EEC06AF1EE10FADF
:1086500008DD5CF055F9304A062155F0F5FA0120A5
:1086600002B070BDD1ED037AF5EEC07A04F59264E4
:10867000F1EE10FA94ED006A12DDF4EEC67AF1EE36
:1086800010FA0DD55CF03CF905462068F7F734FF89
:10869000224ACDE900010621284655F0D5FADEE749
:1086A000DFED1F7A337CB4EEE76AF1EE10FA54BFC7
:1086B000B0EE677AB0EE467A0BB90020D0E7B5EE9F
:1086C000C06AF1EE10FA0CDC86EE876A03EB8303D6
:1086D00007EE903AF8EEE77AF4EEC67AF1EE10FA89
:1086E000EBD595F82440002CE7D189F0D3FBAB6A99
:1086F000C01A337C4FF47A7253439842DDD9012378
:1087000085F8243089F0C6FBA8622046A8E700BFA0
:10871000707B00200AD7233CBC2B0D08CD2B0D0805
:108720000AD723BC38B5054678F0D6FF77F0E4FDCC
:10873000044640B989F0AEFB2B6AC01AEB69984237
:1087400084BFEC610124204638BD000038B50446E2
:108750000D4689F09FFB04F5A0439FED077AC3F80F
:10876000EC06D5ED027A67EE877AFDEEE77A17EE32
:10877000902AC3F8E82638BD00007A4410B50446B4
:1087800089F088FB04F5A043D3F8EC26801AD3F8CF
:10879000E82690424FF0000084BFC3F8E8060120AD
:1087A00010BD000000F5A04303F59361D3F8E8265F
:1087B00091ED007A22EAE27207EE902AF8EEE77A6B
:1087C0000020B4EEE77AF1EE10FA44BFC3F8E806F1
:1087D0000120704710B500F5005300F5A040B3F933
:1087E0007A31002BB4BF4FF0FF33012380F8D0362D
:1087F00000F5E36400F5E1600FC884E80F0010BDE8
:1088000038B504462DED028BF0EE408AB0EE608A5A
:1088100009B301295ED0B5EEC08AF1EE10FA69DD28
:10882000DFED357AB4EEE78AF1EE10FA62D8FCEEAD
:10883000C87A04F54E5017EE903A304A06210830B7
:1088400055F002FAFDEEC87A04F5005417EE903A9E
:1088500084F847313CE0F8EE000A2BF0D3F940B140
:1088600004F580444FF0FF33C4F8F83EBDEC028BB2
:1088700038BD04F50053B3F9502107EE902AF8EE05
:10888000E77AF4EEE87AF1EE10FAC4D8B3F952318F
:1088900007EE903AF8EEE77AF4EEE87AF1EE10FAA5
:1088A000B9DBDFED157A68EEA77A04F58043FDEEBB
:1088B000E77A04F54E5017EE902AFCEEE87AC3F8FA
:1088C000F82E062117EE903A0D4A083055F0BCF903
:1088D0000120CBE7FCEEC07A00F54E5017EE903A3F
:1088E000084A0621083004F5005455F0ADF9C4EDEE
:1088F000578AEDE70020B9E70000C842132C0D08A5
:10890000EC2B0D08002C0D08D1F80D3000EE903A3C
:10891000D1F80930097A00EE103AFFF771BF000074
:1089200070B58B88012B04460D4611D100F5907669
:108930003046F9F76BFA02280AD994F8E413B02309
:1089400003FB01612046AC31BDE87040FFF7AABAD5
:1089500014F00CFE05F10801BDE8704014F01EBAD9
:10896000F0B500F5A047002489B0054687F8B94462
:1089700008460E462FF0D6F8A0B3012387F8B0348E
:1089800005F54053D3F8A4050368DB6B984787F8D7
:10899000B744C7F8D44603A81AF06CFAB7F85C15C8
:1089A0004FF6FF73994208BF2146013105F5AA40F1
:1089B00001AA89B2203031F069F8F0B1BDF8063073
:1089C000A3F115025342534187F8B13450B105F574
:1089D000AF40BDF80610503008F0ECFC10B1002399
:1089E00087F8B13473885E2B4ED8522B07D8103BD2
:1089F0009AB20F2A22D90024D5E00346E4E7533B7C
:108A00000B2BF8D801A252F823F000BFA18B01086C
:108A1000AD8B0108BD8B0108F7890108F7890108B2
:108A2000F7890108F7890108F7890108F789010822
:108A3000F7890108098C0108BD8B01080F2BDAD8D2
:108A400001A252F823F000BF258B01085F8B0108BB
:108A5000698B0108738B0108878B0108318B010832
:108A6000F78A0108F7890108F7890108F7890108E1
:108A7000F7890108F7890108F7890108F7890108D2
:108A8000978B01087D8B0108BD2B1AD8BB2B47D8CB
:108A9000B22B00F0A7800DD8702B00F09E80722BB7
:108AA000A9D1D6ED027AFDEEE77A17EE903AC7F833
:108AB000E83635E0B32B9ED131462846FFF730FF2C
:108AC0002EE0D42B00F0938040F6B832934200F0B1
:108AD0009680D22B8FD1B388012B21D803F00103CC
:108AE00087F8B23405F54E50B3884B4A062108305A
:108AF00055F0AAF814E0002305F5AF4487F8E934EF
:108B000050347188204607F0F9FE314628B12046DE
:108B100009B0BDE8F04008F0F3B82846FFF732FA94
:108B2000012440E006F108012846FFF79BF8F7E72B
:108B300005F5AF4450341521204608F03BFC48B100
:108B4000002387F8E9343146204609B0BDE8F040FB
:108B500007F0DABF31462846FFF760FAE0E7314612
:108B60002846FFF7BDFADBE731462846FFF7D2FA81
:108B7000D6E731462846FFF707FBD1E731462846BE
:108B8000FFF78CFBCCE705F5984129224C312846AC
:108B90000EF0E4F8C4E731462846FFF719FBBFE7BB
:108BA000012487F8B744204609B0F0BD002305F53D
:108BB000AF4087F8E93431465030A9E705F5AF47B3
:108BC0005037384608F0DAFB3146044618B12846DB
:108BD000FFF760FAE7E73846B7E731462846FFF780
:108BE000B5FD9DE731462846FFF78EFE98E7B18830
:108BF000003918BF0121284600F026FF90E7317A9E
:108C0000064807F073FA8BE705F5984031462030A7
:108C1000FFF762FB84E700BF242C0D08408300208F
:108C200000F5804200F59843D2F8C02E20339A42D6
:108C300001D1FFF795BE01207047000010B500F587
:108C4000804200F59843D2F8C02E20339A42044661
:108C50000ED100F5984108224C310EF07FF804F552
:108C60004E50044ABDE810400621083054F0ECBFD5
:108C700010BD00BF342C0D082DE9F04F2DED048BF5
:108C800000F5A04808F5056393ED008ADFEDD77A7B
:108C9000B0EEC87AB4EEE77AF1EE10FA48BF00F50C
:108CA0000053DFEDD37A42BFB3F97A3108EE103AC0
:108CB000B8EEC88A00F58045B4EEE78AF1EE10FA06
:108CC00094BF4FF0FF37012788F8D076D5F8E83EFB
:108CD0009BB004460E46F0EEC88A052B16D8DFE896
:108CE00013F006002C0069008800C500600100F543
:108CF00040543A46D4F8A4050368B0EE680ADB6A2B
:108D000008319847BB4806F00BF908B9002049E143
:108D1000B94CD4F8F436B4F990185B68642201FBBE
:108D20000231A4F5A040FFF7D9F8A4F5A04005F062
:108D3000C1FC0123C5F8E83EE8E700F540533A4698
:108D4000D3F8A4050368B0EE680ADB6A08319847D7
:108D5000D8F8CC36002BB8BF5B42012BD6DD98F893
:108D6000D1361BB998F8D236002BCFD004F5AE53CC
:108D7000D3ED040A93ED050AF1EE600AB1EE400A64
:108D8000ADF022FCDFED9D7A20EE270A05F6EC63BC
:108D900083ED000A10EE100AF7F7AEFB04F54E540F
:108DA0000834CDE90001964A0621204654F04CFFD4
:108DB0000223BFE700F5AE4901F1080A09F10809ED
:108DC000494650461AF086FB30EE680AF1EE047A06
:108DD000B0EEC00AB4EEE70AF1EE10FA00F3E78055
:108DE000D8F8CC360133022B40F2EB800323C5F8D0
:108DF000E83E04F5405306F10808D3F8A4050368DB
:108E00003A46DB6AB0EE480A41469847DFED7D6A94
:108E10009FED7D7A05F6EC63D3ED007A012F18BF44
:108E2000B0EE667A04F5A35377EE877A93ED050AE0
:108E30009FED767AA7EEC70A2AF0E2FFDFED747A9B
:108E4000B0EEC00AB4EEE70AF1EE10FA7FF55EAFBD
:108E500004F54E50062108306E4A54F0F5FE042306
:108E6000C5F8E83E41462046FEF7FCFE06F108053F
:108E700095E80F000AAF0DF1380887E80F0088E881
:108E80000F0004F5804303F6EC6A9FED639A9AEDB8
:108E9000000ADFED620A0393384630EE090A1AF041
:108EA000BFFBDFED5E0A9AED000A9FED5D8A40464A
:108EB0001AF0B6FB04F540534246D3F8A405036804
:108EC00039469B6AB0EE480A984795E80F0004F5CA
:108ED000AF490DF1480B09F150098BE80F00DAEDAD
:108EE000009A484607F030FD79EE899A04F5AE48BD
:108EF000F0EE400A5846B0EE690A08F108081AF088
:108F00008FFB5A46394640461AF050FA834695E898
:108F10000F009AED000A16AF87E80F00F0EE680A1E
:108F200030EE090A38461AF07BFB394640462A469D
:108F30001AF006FA04F5935007A90830F0EE408ABB
:108F40008DED078A8DED088A8DED098A14F00CF9F4
:108F5000002867D0294640461AF0C8F905A907A895
:108F6000CDED060A8DED050A2DF044FFDFED237AE5
:108F700020EE270A2AF0D8FEB0EEC00ABBF1000F9F
:108F80003FF4C4AEF3EE0E7AB4EEE70AF1EE10FA57
:108F900023D5039A0523C2F8E83E3146484607F038
:108FA000B3FD01201BB0BDEC048BBDE8F08F49463A
:108FB00050461AF08FFAB4EEE80AF1EE10FA7FF597
:108FC0000FAF04F540543A46D4F8A4050368B0EE58
:108FD000680ADB6A5146984798E6F6EE007AF4EEA6
:108FE000E78AF1EE10FAD4DC90E600BF000000340E
:108FF000000000B4702B0020707B0020E02E654242
:109000005C2C0D080000B4420000874335FA8E3C0A
:10901000C2B8B23D7E2C0D080000344300007A44F3
:1090200000000000BBF1000F3FF470AEB1E700BFDD
:109030002DE9F041074600F5AF408EB0503088462C
:1090400008F0DCF9044650BB09AE07F5A0453046F0
:1090500019F010FFB5F85C354FF6FF72934208BF68
:109060000023013307F5AA4007AA99B2203030F057
:109070000DFDC0B1B8F1000F01D0C5F8CC4696E89F
:109080000F0001AC84E80F00D5F82437009305F5F4
:10909000E36595E80E00054803F0CCF90446204648
:1090A0000EB0BDE8F0810124F9E700BFD8770020B9
:1090B00070B5064606F5A045002106F001F8D5F882
:1090C000D4467CB9304605F02BFF10B90024204669
:1090D00070BDD5F8CC36012BF8DD88F0DBFEC5F885
:1090E000D406F4E7D5F8E81661B188F0D3FED5F8D8
:1090F000D436C01AD5F8E0369842E7D90023C5F82F
:10910000E83601213046FFF793FF04460028DDD002
:1091100006F54E50044A0621083054F095FD002310
:1091200085F8B934D3E700BFA02C0D0870B50A4606
:109130008B88190A137E0546DB0748BF01EB8101C6
:1091400005F5A04448BF4900002605F0B9FF84F8A2
:10915000B964284605F0E4FE10B90024204670BD2D
:10916000D4F8E81651B1D4F8CC36D4F8C8269342D6
:10917000F3DD012BF1DDC4F8E86601212846FFF795
:1091800057FF04460028E8D005F54E50024A062154
:10919000083054F059FDE1E7B82C0D0838B5054604
:1091A00005F5A044898805F08BFFD4F8E83683BB29
:1091B000D4F8CC36002BB8BF5B42012B02DC002474
:1091C000204638BD94F8D12694F8D23672B9002BD7
:1091D000F5D005F54E50D4F80C276423062192FBF8
:1091E000F3F308300C4A54F02FFD01E0002BF0D1CE
:1091F0000121C4F8E8162846FFF71AFF04460028A4
:10920000DDD005F54E50054A0621083054F01CFD0E
:10921000D6E70021EFE700BFD02C0D08EE2C0D089B
:1092200010B504460B4808F0D3FE48B10A4BDFEDF9
:109230000B7AD3F80C3893ED090A20EE270A10BDFB
:1092400004F50054B4F9A83100EE103AB8EEC00AA3
:10925000F5E700BF40830020707B00200AD7233C45
:1092600038B52DED028B00F5005300F5A045B3F99C
:10927000AC110029ACBF01234FF0FF330029B8BF68
:10928000494285F8D036044689B205F019FF05F544
:109290009365204695ED008AFFF7C2FFB5EEC00A40
:1092A000F1EE10FAD8BF9FED0E0ABCEEC00AB8EE80
:1092B000400AB4EEC08AF1EE10FA0AD804F54E5016
:1092C0000830084A062154F0BFFC0120BDEC028B97
:1092D00038BD204605F024FE0028EFD1F6E700BF98
:1092E00000000000082D0D082DE9F04700F5A0470B
:1092F0002DED028B4FF0FF33C7F8703407F5E363B1
:109300008C4605460FCBBCF804609CF8049088B0EE
:1093100004AC360A84E80F0020D005F5AD4808F10A
:109320007808214640461AF0D5F821464046B0EE6E
:10933000408A19F09FFFDFED587AB4EEE78AF1EE2C
:1093400010FA0BDBF3B200EE903ADFED547AF8EE50
:10935000600A20EE270A20461AF062F905F5405A05
:1093600097F8B424DAF8A4059FED4D0A036805F5D3
:10937000AE489B6A08F1080832B305F5AD412246B4
:109380007831984705F50053B3F9AA31002B1EDD5B
:1093900007EE903A07F59362F8EEE77A92ED007ADD
:1093A000B4EEE77AF1EE10FA11DD05F5AD41224693
:1093B0007831404619F0FAFFF8B90026304608B077
:1093C000BDEC028BBDE8F08722464146D9E7B9F1F2
:1093D000000F1DD1002E3DD1DAF8A4653368284670
:1093E000D3F82090FFF71CFF07F28C43D3ED000A5F
:1093F0003046C847B0EE408A0EE0002EDDD107F5BA
:10940000DF6407F5E16797E80F0084E80F00D5E710
:1094100007EE909AB8EE678A214640461AF05AF84D
:10942000B4EEC08AF1EE10FA17DBB7F85C3503939F
:10943000214640461AF04EF8BCEEC00A05F54E50E3
:10944000039B184A8DED000A0621083054F0FCFBFE
:109450000126B3E79FED128ADEE705F5AD4122460E
:109460007831404619F0A2FF06460028A5D0B7F88B
:109470005C350393214640461AF02CF8BCEEC00A36
:1094800005F54E50039B084A8DED000A0621083071
:1094900054F0DAFB92E700BF00000034E02E654292
:1094A00000000000202D0D083E2D0D082DE9F0478D
:1094B0004B881F2B8AB004460D466BD80F2B41D822
:1094C00004F54E50BF4A0421083054F0BDFB9BE028
:1094D000A3F1BC02182AF3D801A151F822F000BF71
:1094E0000996010809960108C1940108C194010870
:1094F000C1940108C1940108C194010809960108AA
:10950000C194010809960108C1940108C194010899
:10951000C194010809960108C1940108C194010889
:10952000C1940108099601080996010809960108E5
:10953000C1940108C194010809960108C194010869
:1095400009960108A3F110020F2AB9D801A151F818
:1095500022F000BF459601082B97010835970108B6
:109560004197010857970108519601081B96010879
:10957000C1940108C1940108C1940108C194010873
:10958000C1940108C1940108C194010861970108C0
:109590004B9701085E2B21D8522B91D9A3F153028E
:1095A0000B2A8DD801A151F822F000BF6B9701085A
:1095B0007D97010887970108C1940108C1940108AB
:1095C000C1940108C1940108C1940108C194010823
:1095D000C1940108B197010887970108722B00F028
:1095E000E28007D8702B7FF46BAF0AB0BDE8F0477C
:1095F000FFF7C4B8D42B09D8BB2B3FF669AFA3F152
:10960000B202012A3FF65CAF012052E0DF2BFBD013
:1096100040F6B8329342F7D052E700F5AF465036E5
:109620001621304607F06AF930B1294630460AB0B3
:10963000BDE8F04707F056BC20460AB0BDE8F04749
:10964000FEF780BE29460AB0BDE8F047FFF74CBEE2
:1096500000F5AF4550351521284607F0ABFE28B17F
:1096600028460AB0BDE8F0470BF0A2B904F5A045C2
:1096700004F5AC46D5F8FC3404F5AD4704F5AE4826
:1096800004F5AE49072B06F1380607F1780708F113
:10969000180809F108090FD104F5A9447834019498
:1096A000D5F88034009342464B463946304685F023
:1096B00075F80AB0BDE8F0870DF127018DF8270095
:1096C0004148FEF761FA05F2BC43D3ED007AD5F8C4
:1096D000A0A405F59263D3ED000A05F29C4330EE99
:1096E000670A93ED001A8DED070A04F5AF400830C4
:1096F000CDED060A8DED051A76F0F4FD05462046FF
:1097000000F074FF9DF827309DED051ADDED060A87
:109710009DED070ACDE90203CDE900A54B4642467F
:109720003946304684F090FFC3E7A98805F0C8FCAD
:109730000020BEE729460AB0BDE8F047FFF7F6BCB7
:109740000AB0BDE8F047FFF7B3BC29460AB0BDE850
:10975000F047FFF723BD0AB0BDE8F047FFF780BD33
:109760000AB0BDE8F047FEF7E3BE04F5984029468D
:1097700020300AB0BDE8F047FEF756BF04F5AF4011
:109780002946503053E704F5AF465036304607F0CF
:10979000F5FD08B9304664E729462046FFF76CFA24
:1097A0000028F7D185E70AB0BDE8F047FEF7FABF19
:1097B00004F59840294620300AB0BDE8F047FEF78E
:1097C000B1BF00BF5C2D0D08702B002070B500F5F7
:1097D000804200F59843D2F8C02E20339A420546C5
:1097E0000E4602D00024204670BDFFF75FFE0446FF
:1097F0000028F7D005F54E503188083058F064FB4A
:10980000F1E7000021F04003152B04D0A1F15E0325
:1098100058425841704701207047000000F58042CF
:1098200000F59843D2F8C02E20339A4207D100F5B4
:10983000A040B0F85E355B1A58425841704700208E
:1098400070470000192963D8DFE801F00D111519E0
:109850001D2125282C62303437563A3A3D40434783
:109860004A4E62525A5E00F599404030704700F50A
:1098700096401430704700F596403030704700F540
:1098800096404C30704700F596406830704700F5C0
:1098900097402430704700F59740E6E700F5974081
:1098A0005C30704700F598400430704700F59840F0
:1098B0002030704700F59840E3E700F59840E4E772
:1098C00000F59940F0E700F59940E2E700F599408E
:1098D000E6E700F599407830704700F59A40C8E710
:1098E00000F59A403430704700F59A405030704788
:1098F00000F59A407030704700F59B402830704763
:1099000000F59B406430704700F59B400C30704779
:109910000020704700290DDB074890F8EC2BCBB2F4
:109920009A4207D3D0F8E83B0122595CA0F50050D9
:109930000DF0ECBA704700BF704B00202DE9F341E9
:1099400000F5005300F54E5593F8B83B03F00106BF
:1099500003F0020803F004075B07044605F108055D
:1099600035D01F4A0621284654F06EF926B104F579
:109970003B503C3078F0BEFCB8F1000F04D004F549
:109980004150143078F032FA27B104F546502C30AB
:1099900079F0DAF804F5A044012384F8213B114A58
:1099A000114B1249B8F1000F08BF1A46002F08BF2B
:1099B0001946CDE900210E4A0621002E18BF134694
:1099C00028460C4A54F040F902B0BDE8F0810A4A3A
:1099D0000621284602B0BDE8F04154F035B900BF79
:1099E000892D0D087E2D0D08BC150E08852D0D083E
:1099F000782D0D089A2D0D08AC2D0D0810B50446D4
:109A000000F53B503C3078F0A1FC04F54150143097
:109A100078F018FA04F546502C3079F0CFF804F5B8
:109A2000A04393F8212B5AB1002283F8212B04F58F
:109A30004E50044ABDE810400621083054F004B9E5
:109A400010BD00BFCC2D0D0809B1FFF777BFFFF7A0
:109A5000D5BF000000F580430A4AD3F8C01E9142EA
:109A60000DD093F8CD3E43B900F598422032914293
:109A700003D100F5A04090F8B23418467047002397
:109A8000FBE700BF3078002010B5044688F002FAEA
:109A9000054BD3F8E03EC01A642804D82046BDE840
:109AA00010405CF049B910BD706B002010B500F596
:109AB0002E54D4ED0A7AF5EEC07AF1EE10FA8AB09F
:109AC0004FF0000304F1280445D907930893099344
:109AD00006AB019300F5935007AB009303AA05ABC7
:109AE00004A9083013F0E0F930B3DDED080A9DED6C
:109AF000070AACF0CDFBDDED090AACF0C9FBD4EDF3
:109B0000007A9DED047A77EEA76AB4EEE70AF1EEEB
:109B100010FAF4EEC76AACBF01200020F1EE10FA93
:109B20000CD802309DED037AF4EEC77AF1EE10FA0C
:109B30000CD8003818BF01200AB010BDF4EEC77A67
:109B4000F1EE10FA9CBF0130C0B2EBE7012894BFE0
:109B500000200120F0E70020EEE7000038B5124BAE
:109B60001A7A0446FAB901251D7251F0A9FF2A4656
:109B700004F5AF451121503551F0FEFE284607F09F
:109B800081FC80B1284607F039FC062238B104F583
:109B90009A413431BDE8384004480DF0DFB804F58F
:109BA00099417831F6E738BDA8860020702B002057
:109BB00010B5074B1A7A4AB100241C7251F080FF8D
:109BC00022461121BDE8104051F0D6BE10BD00BFA5
:109BD000A88600202DE9FF41054605F59358684603
:109BE00008F1080819F046F96946404613F0B0FA42
:109BF0000646E8B1374876F075FB50B105F52E53AF
:109C0000D3ED0A7AF5EEC07AF1EE10FA94BF012690
:109C1000002605F5AF40503007F034FC2E4C2F4F96
:109C200000B146B1002328462380FB73FFF7C0FF35
:109C300004B0BDE8F0812846FFF738FFA0B3637891
:109C40007BBB23780133DBB2082B237002D1404663
:109C500013F096F92378092B02D1404613F088F9C6
:109C60002378092B1DD94FF48573238051F028FFE9
:109C70000222102151F080FE88F00CF96368C01AAE
:109C800047F23053984209D905F54E50144A022143
:109C9000083053F0D9FF88F0FDF860602846FFF7E0
:109CA0005DFF6378FB73C3E72378002BF9D0013B9A
:109CB0006278DBB22370002AF3D0002BF1D16670FA
:109CC00051F0FEFE3246102151F056FE2846FFF7B5
:109CD0006FFFE6E7F8820020A88600205587002065
:109CE000E02D0D0810B500F5A044D4F8FC34042B89
:109CF00001D1012010BD00F5AF40503008F04EF901
:109D00000028F6D194F82805F4E7000073B500F5B3
:109D100080450192A5F8D81E044688F0BBF8C5F826
:109D2000DC0ED5F8C00E03685B68984785F8D60E40
:109D3000D5F8C00E03685B689847019A182818D8B0
:109D4000DFE800F00D170D0D0D0D0D0D0D1752175D
:109D50005917595917414141171717415900334BAA
:109D600093F8223B03B304F59741243120460CF0CD
:109D7000F5FFD5F8C00E95F8D66E03685B68984776
:109D800004F54E54864204F1080447D0D5F8C00EBD
:109D900003689B689847264A03460421204602B080
:109DA000BDE8704053F050BF04F5005393F9BC3147
:109DB000022BD8D0042B0BBF04F5974104F5964134
:109DC00040311431D2E704F5A043D3F8943AD902D4
:109DD00003D504F598414C31C8E704F59A419B0638
:109DE0004CBF50313431C1E720460192FFF77AFF72
:109DF000019A0028BDD104F50056019296F9BC31B4
:109E0000002BB6D0D5F8C00E03685B68984785F87C
:109E1000D60E96F9BC31019A022BCAE7054A0421F5
:109E2000204602B0BDE8704053F00EBF707B0020AA
:109E3000F02D0D08122E0D08F0B5044604F58046ED
:109E400085B00F4615465BF0FDFED6F8C00EA6F8AD
:109E5000D87E03685B68984718281ED8DFE800F0B2
:109E60000D0D0D0D0D0D0D0D0D1D64810D0D707081
:109E70001D5252521D1D1D520D003D4AD2F8FC14B8
:109E8000012921D104F5005393F8BD31023B012B88
:109E90001AD904F5405383F88413D6F8C00E354A16
:109EA000354B052D18BF13460268039392689047FF
:109EB00004F54E5408340090039B304A0421204698
:109EC00053F0C2FE05B0F0BD92F8223B3BB104F561
:109ED00097412A46243120460CF040FFDDE704F587
:109EE000005393F9BD31032B03D1204605F050F9FF
:109EF000D3E7022BEBD0042B2ED104F598412A4650
:109F00002031E8E704F5A043D3F8943ADA0223D4E9
:109F10009B0604D504F59A412A465031DBE704F547
:109F20009A412A463431D6E72046FFF7DBFE002867
:109F3000B3D104F5AF40503007F0CEFA0028EED18F
:109F400004F5005393F9BD31032BCED0022BBED0C4
:109F5000042BD2D0012BA0D104F598412A464C31D4
:109F6000B9E704F5005393F9BD31042B95D1C4E74B
:109F7000707B0020282E0D08A4120D08302E0D082D
:109F800070B500F54E5504460835124A042128469E
:109F900004F5804653F058FE0023A6F8D83E04F599
:109FA000005393F80431032B12D196F8D61E3022B9
:109FB00020460CF0ABFFD6F8C00E03689B689847AC
:109FC000054A034606212846BDE8704053F03CBED2
:109FD00070BD00BF442E0D085B2E0D0800F54053E8
:109FE00010B500220529044600F54E5083F884235D
:109FF00000F108000CBF054A054A042104F580441D
:10A0000053F022FE0023A4F8D83E10BD742E0D0894
:10A01000852E0D08013A38B50446052A3ED8DFE8FA
:10A0200002F04B1B8711900300F5A04393F8E4382E
:10A0300043B100F59B4104220C314448BDE838404F
:10A040000CF08CBE04F5A04393F8E43823B104F57A
:10A050009A4104223431F0E704F58043D3F8C02E4E
:10A0600004F59A4334339A4226D004F59B430C33CB
:10A070009A4221D004F5A043D3F8FC34042B1BD022
:10A08000334D95F8F13EBBB1324905F5A95030F09A
:10A09000CFF820B1304B012283F8282538BD2D4957
:10A0A00005F5A95030F0C4FB30B104F59841042205
:10A0B0002031A5F58040C1E704F58043D3F8C02ED8
:10A0C00004F59A4334339A42E8D004F59B430C33A9
:10A0D0009A42E3D004F5A04304F5AF405030D3F8E2
:10A0E000FC5407F05BFF0028D8D1042DD6D004F52E
:10A0F000005393F98731022B0DD004F59841204687
:10A1000004224C310CF02AFE04F505500730BDE85E
:10A11000384048F035B90E4890F8F13E002BECD0AD
:10A120000C4900F5A95030F083F80028B2D1E4E7DB
:10A1300000F5AF40BDE83840012214210830F7F7A0
:10A1400019BDBDE8384005F023B800BF702B0020D2
:10A15000706B002078820020707B002070B52DEDA0
:10A16000068B044687F08AFE414BB4F8BE101A886D
:10A17000404E8A420546404A06D01980002330608E
:10A180001370BDEC068B70BD33683C49C31A8B421B
:10A1900065D9012313705BF055FE5BF00DFD356052
:10A1A0005BF050FE5BF008FD5BF02EFD0428E8D963
:10A1B0005BF048FD204600210BF00CF82046002102
:10A1C000B0EE40AA0BF010F820460121F0EE409AC4
:10A1D0000BF0D0F900212046B0EE408A0BF00EF8CB
:10A1E00004F5AF400830F0EE408A76F085F89FED38
:10A1F000249A0028B0EE4A0A4FF0040008BFB0EEDF
:10A20000498A5DF031F9B0EE690A13205DF02CF94E
:10A21000B0EE680A15205DF027F9B0EE680A1A2042
:10A220005DF022F9B0EE480A46205DF01DF90121EB
:10A2300008465DF025FCB0EE490A02205DF014F9F5
:10A24000B0EE490A03205DF00FF920460BF0C0FB89
:10A25000BDEC068B2046BDE870400CF00BBB1278BD
:10A26000002A8ED044F6206293428AD993E700BF39
:10A27000B4860020B8860020B6860020400D03007A
:10A280000000000000F5804200F59843D2F8C02E8F
:10A2900020339A4204D100F5A04090F82805E8B197
:10A2A0000F4B93F8040103F54053A0F12702012A54
:10A2B00093F8303B0FD92C2809D00A2809D0A0F1F7
:10A2C0003102504250410A2B18BF00207047012034
:10A2D000F9E7012070470A3B58425841704700BFD8
:10A2E000704B002008B500F5005393F8482042B1A8
:10A2F00093F884302BB1FFF7C5FF80F00100C0B2A6
:10A3000008BD0120FCE700002DE9F04700F50055ED
:10A31000B04E95F884A0044600F5AF408AB00830EE
:10A3200075F0E0FFD6F8FC34042B814642D10121C0
:10A3300004F5015808F10808404666F013F896F84D
:10A34000303B0A2B074605D1B9F1000F54D1002349
:10A3500086F8303B95F84830002B58D195F94E30AF
:10A360009D4D012B03D0063BDBB2012B11D895F894
:10A3700004310A2B0DD104F58047D7F8C00E0368CD
:10A380001B6A984728B1D7F8C41E2B2220460CF030
:10A39000E5FC96F8303B0A2B04BF372386F8303BA8
:10A3A00095F804310A2B02D1372385F804310AB01D
:10A3B000BDE8F0870028BAD004F58043B6F85E7592
:10A3C000D3F8C00E03685B6898471428AFD004F533
:10A3D000AF40503007F030FC0028A8D13946A6F530
:10A3E000A040FFF70FFA01460028A1D096F82415E7
:10A3F0004B1E594259419BE740EA0A03DBB2002B4E
:10A40000A8D1764800F0F2F80028A0D0A2E7B9F170
:10A41000000FCCD004F5AC40383084F08BF8002825
:10A42000C5D12046FFF72EFF0028C0D1002F00F035
:10A43000BF806B493A46404665F06CFB95F94E90FB
:10A44000B9F1010F07D040F38780A9F10603DBB211
:10A45000012B00F281805FFA89F9B9F1010F4ED129
:10A4600004F5804204F59843D2F8C02E20339A4276
:10A4700009D104F5A04393F8283523B195F8873125
:10A48000013B012B93D904F598410A224C31204617
:10A4900006AE0CF063FC304618F0ECFC95F9612038
:10A4A00092BBB9F1010F2FD004F5A049B5F9623084
:10A4B000D9F8F416DFED4B5AD1ED017A002BF8EE06
:10A4C000E77A52DD07EE103AF8EEC76AE6EEA57AB3
:10A4D0003046FDEEE77A17EE901A18F0D1FC002313
:10A4E0004046CDE9043365F0D9FF04A966F01AFDB2
:10A4F000002857D0049B0893059B099317E004F5A7
:10A5000099410A220431C2E72046FCF787FE07EE94
:10A51000900AE84604F5AE42083221464046B8EEBD
:10A52000E70AFDF725FD98E80F0086E80F0095F98A
:10A530004E30012B10D031462046FCF7C5FF314686
:10A540002046FDF7FBFB95F94E30072B04D104F5AF
:10A550004054012384F8823351F0B2FA3A4609217B
:10A560000AB0BDE8F04751F007BAD5ED146A95ED91
:10A57000175A95ED157A35EE076A36EEC57AB4EEC0
:10A58000C67AF1EE10FA89BF37EE067A95ED7A7A3F
:10A5900027EE257AF6EE006A94BFE7EE257AE7EE1D
:10A5A000267A95E7D9F8F4369A680892DB68A4E72A
:10A5B000BAF1000F3FF4FBAE95F88430002B7FF426
:10A5C000F6AE04F54E50084A0521083053F03CFB26
:10A5D000C2E700BF707B0020704B0020702B002072
:10A5E000A02E0D080000C842A92E0D0810B5044683
:10A5F00000F5AF40083075F07FFE98B104F5AF402C
:10A60000503008F0C1F960B904F5AA4494ED007A1D
:10A61000DFED087AB4EEE77AF1EE10FAACBF012074
:10A62000002010BD04F5AA4494ED007ADFED027A13
:10A63000F0E700BFCDCCCC3D6666663F70B500F557
:10A64000804600F59B43D6F8C02E28339A42044634
:10A6500000F5A04502D195F8F804D8B904F5AF404B
:10A66000B5F85E15503006F049F9A0B9D6F8C03EED
:10A6700004F598442034A3420CD195F8F8344BB13A
:10A68000D5F8FC34032B05D1B5F85E05A0F116030F
:10A690005842584170BD0020FCE700002DE9F74FFB
:10A6A00000F5804200F59843D2F8C02E20339A423C
:10A6B000044600F5A04504D100F5005B9BF960312C
:10A6C0003BB90023C5F8EC3485F8E93403B0BDE8A4
:10A6D000F08F87F0DFFBD5F8A464804636B1861B87
:10A6E00040F6C3139E4294BF002601262046FFF782
:10A6F0007DFF019028B1002785F8E8744FF0000A2B
:10A7000046E004F5AF40083075F0ECFD81460028C6
:10A71000F1D004F5AC4A0AF1380A504683F00AFF3A
:10A720000746002845D095F8E8A4BAF1000F3BD1C0
:10A7300056B304F5805041F27071D0F86024002ABD
:10A74000B8BF52428A4206DCD0F86424002AB8BF5F
:10A7500052428A422BDD04F5AA4104F5AE40643131
:10A76000083018F0B7FEDFED487AC5F8EC84B4EE97
:10A77000E70AF1EE10FA4FF000024CBF4FF0010A69
:10A780004FF0000AC5F8F024012285F8E824374686
:10A7900004F59070F7F73AFB022832D9002F44D124
:10A7A0000023C5F8EC3491E7019EB246ECE756462B
:10A7B000EAE7504683F0A6FE824648B1002E9DD0BF
:10A7C0004FF4FA73C5F8F0344FF0000A4F46DFE754
:10A7D000D5F8FC24012A07D0032AD9D12046FFF757
:10A7E0002DFF00288AD1E9E7DBED807AF5EEC07A0B
:10A7F000F1EE10FA82DD95F8F834002B7FF47EAF8D
:10A80000DEE704F5F45604F58059103699F8DE1F9A
:10A81000304610F05FFB0028C2D099F8DE1F3046AA
:10A8200010F050FC0028B9D1BAE7D5F8EC0410B903
:10A83000C5F8EC844AE7D5F8F024A8EB0008904569
:10A84000FFF444AF95F8E924002A7FF43FAF0122DA
:10A8500085F8E9249BF86011CB0705D504F5AF40D6
:10A860000C210830F7F786F904F54E500830BAF19C
:10A87000000F06D0054A022103B0BDE8F04F53F0A7
:10A88000E3B9034A5146F7E700009642C02E0D088F
:10A89000D62E0D082DE9F04F2DED028B044685B024
:10A8A000002304F50059039387F0F4FAD9ED577AA1
:10A8B000F5EEC07AF1EE10FAC4BF9FEDC47A67EEF0
:10A8C000877A04F5907BC8BFFCEEE77A804658464D
:10A8D000CCBF17EE907A9627F7F798FA022840F245
:10A8E0000C8194F8E4339FEDBA7AB02202FB034363
:10A8F000D3ED777A67EE877AFCEEE77A17EE903A37
:10A900009F428CBF00270127B9F95031022BB8BFF5
:10A91000022307EE903A04F59350B8EEE78A03A9B4
:10A92000F6EE087A083028EE278A12F0EFFB05468B
:10A9300040B1DDED037AF4EEC87AF1EE10FAACBF67
:10A94000012500255846F7F761FA01281AD804F5C1
:10A95000AF40083075F0C6FCA0B19DB904F5AA431C
:10A9600093ED007ADFED9B7AB4EEE77AF1EE10FA20
:10A9700008DDDDED037AF4EEC87AF1EE10FAACBF33
:10A980000125002504F5AF40503005F009FA04F523
:10A99000A0468246002840F0018104F5AF4008300F
:10A9A00075F0A0FC002800F0078194F8E43304EB74
:10A9B0000313D3F890317BB158460193F7F726FA89
:10A9C000012800F29C80019BA8EB030041F2873331
:10A9D00098428CBF00230123D6F8A02402B11BB9F2
:10A9E000002D40F08E803D4604F5804204F59843EA
:10A9F000D2F8C02E20339A421AD199F98831002B0F
:10AA000040F08780002386F8EA34D6F8FC34042B23
:10AA100000F0B080072B00F0C380032B08D1204644
:10AA2000FFF70CFE20B1002586F8E954C6F8A454BF
:10AA300096F8EA3403B18DB907EE905A9FED667A25
:10AA4000F8EE677A04F5AA4367EE877AD3ED006AD9
:10AA50009FED627AE6EE877AC3ED007A2046FFF733
:10AA6000C5FD0546A8B196F80415C6F8A08409B935
:10AA7000C6F8088504F5804204F59843D2F8C02E44
:10AA800020339A4205D1D6F8A43403B109B9C6F8E7
:10AA9000A48496F82C3686F8045565F3C30386F82B
:10AAA0002C366EF0AFFB29466EF088FB4C4B2046EF
:10AAB0005D71FFF7F3FD2046FAF75EFD35B199F8B9
:10AAC00006311BB987F0E6F9C9F8080189F8065183
:10AAD0002046FFF78BFD002840F08E8004F5AF4044
:10AAE000083075F009FC80F00100C0B286F80C0552
:10AAF00005B0BDEC028BBDE8F08F002704E753469C
:10AB00006AE728F055FC27F0A3FD00287FF46BAF1F
:10AB10006AE75B4207EE903A04F69803F8EEE77AAC
:10AB200093EDDB7AF4EEC77AF1EE10FA13DD012330
:10AB300086F8EA34C6F8F48404F5AA43DFED297AEE
:10AB400093ED007AB4EEE77AF1EE10FA7FF75DAF9D
:10AB5000C3ED007A59E796F8EA34002B3FF455AF7D
:10AB6000D6F8F43440F6B832A8EB030393423FF62C
:10AB700049AF4AE704F5AC40383083F0C3FC002805
:10AB80003FF456AF06F5926393ED007ADFED157A48
:10AB9000B4EEE77AF1EE10FA7FF74AAF012547E706
:10ABA00006F5926393ED007AFEEE007AB4EEE77A52
:10ABB000F1EE10FAF2D43BE7D6F8FC34002D18BFC2
:10ABC0003D46012B10D1002532E700BF0000B44202
:10ABD0000000C8429A99993E9A99193E9A99593F0C
:10ABE00055870020CDCC4C3E04F5AC40383083F086
:10ABF0007FFC0028E7D11BE7002077E700207047A3
:10AC00000020704701207047034BD3F8FC04431E1B
:10AC100058425841704700BF707B002030B587B064
:10AC200002A818F027F9374883F062FC20B13649B2
:10AC30003648FCF729FB1FE0324883F063FCE8B19B
:10AC4000334C04F12405234604F11002A4F1100151
:10AC5000A4F1D000009583F07BFCCDE90045A4F57C
:10AC60001C7292ED000A2B4904F11003A4F11002AA
:10AC7000A4F1D00083F02EFC07B030BD214802A91A
:10AC800083F07EFC08B102A9D2E7234CD4F8703BD4
:10AC9000002B0CDD94F8103B4BB1A4F500501C497F
:10ACA000FCF7F2FAA4F50050FCF7A6FBE4E717481E
:10ACB00004F036F90028BAD1184CD4F82C37002B00
:10ACC000B5D004F5E36204F5DF6104F5E16018F046
:10ACD0006DFB0028ABD104F29C45D5ED007AB7EEB0
:10ACE000000A04F5E361A4F5A04030EE670AFCF722
:10ACF00031FC04F5DF6204F5E361A4F5A040FCF744
:10AD0000DBFAB9E7A881002088820020702B0020A0
:10AD10007882002060570020704B0020707B00205C
:10AD200008B50A4890F8F931013B012B03D8A0F58A
:10AD30000050F8F7FFFA0648F8F7CAF90448F8F7A0
:10AD4000B9FABDE808400248F8F71EBE704B002073
:10AD5000702B002010B5044607480CF0F3FE50B1EC
:10AD6000064B93F8110930B1236820469B6B984736
:10AD700080F00100C0B210BD78850020707B0020FB
:10AD8000124B984210B5044601D1002010BD03F1CA
:10AD90001C029042F9D003F138029042F5D003F141
:10ADA00074029042F1D0D4339842EED003681B6A0B
:10ADB000984720B1064B93F88233002BE5D12069E8
:10ADC00007F006F980F00100C0B2DFE7A0760020AE
:10ADD000705B0020174B984210B504460ED003F16B
:10ADE0001C0290420AD003F13802904206D003F1CF
:10ADF0007402904202D0D433984206D10E4B93F99C
:10AE0000B101B0FA80F0400910BD03681B6A984791
:10AE100018B10A4B93F8823343B9206907F0D8F888
:10AE200030B12069BDE8104009F078BC0020EBE7A4
:10AE30000120E9E7A0760020704B0020705B002025
:10AE400073B50F4E0D46114696F99C281AB9012488
:10AE5000204602B070BD036801915B6998470446C3
:10AE60000028F4D1D6F8943A019913F4802FEED04B
:10AE70000448054B00682A46C06A25F047FCE7E70E
:10AE8000707B00206C2B0020E82E0D08084A026021
:10AE9000084A4260111F816002F10801C160A2F1FD
:10AEA000380102F59C724261034A01618261704778
:10AEB000342F0D0878830020D83D002008B50368A2
:10AEC0001B6E98470648D0F8C02E00F604439A42FD
:10AED00005D0BDE80840A0F58040FEF78FBD08BD55
:10AEE000706B00202DE9F3415A4C04F58F6300226A
:10AEF0001A60A4F57873C11A4B42A4F500584B416F
:10AF000088F8183604F59163002684F85C64A4F888
:10AF1000B26484F8B66484F8746484F8E96484F8EC
:10AF2000EA64C4F8DC64C4F8D864C4F8D464C4F82F
:10AF3000E4641A608369D3F8FC31A4F8AC3404F5F6
:10AF4000E16305460FCB04F5DF6787E80F0084F85F
:10AF5000B56484F8C464C4F8D46686F09BFFA4F595
:10AF60008057C7F8C80E2B6828465B6998474FF092
:10AF7000FF3384F8B964C7F8F83E88F8846384F82E
:10AF8000B804286906F0B2F984F8B7642B6828463B
:10AF9000DB6D98470646002858D02B6828469B6BE7
:10AFA000984784F8F804D8F8A4050368DB6B984741
:10AFB000A4F5E75077F006FBA4F5A0400AF05CF892
:10AFC000A8F6B87065F034FA94F82835CBB1A4F53A
:10AFD000A040FFF70BFBA0B904F5F16075F08CF908
:10AFE00078B9D7F8C00E03685B6B984748B959F039
:10AFF00087FC194A062152F027FE04F5A4602FF0C1
:10B00000C3F91648F7F7DCF92B6993F9CC206AB13C
:10B01000586801A912F07AF82C699DED010A0146E1
:10B0200004F18800FBF7A2FE84F841012B68284652
:10B030005B69984750B12B6993F93C22002A02DDE5
:10B0400093F8A03213B9002387F8CD3E304602B002
:10B05000BDE8F081707B0020F42E0D08702B0020DD
:10B0600070B503685B6E0E4615469847044650B9A6
:10B0700095F900303BB90548054B00683246C06A77
:10B08000294625F043FB204670BD00BF6C2B0020F5
:10B09000182F0D0810B50E4C204677F08FF804F5E8
:10B0A000AC7076F007FE04F52C7077F035FD094B97
:10B0B00003F5A042002182F8741402F58F6200218A
:10B0C00003F500531160012283F8482E10BD00BF24
:10B0D0006C5A0020702B002008B52DED028B152036
:10B0E000B0EE408A5CF0C0F9B0EE480ABDEC028BCD
:10B0F0001A20BDE808405CF0B7B9000008B5084860
:10B1000090F9B1310121A0F5005033B10AF032FAC3
:10B11000BDE8084046205CF0A7B90AF053FAF7E70B
:10B12000704B0020012070470120704701207047BC
:10B130000120704701207047192070470048704770
:10B140009C2F0D0800487047AC2F0D0884B010B537
:10B1500003AC84E80E000369B3F9C01064235943BB
:10B160002046012217F08CFE04482146FCF7E6FD3C
:10B17000BDE81040012004B0704700BF702B0020D4
:10B1800013B50F4901AAA1F1100017F02FFF40B12C
:10B19000DFED0C7A9DED017AB4EEE77AF1EE10FA6C
:10B1A0000CD8094CD4F8A40503689B6B984728B1C8
:10B1B00006492E22A4F540500BF0D0FD02B010BD80
:10B1C00088820020000000B4705B0020A47800207A
:10B1D00030B51D4C0546D4F8C40E036887B05B69D2
:10B1E000984738B119491A482F220BF0B7FD0120B2
:10B1F00007B030BD174806F0EBFE0028F2D1A4F5E9
:10B200008054D4F8A40503689B6B984728B1D4F800
:10B21000A40503681B6C984798B10F4B0FCB02AC89
:10B2200084E80F00284601F065F82868059B009324
:10B2300094E80E00446C2846A0472846FFF7A0FF7C
:10B24000D5E7064BEAE700BF706B0020A47800202A
:10B25000702B00204083002078820020888200200C
:10B2600010B50446FFF78CFF2046BDE8104001F002
:10B270007DB800000420704700487047A1350D08D4
:10B2800000487047A1350D08037F73B1D0ED087AEF
:10B29000FDEEE77A17EE903A084AC2F81035437F80
:10B2A0003BB1436AC2F8143570478369D3F8F8316B
:10B2B000F2E78369D3F8FC31F4E700BF707B00202C
:10B2C00008B50023838300F12801806911F034FF61
:10B2D000012008BD70B56E4E2DED048B06F59E4322
:10B2E00004460121304693ED049ADFED6A9A09F095
:10B2F00071FF0121B0EE408A304609F075FFC8EEBB
:10B30000297A06F50055A069B5F9D43104F1280170
:10B3100008EE903AF8EEE88AB5F9D63168EEA78AD9
:10B32000C0EE297A08EE103AB8EEC88A28EE278ACD
:10B3300011F002FF95F9DA3163B39FED577AF0EE21
:10B34000E87AF4EEC77AF1EE10FA23D5227FA369EA
:10B35000002A55D1012222770022226294ED087A38
:10B36000DFED4E7AD3F8F8314D4A4E4867EEC77A92
:10B370009FED4D7A67EE877AB0EE490AFDEEE77AE7
:10B3800017EE901A0B44C2F810350023012276F014
:10B39000A5FE08E0002343482377F0EE490AB0EE0B
:10B3A000680A76F097FE04205CF05EF895F9DA31D1
:10B3B00043B19FED397AF0EEC87AF4EEC77AF1EE38
:10B3C00010FA28D4002339486377F0EE490AB0EE2A
:10B3D000480A76F0D9FA13205CF046F8B5F9D8316E
:10B3E000002B03DD324E96F9C23163BB2848202181
:10B3F000F7F71AFB002843D1254809F00DFD42E07C
:10B40000D3EDC56A96ED467AD4ED087AE6EE877AF2
:10B41000C4ED087AA2E7637F2BB901236377A369A0
:10B42000D3F8FC3163621E4B616AC3F81415A3693B
:10B43000D3F8FC010023091A1A461C48B0EE490A49
:10B4400076F088FBC7E70121A6F5405009F0D6FE4B
:10B4500080EE297AB5F9D831002106F5D67007EECD
:10B46000903AF8EEE77AF0EE490A27EE870A77F08D
:10B4700053FABDEC048B2046BDE87040FFF72CBEAC
:10B480000348F8F7EDF807EE900AB8EEE70AF0E7A0
:10B49000702B002000A08C4500000034E02E654297
:10B4A000707B00206C5A00200000C842C45B002062
:10B4B000705B00202DE9F04F2DED0C8BDFF8A4A37D
:10B4C0009FEDDDDA9FEDDD9A97B00AF59E4300F11E
:10B4D000280504460121504693ED04BA09F07AFE8E
:10B4E00001215046F0EE408A09F07EFE01215046CF
:10B4F000B0EE408A09F082FEDFEDD17A88EEA77ABD
:10B500000AF5005601A8B6F9D4310AF5A04B0AEEA7
:10B51000903AF8EEEAAAB6F9D631DFEDCA8A6AEEB9
:10B5200087AA88EE277A0AEE103AB8EECAAAB6F9C8
:10B53000D8319FEDC58A2AEE07AA80EE277A09EE58
:10B54000903AF8EEE99A6AEE8D7A69EE879AF0EE13
:10B55000EACAF4EEC8CACDED017AB0EECACA6AEE04
:10B560000D7AF1EE10FAF0EEE9BAB4EEC8CACDEDFC
:10B57000027A58BF4FF0010969EE8D7A48BF4FF04B
:10B580000009F1EE10FAF4EEC8BA9AED460ACDEDD4
:10B59000037A54BF4FF001084FF00008F1EE10FAA3
:10B5A00054BF012700272BF097FD01A928462BF057
:10B5B0003DF828462BF034F928462BF0A3F820EE6E
:10B5C000090A284620EE280ABDEEC00A10EE103AFD
:10B5D000CBF810352BF0B0F820EE090A20EE280A3F
:10B5E000DFED9A8ABDEEC00ACDED0D8A10EE103A5D
:10B5F000CBF814350DF1280B4FF07E535946A06956
:10B600000A93CDED0C8ACDED0B8A11F095FD00214A
:10B61000504609F0AFFFB0EEC00AB4EEC80AF1EE32
:10B6200010FA16D55046FEF7E1FF90B9F4EEC8CAFD
:10B63000F1EE10FA0DD5B4EEC8CAF1EE10FA08D545
:10B64000F4EEC8BAF1EE10FA44BF9BE80F0085E8AB
:10B650000F000AA82BF048F9294612A88DED141AFC
:10B660008DED120ACDED130ACDED151A2BF04EF922
:10B670000DF1100A51460EA88DED101ACDED048A79
:10B68000CDED058ACDED068A8DED0E0ACDED0F0AC2
:10B69000CDED111A2AF004FFB6F9D431DFED6C7A42
:10B6A00001EE103AB6F9D63109EE103AB6F9D831B2
:10B6B00008EE903AB8EEC11AB8EEC99AF8EEE88AE8
:10B6C00021EE271A29EE279A68EEA78AF4EEC8CA57
:10B6D000F1EE10FA21EE0D1A29EE0D9A68EE8D8A20
:10B6E00007D594F83830DFED597A002B18BFB0EE4B
:10B6F000671AB4EEC8CAF1EE10FA07D594F83930DB
:10B70000DFED527A002B18BFB0EE679AF4EEC8BA9C
:10B71000F1EE10FA07D594F83A30DFED4C7A002BB1
:10B7200018BFF0EE678A9AE8070007AE86E80700C0
:10B73000F1EE410AC2209DED070A28F075FBC320F7
:10B740008DED070AB0EE491AF1EE490A9DED080A9F
:10B7500028F06AFBB0EE681AF1EE680A8DED080A6F
:10B76000C4209DED090A28F05FFB514630468DED5F
:10B77000090A2BF047FC12A928468DED120ACDEDDF
:10B78000130A8DED141A2AF051FF28462BF048F8C1
:10B79000304BDDED076A93ED007A9FED280AC6EE87
:10B7A000877A3046DDED086ACDED077AD3ED567A1B
:10B7B00086EEA77ADDED096A8DED087A86EEA77A26
:10B7C0008DED097A2BF088FCB9F1000F01D0CDED99
:10B7D00007AAB8F1000F01D08DED08AA0FB1CDED89
:10B7E000099AF0EE4B0A9DED070A1B4876F072FCB1
:10B7F00004205BF039FEF0EE4B0A9DED080A174875
:10B8000076F0C2F813205BF02FFE0021F0EE4B0A19
:10B810009DED090A124877F07FF82046FFF75CFC9F
:10B8200084F8389084F8398084F83A7017B0BDEC09
:10B830000C8BBDE8F08F00BF35FA8E3CE02E6542E0
:10B8400000A08C450000C842000000340000000049
:10B85000CDCC4C3E705A00206C5A0020C45B0020B6
:10B860001C5D0020702B002010B50446FFF746FC3D
:10B870000B4B93F9DA21022A0DD1B3F9D821002A12
:10B8800009DD03F5805393F9C23123B12046BDE8A9
:10B890001040FFF70FBE2046BDE81040FFF71ABD6D
:10B8A000704B00200A20704700487047AE550D08C5
:10B8B00000487047AE550D080120704701207047C1
:10B8C0000120704701207047034BD3F8FC04031F8D
:10B8D00058425841704700BF707B002038B505467C
:10B8E0002C48D0F8C42E00F684439A4215D12B6917
:10B8F00093F844318BB100F5A9502EF00FF90446AE
:10B9000058B958F0FDFF244A032152F09DF92B69E4
:10B91000012283F84321204638BD204C94F8E438B6
:10B9200023B194F99C389A1E5342534184F8B83499
:10B9300004F5E1630FCB04F5DF6504F5E36485E806
:10B940000F0084E80F0016482EF05EFF154B1C68B0
:10B95000E56A2B6828465B689847A8B195F84D3092
:10B9600093B1E36A9B8F7BB158F0CAFFE36A0E4A3A
:10B970009B8F062152F068F9E36A0948998F2EF0EF
:10B980002FFDE36A00229A87084883F033FD0124E3
:10B99000C1E700BF706B002094300D08707B002061
:10B9A000908000206C2B0020AE300D08F854002051
:10B9B00038B50D4C94F82435012B11D104F5A46051
:10B9C0002CF024F8B4F85E5504F5FA60294605F029
:10B9D000F1FC28B9152D03D104F5C76082F068FE8B
:10B9E0000023C4F8A43438BD707B002008B511F0E2
:10B9F000BDFD90F87C32DB0704D5BDE80840024865
:10BA00002EF09EBD08BD00BF9080002038B5354C9B
:10BA100094F82435012B0ED0A4F56D710822A4F5FD
:10BA2000A0400BF09BF958F06BFFBDE838402E4A60
:10BA3000062152F009B904F5FA60B4F85E5505F034
:10BA4000DDFC28B104F5FA60BDE8384008F010BE0E
:10BA5000162D05D0152D36D1D4F8FC34072B0AD17C
:10BA600022480CF08DFF21480DF0D6F8BDE8384093
:10BA70001E480CF0E7BFA4F5A040F8F713F9A4F5B1
:10BA8000A040F7F7F1FFA4F54053D4F8101593F94F
:10BA9000182264235A4304F5C76082F065FDC4F898
:10BAA000100504F5C76082F0A1FE30B1BDE8384052
:10BAB0009FED0F0A46205BF0D7BCA4F5A040BDE87F
:10BAC0003840F7F7B5BD1E2D18BF4FF0FF330748BC
:10BAD00018BFC4F87034F8F7E5F80448F7F7C4FF66
:10BAE0000248ECE7707B0020C8300D08702B002066
:10BAF0000000000070B5134890F99C380E461546BA
:10BB000013B90124204670BDD0F8943A5B0310D5D8
:10BB1000B0F85E1500F5FA6004F0F0FE044640B996
:10BB2000094B0A48006832462946C06A24F0EEFDF7
:10BB3000E8E707482DF0F2FF04460028E1D1054B65
:10BB4000EFE700BF707B0020F4300D086C2B002065
:10BB50009080002008310D0810B5144BB3F85E3505
:10BB6000532B04461ED10AF009F99FED110A462015
:10BB70005BF07AFC9FED0E0A49205BF075FC9FEDAF
:10BB80000C0A4A205BF070FC46205BF04DFD49201A
:10BB90005BF04AFD4A205BF047FD2046BDE81040BF
:10BBA000FFF778BABDE81040FFF7BAB8707B002005
:10BBB00000000000082070470048704794310D08CD
:10BBC00000487047A0310D080120704708B50248B1
:10BBD000FDF7B4FE012008BD702B0020014800F0E5
:10BBE00061B900BF1477002010B50446FFF798F83C
:10BBF0002046BDE81040FFF781BA000001207047E1
:10BC00000048704718320D080048704720320D0870
:10BC1000012070470120704710B5054B03F5E36420
:10BC200003F5E1630FCB84E80F00012010BD00BFD6
:10BC3000707B002008B50B4800F5A04200F50053CA
:10BC40000321D3F8E03B93FBF1F3C2F81035F7F78B
:10BC50006FFF0448F7F708FFBDE808400148F7F711
:10BC6000E7BC00BF702B00200720704700487047DA
:10BC700061140D080048704798320D080120704784
:10BC800001207047012070477047000008B500236D
:10BC900003774362034883F0ADFB0348FBF7EAFAFE
:10BCA000012008BDF8540020702B002010B5194C5D
:10BCB000D4F8C83BB3F9083023B9D4F8D43BB3F96E
:10BCC0000830F3B1002303774362D4F8C80B5AF06D
:10BCD000A9F904F53E63D3ED007A0F48F8EEE77A50
:10BCE00027EE800ABDEEC00A10EE103AC0F81035FB
:10BCF000A0F5A040F7F71CFFBDE81040074803F08F
:10BD000003B8037F002BE0D0A4F50050F7F7CAFF7B
:10BD1000F2E700BF704B0020707B0020702B0020EA
:10BD200070B54E4DDFED4E7A95F8E4339FED4D7AC8
:10BD30002DED048BB02606FB035393ED788A9FED1F
:10BD40004A9A28EE278A05F5A353BDEEC88A93EDDB
:10BD5000050AF8EEC87A044667EE897A97EE870AF4
:10BD600028F04EF8237FF0EE408A002B62D105F5D3
:10BD70000053D3F8C83BB3F90830002B5AD12846FA
:10BD800009F04AF8002855D195F8E43395F82814BD
:10BD900006FB035393F8C12100294BD1012A49D94D
:10BDA00093ED777AF0EE087AB4EEE77AF1EE10FAD6
:10BDB00040DBDFED2E7AB0EEE80AB4EEE70AF1EEF2
:10BDC00010FA37D5636A93B386F064F8636AC01AD1
:10BDD000B0F5FA7F32D8237F002B3CD0244DA5F15B
:10BDE000200696E80F0085E80F0094ED088AA5F17B
:10BDF00010013046B8EEC88A17F06CFB28EE098AAD
:10BE0000DFED1C0A284670EE200AB0EE480A17F053
:10BE100007FC194B9FED190AD3F8A405BDEC048B60
:10BE200003682A4631469B6ABDE87040184786F091
:10BE300031F86062636A002BCDD0C5E7104D84ED08
:10BE4000088A012323770023636205F110030FCBD7
:10BE500085E80F00BFE7BDEC048B70BD702B0020A0
:10BE60000000C84235FA8E3C0AD7233CDB0FC93F9D
:10BE70008882002000007A44705B002000000000EF
:10BE800068820020036A0B60007F704705207047BE
:10BE90000048704710330D080048704720330D08E4
:10BEA0000120704738B54B4D2DED028BD5F8C80BEE
:10BEB0009FED498A5AF0B6F8D5F8E03B07EE903A84
:10BEC000F8EEE77A05F5405427EE800AA5F5005014
:10BED000BDEEC00A10EE103AC4F81035F7F728FE90
:10BEE000D5F8CC0B5AF09EF8B5EEC00AF1EE10FA78
:10BEF000DABF05F6E433D3ED007AD5ED5A7A374848
:10BF0000CBBF20EE270A20EE270A20EE080A28EEF3
:10BF1000400ABDEEC00A10EE103AC4F81435F7F727
:10BF2000D3FD95ED5A7AD4F8140505F6E43327EEDF
:10BF3000087AD3ED007A27EE888AFDEEC77A17EEED
:10BF4000902AFDEEC87A17EE901A28F00DF8C4F882
:10BF500014052248FDF77EFD20B1D4F814355B426C
:10BF6000C4F814351E4B93F8D43E63B195F9BC3137
:10BF7000022B08D1002301214620C4F81035C4F853
:10BF800014355BF0D5FD59F05DFF5F215AF01EFFBF
:10BF9000E8B15AF0EBFE022819D194F8B534B3B9E0
:10BFA00004F5916393ED007AD5ED827AB4EEE77AE9
:10BFB000F1EE10FA0BD5012384F8B534BDEC028BF9
:10BFC000084A0948BDE83840042151F03DBEBDECA7
:10BFD000028B38BD704B00200000C842702B00203F
:10BFE000706B002028330D08F85E002010B5044661
:10BFF000FEF796FE2046BDE81040FFF77FB8000030
:10C000000620704700487047A8330D080048704765
:10C01000B8330D0801207047012070470120704798
:10C02000012070477047000008B5044883F0E2F92A
:10C030000348FBF71FF9012008BD00BFF85400209A
:10C04000702B002038B50F4C04F50055D5F8C80BFF
:10C0500059F0E8FF05F53E62D2ED007AF8EEE77A96
:10C0600004F5A04327EE800A2046BDEEC00A10EE7C
:10C07000102AC3F81025F7F75BFD2046BDE83840CD
:10C0800002F042BE702B00200F207047004870471E
:10C0900030340D080048704738340D0801207047CF
:10C0A0000120704701207047012070470120704730
:10C0B0000120704730B5184B2DED028B002283F81C
:10C0C000822303F51C53083305460FCB85B06C461D
:10C0D00084E80F00114804F0CFFB90B1A86900F587
:10C0E0007F702AF029FE0D48B0EE408A04F02CFC47
:10C0F000F0EE400A9FED0A0A204628EE000A17F0EB
:10C100008FFA00230748EB612146FBF717FE012059
:10C1100005B0BDEC028B30BD705B00204083002079
:10C12000E02E6542702B002038B5424C94F8B934AB
:10C1300043B194F8E4382BB104F5FA60BDE8384017
:10C1400008F066BAD4F8D434002B18DC3A48F7F774
:10C15000A9FDD4F8D834002B29DC3748F7F784FC44
:10C16000364890F88233002B46D00121A0F540508C
:10C1700009F000FABDE8384046205BF075B985F05B
:10C1800089FED4F8D434C01A40F6B7339842DDD8CB
:10C190002B4DD4F8C804D5F8E02B514227F0E4FE2B
:10C1A000C4F81005A5F50050F7F7C2FCD1E785F0FB
:10C1B00071FED4F8D834C01A40F6B7339842CCD8C0
:10C1C0001F4BDFED206A93ED5A7AD4F8CC0403F6C6
:10C1D000E433D3ED007A27EE267A67EEA67ABDEE39
:10C1E000C77AFDEEE77A17EE102A17EE901A27F0BD
:10C1F000BBFEC4F81405B3E7A0F5805090F94731B1
:10C20000012B04DCBDE838400B48F7F711BAD4F82D
:10C21000E434002BF6D085F03DFED4F8E434C01AA7
:10C2200040F6B7339842EDD804F59C6494ED000ACB
:10C23000A0E700BF707B0020702B0020705B002007
:10C24000704B00200000C842D0ED077A0348FCEE96
:10C25000E77A17EE903A99B202F032BF702B0020C5
:10C2600084B010B503AC84E80E000B4821466F2261
:10C27000FBF7AAFC9DF80C1011F0040102D1204636
:10C2800016F090FE04482146FBF758FDBDE810402B
:10C29000012004B0704700BF702B0020B0EEC00A30
:10C2A000FDEEC07A38B54FF6FF7205460C4617EE24
:10C2B000900A002127F058FE07EE900A002CF8EEB5
:10C2C000E77A054BC5ED077A14BF4FF0FF32012224
:10C2D00083F8D02638BD00BF707B0020FEF79EBCDF
:10C2E0000C2070470048704711370D080048704710
:10C2F000E6710E0808B50C48FCF76CFA0A480B49C1
:10C30000FBF7E2F80848F6F709FE40B106484FF49B
:10C310008051F6F789FB10B10348FAF7ABFF0248EA
:10C3200002F0C8F9012008BD702B0020888200208F
:10C3300008B50D48F7F7B6FC0B48F6F7EFFD50B11E
:10C3400009484FF48051F6F76FFB20B1BDE8084073
:10C35000054802F0D9BC0448F7F786FBBDE8084061
:10C360000148F7F765B900BF702B002008B50A48EF
:10C370004FF48051F6F758FB38B108480022D0F846
:10C38000281700F5E36016F07BFDBDE80840024881
:10C39000002102F095BE00BF702B0020707B0020B2
:10C3A000881A10B527F008FD104BD3F8CC260028CA
:10C3B000B8BF4042002AB8BF524248F6A041B2FB83
:10C3C000F1F24FF47A7102FB011188420CDC93F810
:10C3D0001827D20606D503F5E36403F5E1630FCB16
:10C3E00084E80F00012000E0002010BD707B0020D9
:10C3F00013B504468069019100F57F702AF09CFC1A
:10C40000DFED0A7A20EE270A27F078FCDFED087AC4
:10C41000019920EE270A2046FDEEC07A17EE902AF9
:10C4200002B0BDE81040FFF7BBBF00BFE02E654281
:10C430000000C84284B070B52DED048B86B00FADFE
:10C4400085E80E004E4CDFED4F8A0646D4F8A40571
:10C4500004F5005404F2E46393ED000A0368B0EEBF
:10C46000C00A5B6A9847B4EEE80AF1EE10FAB0EE43
:10C47000408A07DA012006B0BDEC048BBDE87040AD
:10C4800004B070474049284616F030FF02A8CDEDB1
:10C49000030A8DED020A2AF01FFD04A88DED040A9F
:10C4A000B0EE480ACDED050A2AF0D2FB13A92846C2
:10C4B0008DED000ACDED010A16F018FF02A88DEDF2
:10C4C000020ACDED030A2AF081FCB4EEE80AF1EE8F
:10C4D00010FACFDBB4EEC08AF1EE10FA9FED2B9A82
:10C4E000DFED2B8ADFED2B9A2BD802A869462AF0C4
:10C4F0009FFB04A88DED040ACDED050A2AF01CFC73
:10C50000684620EE098A2AF017FC94F9D03607EE27
:10C51000903AF8EEE77A28EE288AA7EEA90A27F0E3
:10C520006FFC20EE090ABDEEC88A20EE280A18EE3C
:10C53000101AFDEEC07A304617EE902AFFF730FF52
:10C5400099E738EE400A38EE088A80EE080AAAF029
:10C5500007F802A8B0EE408A2AF0EEFB94F9D03634
:10C56000F0EE007AB0EE697AA8EE677A07EE903ABC
:10C57000F8EEE77AA7EE270A27F042FCC0E700BFF3
:10C58000705B00200000003478820020E02E6542BD
:10C590000000C842DB0FC93F10B504460848F6F753
:10C5A000BDFC20B92046BDE81040FEF737BB04486B
:10C5B0004FF48051F6F738FA0028F3D010BD00BFD1
:10C5C000702B0020002070470048704720350D0870
:10C5D0000048704728350D0800207047036993F81C
:10C5E000140118B1D3F8C402C0F3801070470000E2
:10C5F00038B5154C05460021204608F0EBFD042017
:10C600005AF032FF0021204608F0EEFD13205AF0C8
:10C610002BFF0021204608F0F1FD2846FEF75CFDC7
:10C620002046012108F0A6FF46205AF01DFFAB6905
:10C6300004F5A044D3F8F831C4F81035AB69D3F849
:10C64000FC31C4F8143538BD702B0020FEF722BD34
:10C650001720704700487047A0350D080048704704
:10C66000A8350D0801207047012070470120704750
:10C6700010B50369002283F8402103690446D3F80A
:10C680003C0103689B689847A36818687CF076FAB9
:10C69000206904F06DFE0349A06910F04DFD0120F2
:10C6A00010BD00BF007700201FB50B4C9FED0B0A9B
:10C6B000D4F804086C302AF0BBFCFDEEE00ABDEEB5
:10C6C000C00A10EE903AC4F8143510EE103AC4F8CF
:10C6D000103504B010BD00BF707B00209F0CB34527
:10C6E00030B52DED028B83B0044685F0D3FB0146B7
:10C6F000206900F50E700BF06FF938B1204603B0D9
:10C70000BDEC028BBDE83040FEF70ABB206990F813
:10C710004031BBB1012104F0B1FDA368DFED400A57
:10C720001868036801215B6EB0EE600A98472069C3
:10C7300003F0FAF93B4803B0BDEC028BBDE8304092
:10C74000FFF792B8384DDFED398A022104F096FDEB
:10C75000D5F8CC0B59F066FC2369D3ED390A93F96F
:10C760003C2220EE200A002A60EE280A3FDD93F8E2
:10C77000A032002B3BD0D5F8D40BCDED000A59F0F8
:10C7800051FC2369D5F8C80B93ED3A8A20EE080ACC
:10C7900020EE288A59F046FC236993ED381A20EEE2
:10C7A000410A20EE281ADDED000A2069CDED010ACC
:10C7B0008DED001A03F0F4F9A36895F9DA211868F1
:10C7C0009DED001ADDED010A0368F0EE408A2AB300
:10C7D0001B6CB0EE480A9847A36818680368F2EE2D
:10C7E000040A5B6E0021B0EE680A9847A2E7D5F80C
:10C7F000C80BCDED000A59F015FC2369D5F8D40B10
:10C8000093ED388A20EE080A20EE288A59F00AFCB7
:10C81000236993ED3A1A20EE010AC2E7DB6BD8E7F1
:10C8200000000000D8760020704B00200000C842B5
:10C83000122070470048704720360D0800487047A6
:10C8400028360D08012070470120704701207047ED
:10C8500038B52DED028B43689FED1C8A1D68044698
:10C86000006904F0A7F9236993ED131AD3ED110AB7
:10C87000434200EE103A21EE081A60EE880AB8EE44
:10C88000C00A28467DF034FB636820691D6804F007
:10C8900091F9236993ED131AD3ED110A434200EE87
:10C8A000103A21EE081A60EE880AB8EEC00A28464F
:10C8B0007DF098FB9FED060A206903F061F920697D
:10C8C00005F016FFBDEC028B012038BD0000C84208
:10C8D00000000000014800F051BE00BF4C7800206D
:10C8E00013B5044600698830FAF7A2FB85F0D2FA46
:10C8F0000146206900F50E700BF06EF828B1204655
:10C9000002B0BDE81040FEF70BBA206990F8403144
:10C910003BB3012104F0B2FCA368DFED170A1868ED
:10C920000368B0EE600A5B6E01219847206903F04E
:10C93000FBF863689FED100A18687EF003FD0F484E
:10C94000F6F7C6FB0D48F6F7B5FC20469FED0A0A40
:10C95000FEF7C2FB2069883002B0BDE81040FAF74C
:10C9600027BC074804F0EEFD2069019004F088F927
:10C97000019806F0C9FAE2E700000000702B0020E1
:10C98000408300201420704700487047A62F0D08F0
:10C9900000487047F9710E08012070470020704769
:10C9A00070B504460E4800F03BF82369002583F873
:10C9B0004051206904F0A2FF6069052103F058FD91
:10C9C000084826690221FAF727FF86EDB70A23698E
:10C9D000C3F848512369C3F84C51012070BD00BF12
:10C9E00084780020702B0020014800F0C7BD00BFF4
:10C9F0004C780020014800F069B800BF847800201E
:10CA0000132070470048704710370D0800487047E2
:10CA100018370D080120704701207047012070472A
:10CA200038B52DED028BDFED240AC3689FED238A14
:10CA30000446B0EE600A186879F022FCE3681868D2
:10CA400079F0FCFC636820691D6804F0B3F8236981
:10CA500093ED131AD3ED110A434200EE103A21EE82
:10CA6000081A60EE880AB8EEC00A28467DF040FA3F
:10CA7000636820691D6804F09DF8236993ED131A1B
:10CA8000D3ED110A434200EE103A21EE081A60EE8F
:10CA9000880AB8EEC00A28467DF0A4FA206905F09D
:10CAA00027FE256985F0F6F9C5F86C01BDEC028B0F
:10CAB00000230120E36138BD000000000000C842EF
:10CAC000014800F05BBD00BF4C78002030B52DED73
:10CAD000048B0446006985B08830FAF7A9FA38B1AA
:10CAE000B74805B0BDEC048BBDE83040FFF7F8BE99
:10CAF00085F0D0F905462069294600F50E700AF048
:10CB00006BFF38B1204605B0BDEC048BBDE830406A
:10CB1000FEF706B9206990F8403163B3012104F0B3
:10CB2000ADFBA368DFEDA70A186803680121B0EE2A
:10CB3000600A5B6E9847206902F0F6FF63689FED1C
:10CB4000A10A18687EF0FEFBDFED9E0AE368B0EEF6
:10CB5000600A186879F094FBE368186879F06EFC55
:10CB60009948F6F7B5FA984805B0BDEC048BBDE8D6
:10CB70003040F6F79FBBC36A93F8CB3013B99348A4
:10CB8000FFF74EFF206903F035F918B1E368186824
:10CB900079F072FB2369D3F86C31EB1AB3F5FA7FA5
:10CBA0000BD9E368DFED870A1868B0EE600A79F008
:10CBB00067FBE368186879F041FC23699FED848A7C
:10CBC000C3F86C510221206904F058FB63682069A6
:10CBD0001D6803F0EFFF236993ED131AD3ED110ADB
:10CBE000434200EE103A21EE081A60EE880A284609
:10CBF000B8EEC00A7DF07CF9D4E90335186879F005
:10CC0000A9FBA368186803689B6EF0EE408A9847FA
:10CC100003AAF0EE400A02A9B0EE680A284603F023
:10CC200003F8E368DDED030A18689DED020A79F068
:10CC300027FB636818687DF04DF918B963681868B8
:10CC40007EF03EF8E368634D1868012179F062FDDB
:10CC5000E3681B689B68D3EDCF7AFDEEE77A05F5B4
:10CC6000FA6017EE903AC5F81035E3681B689B68C8
:10CC7000D3EDD07AFDEEE77A17EE903AC5F8143589
:10CC800004F060FC2369D3F83C01036805F21452F8
:10CC90005B6B05F5A261984748B163681B68D3F8E0
:10CCA0008823C3F89423D3F88C23C3F898232069EE
:10CCB000DFED499A04F056FBD5F81035206907EEF0
:10CCC000903A012105F21453F8EEE78A93ED009AA9
:10CCD00006F0B4F8A368B8EEC99A186820EE290ADD
:10CCE000036868EEA98A29EE299ADB6A20EE081A01
:10CCF00069EE080A28EE880A9847384BD3F8C02E08
:10CD000003F634518A4248D1636993F86430062BA4
:10CD10000AD8206903F0C2FC30B16069072103F032
:10CD2000A7FB206904F0EAFD27480221FAF774FD09
:10CD3000206903F08BF8636993F86430072BB0EE39
:10CD4000408A08D12369D3F8C4329B0403D4A06974
:10CD5000012110F0B7FE6368B5EEC08AF1EE10FA5B
:10CD60001868CCBF01210021B1EE480A7DF046F9D8
:10CD7000206907F0DDFD206903F03AFF1248F6F75D
:10CD8000A7F91148F6F796FA9FED0E0A2046FEF72E
:10CD9000A3F905B0BDEC048B30BD03F684439A4281
:10CDA000206907D190F8423123B19FED060A02F0C5
:10CDB000E7FEE0E7019003F063FF0198F7E700BFAB
:10CDC0006878002000000000702B0020847800208C
:10CDD0000000C842707B00200AD7233C706B002003
:10CDE000152070470048704790370D08004870477D
:10CDF00090370D08012070470120704700207047D0
:10CE0000C369012B06D1044B93F8A409431E584271
:10CE10005841704700207047707B00200E4BB3F9DB
:10CE20007A21B3F9AC3107EE102A07EE903AB8EE4A
:10CE3000C77AF8EEE77AB0EEC77AF0EEE77AB4EEAA
:10CE4000677AF1EE10FAC8BFF0EE477AB7EE080A3B
:10CE500027EE800A704700BF704B00202DE9F0419B
:10CE6000774C2DED048B94F814898AB00546B8F1FF
:10CE7000000F0CD03122A4F53371A4F5A04009F0C5
:10CE80006DFF01200AB0BDEC048BBDE8F0810123E9
:10CE9000C36104F5E16696E80F0004F5DF6787E8F3
:10CEA0000F002B69D4F8F426B3F8C070DB6A52681F
:10CEB00093F8A0306421022B17FB012740F09880E3
:10CEC00007EE907A3246B8EEE70AA4F5A04106A82C
:10CED000FBF74EF806A9304616F0FCFA2846F0EEAD
:10CEE000408AFFF79BFF2B69B3F9C020D3ED310ACD
:10CEF00001EE102AB3F9C220B0EE409A00EE102ADB
:10CF0000B8EEC11A1A20B8EEC00A26F08DFF2B69C0
:10CF1000B3F9C030F4EEC98A07EE903AF1EE10FA98
:10CF200054BFF0EE686AF0EE496AB8EEE77AC8EEF0
:10CF3000A67A42460821A4F5A040B0EE408A67EEEA
:10CF4000877AB4EE670AF1EE10FA48BFB0EE678A4E
:10CF5000FAF728FCDFED3B7A38EE408AB4EEE78A38
:10CF6000F1EE10FA1DDBC5F81C8096E80F0004F501
:10CF7000E36585E80F0004F20C73D3ED008ADFED62
:10CF8000327AF8EEE88A3046E8EE278A15F0A2FFFA
:10CF9000FDEEE87A024617EE901A284615F070FF6B
:10CFA0006FE7F4EEC98AF1EE10FA21D505AA4146E1
:10CFB000304615F09BFF18B1059B9F42A8BF1F4646
:10CFC00057F09EFC064619EE100AF3F795FACDE9E4
:10CFD000020118EE900AF3F78FFA1C4ACDE900011E
:10CFE0000621304650F030FE6869032103F040FA14
:10CFF00039461748FAF772FF286903F0C5FC15484F
:10D0000005AA002115F072FF98B1134806AA002165
:10D0100015F06CFF68B1DDE905316A698B4292F861
:10D020002010D4BF0023012363F3000182F82010F5
:10D0300027E76A69D4F80C37D4F81C17EEE700BF6D
:10D04000707B0020000000340000C84298370D08B3
:10D05000702B00207882002088820020014800F098
:10D060008DBA00BF4C780020F0B52DED028B99B041
:10D07000044684F00FFF0146206900F50E700AF0A7
:10D08000ABFC054638B1204619B0BDEC028BBDE8BB
:10D09000F040FDF745BEE36983B1012B00F01E812E
:10D0A000A048F6F715F89F48F6F704F99D4819B01F
:10D0B000BDEC028BBDE8F040F6F766BC9FED9A8AA6
:10D0C00060688DED098A8DED0A8A8DED0B8A8DEDF4
:10D0D0000C8A0BAA09A901230068944D7CF01EFE5E
:10D0E0002069B0EE480A03F00DF963681B68D3EDC0
:10D0F000CF7AFDEEE77A05F5FA6017EE903AC5F8BB
:10D10000103563681B68D3EDD07AFDEEE77A17EE31
:10D11000903AC5F8143504F015FA2369D3F83C01A8
:10D12000036805F214525B6B05F5A261984748B19C
:10D1300063681B68D3F88823C3F89423D3F88C233F
:10D14000C3F89823206904F013F9A36820691E68C6
:10D150003368DF6AD5F8103507EE903AD5F8143504
:10D16000F8EEE78A07EE903AF8EEE70ACDED050A09
:10D1700005F0D8F8DDED050AB0EE401A3046B0EE05
:10D18000680AB8472069C36B93ED070A02F0F8FC00
:10D19000206903F02DFD63688DED0D8A8DED0E8AFB
:10D1A0008DED0F8A18680FA97DF00AF90D9B149375
:10D1B0000E9B159302220F9B169314A910A816F02C
:10D1C000FFF95B4907AA10A815F010FF48B1DFED81
:10D1D000597A9DED077AB4EEE77AF1EE10FAFFF690
:10D1E0005FAF0123E36105F5E1630FCB05F5DF6672
:10D1F00086E80F00D5F8F43622695B68B2F8C060A3
:10D200004849642216FB023607EE906A4A4AB8EE95
:10D21000E70A14A8FAF7ACFE474814A916F05AF921
:10D220002046B0EE408AFFF7F9FDB4EEC08AF1EE79
:10D2300010FAF0EE408A21D53D4808AA002115F0E9
:10D2400055FE18B1089B9E42A8BF1E4657F058FBDA
:10D25000074618EE900AF3F74FF9CDE9020118EEF0
:10D26000100AF3F749F9354ACDE90001062138469D
:10D2700050F0EAFC6069032103F0FAF831462948CE
:10D28000FAF72CFE206903F07FFB294907AAA1F1D8
:10D29000100015F0ABFE636988B19DED077ADFEDF4
:10D2A000257A93F82020B4EEE77AF1EE10FAACBFBD
:10D2B0000121002161F3000283F82020F0E6D5F877
:10D2C0000C27D5F81C178A4293F82010D4BF0022EF
:10D2D000012262F3000183F82010E1E6206906F0E4
:10D2E0007DF8636993F86430042B08D90F48D0F8AF
:10D2F000F4362A46596800F5E36015F0C1FD63690C
:10D3000093F86430032B02D9206907F051FB23699D
:10D3100093F8D431013B012B3FF6C2AE0148F6F73A
:10D3200009F8BDE6702B002000000000707B002093
:10D3300088820020000000347882002098370D0891
:10D3400030B5C369012B85B004D1414C94F8A439A0
:10D35000012B04D005B0BDE83040FDF75FBCA4F55B
:10D360004053DFED3C6AB3F97A219FED3B0A07EEAB
:10D37000102AB3F9AC2107EE902AB8EEC77AF8EE7E
:10D38000E77AB4F99028B0EEC77AF0EEE77AB4EE17
:10D39000677A00EE902AF1EE10FAC8BFF0EE477AF5
:10D3A000B8EEE07AD3ED7A0A03F6A84270EEC70A27
:10D3B00092ED007A27EE267AF5EEC00AF7EE006AC3
:10D3C000F1EE10FAB4EEE67A48BFDFED230AF1EE93
:10D3D00010FAD8BFB0EE667AF3EE046A77EEA71AB9
:10D3E00067EEA67AC0EE876A04F5936204F5E364FB
:10D3F0006D4693ED557A92ED001AB0EE612AA6EED5
:10D40000872AF4EE427AF1EE10FA48BFB0EE672AAE
:10D41000F4EE421AF1EE10FAC8BFB0EE612A26F01F
:10D4200035FC94E80F0007EE901A9FED0C7AF8EEA9
:10D43000E77A85E80F00E0EE077A09482946FDEE15
:10D44000E77ACDED017AF9F71FFF05B030BD00BFD7
:10D45000707B00209A99193F000000000000C8422C
:10D46000702B0020112070470048704728380D08A5
:10D470000048704734380D0801207047012070477C
:10D4800001207047012070470369002283F8402182
:10D4900001207047164B03F6382292ED007AB3F95B
:10D4A000D827D3F80C09B5EEC07AF1EE10FA07EEE2
:10D4B000902AC8BFDFED0F6AF8EEE77ACABF27EE01
:10D4C000267A20EE270A27EE000A67EEA07ABDEE44
:10D4D000C00AFDEEE77A10EE102AC3F8102517EE09
:10D4E000902AC3F814250368034A5B6B111F184781
:10D4F000707B00200000C842848000201D49DFEDC1
:10D500001E6AB1F9D827A1F54050F5EEC00AD0F84F
:10D51000E03B9342A8BF134607EE903AF1EE10FAB3
:10D52000F8EEE77AD6BF00F6E43090ED5A7A90ED47
:10D53000007A27EE800A07EE902ACCBF27EE267AE3
:10D5400027EE667AF8EEE77ABDEEC00AB4EEE77A27
:10D55000F1EE10FA58BFB0EE677A60EE870A10EE6F
:10D56000103AFDEEE00AC1F8103510EE903AC1F81D
:10D5700014357047707B00200000C84237B52B4C33
:10D58000D4F8C83BB3F908201B8B07EE102A07EE2E
:10D59000903AD4F8CC3BB8EEC77AB3F908201B8B8D
:10D5A000F8EEE77A054687EE270A214807EE102AAB
:10D5B00007EE903AB8EEC77AF8EEE77A8DED010AF9
:10D5C000C7EE270ACDED000A09F0B6FFDDED000A2F
:10D5D0009DED010A28B1284603B0BDE83040FFF7B1
:10D5E00059BF04F54053D3F8942A520405D4284671
:10D5F00003B0BDE83040FFF781BFB3F9D82707EE8D
:10D60000902AF8EEE77A27EE800A67EEA00ABDEED0
:10D61000C00AFDEEE00A10EE102AC3F8102510EE45
:10D62000902AC3F8142503B030BD00BF704B002012
:10D630007885002010B5044684F02CFC0146206952
:10D6400000F50E700AF0C8F920B12046BDE8104080
:10D65000FDF766BB114803F075FF206990F9D030E3
:10D660004BB102F027FA0E48F5F732FDBDE8104045
:10D670000B48F5F71FBE02F093FA206905F0FEFB98
:10D680000748F5F725FD0648F5F714FE20469FEDFF
:10D69000050ABDE81040FDF71FBD00BF4083002014
:10D6A000702B0020000000000B20704700487047DE
:10D6B0004E3B0D0800487047AC380D0801207047FC
:10D6C00001207047012070470020704738B530486E
:10D6D000F6F7E8FA2E48F6F7C7F92D48F5F7A8FF50
:10D6E0002B481021F5F7A0F9E0B12A4AD2F80C37FF
:10D6F000D2F81C279342D4BF00230123254C94F871
:10D70000802772B973B304F5E1630FCB04F5DF65CD
:10D7100085E80F00A4F5A040F9F7A8FF012384F8DD
:10D72000803738BD1C4AB2F9AC1B0029F9DD02F57F
:10D7300040529FED1A7AD2F80C37D2F8FC269B1A89
:10D7400007EE903AF8EEE77A67EE877A07EE101A5E
:10D75000B8EEC77AF4EEC77AF1EE10FACCBF012327
:10D760000023CBE7A4F54053642193F91822D4F8A1
:10D77000100512FB01F2D3F8E01B8A42A8BF0A464B
:10D780005142C3F8E02B26F0EFFBC4F81005C8E7C0
:10D79000702B0020707B0020704B00200AD7233CA8
:10D7A000F0B5304C2DED028B04F5E165074695E8A8
:10D7B0000F0004F5DF6686E80F0083B0A4F5A040F3
:10D7C000F9F72CFD0146A4F5A040FAF787FBA4F574
:10D7D0008052002384F88037C2F8E83E94F8E43899
:10D7E000D3B394F814393BB13122A4F53371A4F5C5
:10D7F000A04009F0B3FA2FE094F99E38032B03D12F
:10D800002C22A4F52C71F2E7013BDBB2012B23D8CB
:10D810003B69DB6A93F8A030022B1DD104F5E3616C
:10D82000284615F057FEA4F52C70B0EE408AFFF79D
:10D83000F5FAB4EEC08AF1EE10FA0DD501AA012175
:10D84000284615F053FB38B1B4F89038642213FB26
:10D8500002F3019A9342D3DC012003B0BDEC028BAA
:10D86000F0BD00BF707B002038B52DED028B244D3C
:10D8700095F99E38012B03D00020BDEC028B38BDFA
:10D88000A5F54053B3F9AC41002CB8BF6442A4B233
:10D890002CB9B3F97A41002CB8BF6442A4B2194B39
:10D8A000D3F8A40503689B6B984730B11649174815
:10D8B000272209F053FA0120DFE7154AA2F12001DF
:10D8C00001F1100015F072FD0028EFD1114805F5A7
:10D8D000936595ED008A03F037F807EE904AF8EE6D
:10D8E000E77AB4EEE70AF1EE10FA44BF07EE904A89
:10D8F000B8EE670AB4EEC08AF1EE10FABCD5D5E7EF
:10D90000707B0020705B0020C0780020702B00200E
:10D91000888200204083002070B5464C94F8E4389B
:10D9200088B0054683BB444DB5F9AC3183EAE37159
:10D93000A1EBE37189B2002955D1404801F0C0FB49
:10D9400094F8B634002B3ED195F98731022B52D191
:10D950003B4D95F8F13E9BB13A4905F5A9502CF0A5
:10D9600067FF68B10123282205F54261A5F58040D3
:10D9700084F8593509F0F2F928BB002384F85935A9
:10D98000012384F8B6341EE094F99E38022BA4F5E6
:10D9900080561AD103AD284615F06CFA04F5E363FE
:10D9A0000FCB85E80F0001A9A4F5A040FBF764F9AF
:10D9B000D6F8E83E052B06D12722A4F52C71A4F554
:10D9C000A04009F0CBF908B070BD84F063FAD6F836
:10D9D000C83EC01AB0F57A7FA5D92846FFF744FFA4
:10D9E0000028A0D0EFE7002BB4BF4FF0FF33012396
:10D9F00084F8D036A1E7012B0CD1104801F090FA41
:10DA000040B10E48F9F79CFD0028B8BF4042B0F580
:10DA10007A7F9DDB95F98731042BD4D1084D95F899
:10DA2000F13E002BACD0074905F5A9502CF07CFF46
:10DA300097E700BF707B0020704B0020702B002008
:10DA4000706B0020788200200220704700487047E9
:10DA500029380D0800487047E0710E08034B00227A
:10DA6000C3F81025C3F81425704700BF707B002051
:10DA700038B5094D04462846F5F72AFB2846F5F740
:10DA800019FC2046F5F72EFC2846F5F77DFF2046C9
:10DA9000BDE83840FDF732BB702B00200D207047E9
:10DAA0000048704794390D08004870479C390D08AC
:10DAB000012070470120704701207047002380F843
:10DAC000273080F8383001207047000001480021DD
:10DAD00001F0F6BA702B0020F0B5BA4CD4F8142738
:10DAE000D4F810372DED088B1343D4F80C271343CB
:10DAF00089B005460FD1B448F6F7D4F8B248F5F727
:10DB0000B3FF9FEDB20A462009B0BDEC088BBDE81B
:10DB1000F04059F0A9BC0FF029FD90F87C32DB07EA
:10DB2000E9D5B5F91C3095F8271009EE103AB5F98A
:10DB3000243008EE903AB8EEC99AF8EEE88A002947
:10DB400040F0DD809FEDA2AA29EE0ABA0122FDEE87
:10DB5000CB7AA4F5A04017EE903AC4F88034F9F7D8
:10DB600021FEA86900F57F700790B0EE408A29F089
:10DB7000E3F8DFED987A20EE270A26F0BFF8079841
:10DB8000F0EE409A29F022F9A4F5A040F0EE40AA68
:10DB9000FCF72CFD00287CD104F5E16696E80F0027
:10DBA00005F1280787E80F0096E80F0004F5DF6706
:10DBB00087E80F0004F5E36787E80F00D4F81C3707
:10DBC000854807EE903AF8EEE77AF0EE680A77EECD
:10DBD0008B7AB0EE690AFDEEE77A17EE903AC4F858
:10DBE0001C3715F01DFD002384F8E93495F9263023
:10DBF000754803EB830303EB83039B000121A4F827
:10DC0000AE34F4F7ABFB94F8F874002F77D1734B74
:10DC10009FED737AB3F9503107EE903AF8EEE77A58
:10DC200067EE877AF4EEE7AAF1EE10FA67DD56F0B8
:10DC300067FE064619EE900AF2F75EFCCDE9040194
:10DC400018EE900AF2F758FCCDE9020119EE100A1D
:10DC5000F2F752FC634ACDE90001062130464FF04D
:10DC6000F3FF84F017F9C4F86C74C4F8580484F016
:10DC700011F90123C4F8680429EE8A0A85F82730CF
:10DC800026F066F8BDEEC00A10EE103AC4F8703403
:10DC900035E084F0FFF8D4F80835C01A42F210736A
:10DCA00098427FF679AFF0EE087AF4EEE7AAF1EE4B
:10DCB00010FA7FF771AFBCEEC88A04F5E36718EE7F
:10DCC000103A9BB208EE103AB8EEC88A04F5E16645
:10DCD000B4EEC89AF1EE10FA48D856F011FE424A56
:10DCE00006214FF0B1FF96E80F0087E80F000123EF
:10DCF00085F827300321A4F5A040F4F72FFB324824
:10DD00000BF0CAF830B130480321F4F727FB0023A9
:10DD100085F82730D4F8FC34012B40F0B880D4F8D3
:10DD20000C37EA6A9FED2AAA9B1A07EE903AD4F8BC
:10DD300070340133F8EEE79A5ED0DFED2C7AE9EE2D
:10DD40000A7AF4EEE79AF1EE10FA0ADA284905F1B8
:10DD5000280015F0BFFBF4EEC08AF1EE10FA00F2D5
:10DD6000968019480321F4F7F9FA90E056F0C8FDBF
:10DD7000204A06214FF068FF96E80F0005F1280CB5
:10DD80008CE80F0096E80F0087E80F00D4F81C37E6
:10DD900007EE903A39EE488AF8EEE77AF0EE680A34
:10DDA000E8EE0A7A3846B0EE690AFDEEE77A17EE39
:10DDB000903AC4F81C3715F033FC012185F8271080
:10DDC00099E700BF707B0020702B0020000000004E
:10DDD0000000C842E02E654288820020704B00207F
:10DDE0009A99993EE5390D08A4390D08000048C3F9
:10DDF00078820020C0390D08B5F91E3007EE903A40
:10DE0000F8EEE77A05F1280667EE8A7AF4EEE79AEB
:10DE1000F1EE10FA55DB4449304615F02BFADFEDF0
:10DE2000437AB6EE008AA0EE278A96E80F00BDEE90
:10DE3000C88A9FED3F0AB8EEC88A04F5E36728EE6A
:10DE4000008A87E80F00F0EE680A3A48B0EE480A08
:10DE500015F0E6FBD4F81C3707EE903AF8EEE77AB7
:10DE600028EE0A0AE9EE0A7AFDEEE77A17EE903A12
:10DE7000C4F81C3725F06CFFBDEEC00A10EE103A56
:10DE8000C4F87034D4F8FC34012B3FF456AF2A4860
:10DE90000AF0E2FF18B128480321F4F75FFAD4F83A
:10DEA000FC34012B17D124480AF06AFD22480AF0FD
:10DEB000B3FE214809B0BDEC088BBDE8F0400AF084
:10DEC000C1BD1949304615F005FBF4EEC08AF1EEEC
:10DED00010FAA0D9D6E795F838302BB9174861F079
:10DEE000DBFE012385F838301348F5F7DBFE1248D6
:10DEF000F5F7BAFD1048F5F79BFB114890F884330D
:10DF00006BB1002380F8843333220221A0F5405006
:10DF100009B0BDEC088BBDE8F040FBF78DBF09B040
:10DF2000BDEC088BF0BD00BF78820020A00CB3458B
:10DF30000AD7233C88820020702B0020B84B002099
:10DF4000705B002010B50446FCF7A0FF2046054B8F
:10DF500040F8283B14F08EFF2046034944F03AF97C
:10DF6000204610BD983A0D08303A0D081820704729
:10DF700000487047003B0D0800487047083B0D08FB
:10DF800001207047012070470120704708B50548FF
:10DF9000F5F788FE0348F5F767FDBDE8084001483E
:10DFA000F5F746BB702B002008B5064881F090FCC1
:10DFB000BCEEC00A044810EE103A99B2BDE8084021
:10DFC00001F07EB8F8540020702B002010B50D4CE5
:10DFD000D4F8703B002B12DDA4F50050FAF7FAFBE1
:10DFE000A4F5005000F066FB04F6881081F0BAFD3D
:10DFF00004F68810044981F053F9012010BD002077
:10E00000FCE700BF704B002088820020F0B5274E4F
:10E01000D6F8C40E03688FB05B689847072837D0DE
:10E020000A2809D0062805D10FF0A0FA90F87C3212
:10E03000DB071DD4012019E006F5805707F25C5577
:10E040000FCD07AC0FC495E8070084E8070009ABC3
:10E050000FCB01AC84E80F00D7F82437009305F507
:10E06000D6730ECB06F66840FEF7E4F90FB0F0BDAC
:10E070000FF07CFA00F51B700FC801AC84E80F00AC
:10E0800006F58055D5F82437009305F5E363E8E7F6
:10E0900007A906F6DC30FDF7F5FE0028CAD007997F
:10E0A00006F66840FEF7A4F9E0E700BF706B0020B9
:10E0B000F0B585B00E4E0391144656F021FC06F5DE
:10E0C00080470546D7F8C40E026892689047039BC4
:10E0D0000090084A284606214FF0B6FDD7F8C41E26
:10E0E0002246304605B0BDE8F04008F037BE00BF1C
:10E0F000702B0020103B0D082DE9F0432DED028B15
:10E1000097B0002507466D4881F00CFC05950695F3
:10E1100007950FF02BFA05A90EF05EFF70B3684B60
:10E1200093ED007AB5EEC07AA3F66C39F1EE10FAF1
:10E1300009F5005427DBDDED067ADDED056A67EEB3
:10E14000A77A27EE077AE6EEA67AF4EEC77AF1EE22
:10E1500010FA18DDD4F8C40E03685B6898470A28E3
:10E1600011D056F0CDFB574A06214FF06DFD262207
:10E1700004F64C41A4F5804008F0F0FD17B0BDEC6A
:10E18000028BBDE8F083504BD4F8C44E01959C42FD
:10E1900002950395049503F5787817D104F63C149D
:10E1A0000FCC08AE0FC694E8070086E8070011A858
:10E1B00014F060FEB8F8B4150FAA08F5A4602BF0AF
:10E1C00065FC78BB02950195049503959FED3F0A88
:10E1D00001A828F049FD03A88DED080A9FED3B0A30
:10E1E000CDED090A28F040FD34488DED0F0AB0EE60
:10E1F000401AF0EE601ACDED100A9DED080ADDED33
:10E20000090A81F0E9FA0628044618D10023C8F863
:10E21000CC3683F03FFE2E49C8F81C0B274881F00E
:10E220003FF8ABE701A911A814F0D0FF0028C9D02E
:10E2300003A90AA814F0CAFF0028C3D0C6E709F64C
:10E24000C82983F027FEDFED237A99ED008AD8F8FC
:10E250001C6B28EE278ADFED207AB4EEE78AF1EE18
:10E2600010FA0546384658BFB0EE678AFFF7CEFE73
:10E2700048B9022C16D0BCEEC88AAD1B18EE103A75
:10E280009D42FFF47BAF013C062C0ED8DFE804F082
:10E29000040A0D0D100D1300104924223846FFF713
:10E2A00007FF6BE70E492522F8E70E491622F5E72E
:10E2B0000D492622F2E70D490122EFE7F85400202C
:10E2C000DC5600202C3B0D08907700200000C8424F
:10E2D0008882002000007A4400409C46523B0D0892
:10E2E000673B0D087C3B0D08943B0D08AB3B0D08CC
:10E2F0000320704700487047303C0D0800487047C5
:10E300003C3C0D08F8B52A4D06460027A5F54050BF
:10E31000A5F88073F5F70CFCB369A5F58052D3F826
:10E32000F811D2F8E03B994205F5005421DBC4F81E
:10E330001035B36992ED5A7AD3ED7F6A9FED1D6A6D
:10E34000F8EEE66A27EE067AF4EEC76AF1EE10FA06
:10E3500018DBBDEEC77A17EE103A1748C4F814352B
:10E36000FBF778FB20B1D4F814355B42C4F81435C0
:10E37000F8BD5B429942DADD012385F88033C4F8A9
:10E380001075D6E702F6E432D2ED007A67EE867AAF
:10E39000F4EEE76AF1EE10FA93BFFDEEE77A01239F
:10E3A00085F8813317EE903A88BF0023D5E700BF88
:10E3B000705B00200000C842702B002070B5002167
:10E3C0002DED028B04463448344D06F003FF3248ED
:10E3D0000021F0EE408A06F007FF95F88033B0EE9A
:10E3E000408AD3B1B0EE680A042059F03DF895F8A0
:10E3F000813393B3B0EE480A132059F035F826481C
:10E40000002106F0FBFE2046FCF766FEBDEC028B09
:10E410002046BDE87040FCF771BE05F50056A5F535
:10E420004050F4F755FED6F81035002B0CDCD6F82A
:10E430001035002BDBDA042059F02AF8B4EEE80A94
:10E44000F1EE10FACED4D2E7042059F021F8B4EE60
:10E45000E80AF1EE10FAEADDC4E7114D0E48F4F7D0
:10E4600029FFD5F81435002B0CDCD5F81435002B1A
:10E47000C5DA132059F00CF8B4EEC80AF1EE10FA20
:10E48000B8D4BCE7132059F003F8B4EEC80AF1EE93
:10E4900010FAEADDAEE700BF702B0020705B0020B1
